:020000040800F2
:10000000F0FF00100DAF06083D31060879CF01085A
:10001000ADAF0608ADAF0608ADAF060800000000A2
:100020000000000000000000000000004131060850
:1000300045310608000000004931060881BF01086B
:10004000ADAF0608ADAF0608ADAF0608ADAF060808
:10005000ADAF0608ADAF060889AE000891AE000846
:1000600099AE0008A1AE0008A9AE000835AB0008A3
:1000700049AB00085DAB000871AB000885AB000818
:1000800099AB0008ADAB0008ADAF0608ADAF0608F0
:10009000ADAF0608ADAF0608ADAF0608B1AE0008BB
:1000A0009DC40008FDC30008ADC40008EDC30008EE
:1000B00025C4000835C4000845C400081DA2000876
:1000C000B1B9000825A20008B5B90008ADAF06080F
:1000D000ADAF0608B5B80108B9B90108BDBA010845
:1000E000B9AE0008ADAF0608896B0608BDC40008AC
:1000F00075C40008CDC4000865C40008C1AB000881
:10010000ADAF0608ADAF060855C40008ADAF060890
:10011000C1BB0108C5BC010881D90008B9D90008D4
:10012000D5AB0008E9AB0008FDAB000811AC000836
:1001300025AC0008ADAF0608ADAF0608ADAF0608A8
:10014000ADAF0608ADAF0608ADAF06084D310608E5
:1001500039AC00084DAC000861AC0008C9BD01080D
:100160002DA20008B9B90008ADAF0608ADAF06086A
:10017000ADAF0608ADAF0608ADAF0608ADAF0608D7
:08018000ADAF0608ADAF0608A3
:10800000074BD0F8E4105B68D0F8F0205B1A9A4276
:10801000B8BFC0F8F030012380F81C310020704751
:10802000001000E0B74B00EB800270B503EBC20418
:1080300053F832205268B2F814C01CF0010F4FEA16
:1080400080016AD15FFA8CFE1EF0020F3DD0BFF3B3
:108050005F8F257F012D5FFA85FC00F0CC80148BAB
:10806000BFF35F8F0C1803EBC404257F022D00F0D3
:10807000E3800C1803EBC404257F032D06D1A47FF5
:1080800024B193F87940002C40F0E5809488A4B2A4
:1080900044F48064948093F978C001EB000E03EB04
:1080A000CE0E9EF81CE00EF1010EE6450CD1002428
:1080B00083F8794093F87A40002C40F0B680084469
:1080C00003EBC00300225A7670BD1EF0040F5BD193
:1080D0001EF0400E00F0C880158A93F978C0666AD9
:1080E000EDB206F80C505FFA8CFE267F0EF101040B
:1080F00064B2E51CAE4283F87840A44600F02A81C1
:108100000D1803EBC5052D7FAC42C6D10EF1020C54
:108110004FFA8CFC83F878C0BFE7B2F800C02CF4AB
:10812000006C4FEA0C4C4FEA1C4CA2F800C0B2F8AD
:1081300000C01FFA8CFC4CF4806CA2F800C0A57F34
:108140004FF0000C83F878C0002D46D093F879509A
:10815000002D3FD0012483F879400C1803EBC404B0
:10816000247F022C04D11488A4B244F40064148047
:108170000C1803EBC404A47E44F0010414820844E8
:1081800003EBC0031B7F70BDA57F4FF0010C83F88C
:108190007AC0002D6FD093F87950002D70D10C1853
:1081A00003EBC404647F002C00F0AE80148893F8C5
:1081B00078C0A4B244F400740CF1010C14804FFA9E
:1081C0008CF483F87840B2F800C01CF4807FFAD1B8
:1081D000A44662E7E47EFF2CBCD00C1803EBC40479
:1081E000A57E05F0FE051582E27EFF2AC7D0FF229C
:1081F00083F87820C3E7A47F002C3FF430AF93F8D6
:108200007940002C3FF42BAF148824F480642404BC
:10821000240C1480BFF35F8F148B148883F87AC00A
:10822000A4B244F40074148030E7948824F44074B9
:108230002404240C948042E7A47F002C3FF419AF5F
:1082400093F87940002C3FF414AF148824F4806430
:108250002404240C1480948824F480642404240CC2
:10826000948093F978C018E71FFA8CF52D0631D465
:1082700093F978C011E793F87940002C8FD095E7F7
:10828000257F022D15884AD925F480652D042D0CF3
:108290001580158A666A93F978C0EDB206F80C501D
:1082A000666A1488A4B244F4007414805FFA8CFCEB
:1082B000158A0CF1010464B2EDB2355595880CF1C4
:1082C000020CADB24FFA8CF445F4806583F8784027
:1082D000958078E793F978506E1C42D0266A765DD7
:1082E0001682247F05F1010C4FFA8CFC644583F85B
:1082F00078C07FF4D2AE948824F480642404240CE3
:108300009480CAE6B01A00201488A4B244F48074A1
:108310001480012483F8794093F9784053E7ADB293
:1083200045F400751580158A666A93F978C0EDB238
:1083300006F80C505FFA8CFC666A158A0CF1010491
:1083400064B2EDB20CF1030C35554FFA8CF483F89E
:10835000784038E7958825F480652D042D0C9580AC
:10836000CEE6E57E1582A57F83F878E01DB9247FEF
:10837000002C7FF404AF948824F480642404240C3B
:108380009480FCE61B4B01681B4A03F5727C03E0FA
:1083900063452CD053F82C2F9142F9D170B593F846
:1083A00004E0427996450AD0634505D053F82C2F56
:1083B0009142F4D06345F9D14FF0FF3070BD9E4635
:1083C0008468DEF80C50A5424FF0000208D001325C
:1083D000032A0EF10C0EE7D0DEF80C50A542F6D1C0
:1083E000DEF81050C668B542F1D150B270BD4FF002
:1083F000FF3070478CCA06080000014030B5EAB172
:108400008E464FEA014C034600F1C005002419686E
:108410009A6841EA0C0142EA0E029A60C3E900142C
:108420000C33AB42F3D1D0F8C030C0F8C44043EABB
:108430000E03C0F8C030C0F8C84030BD4FEA014E4E
:108440008C46E0E783691969B3F80CC00A6830B458
:108450009C6822F0010224680A60A28992B222EA92
:108460000C02A281027D04681F2A06D96568203AA1
:1084700008209040284245D0FEE72568082090401B
:108480002842F9D1202000FA02F2A260264A12788E
:10849000002A35D01A7E012A39D0D3F8F4200132CF
:1084A000C3F8F420EFF31181502282F31288586848
:1084B0005C6C026822EA04029C6C2243C9B202602E
:1084C00081F31188D3E90C401A6999681D6C096819
:1084D00014605061D3E90E40546090600024B3F8FA
:1084E000A800D5604C62C862106801242043106067
:1084F0001C7683F8F1408A899B8913439BB28B8158
:1085000030BC7047202000FA02F2E260BEE7002291
:1085100083F8F120D3F8F8000A68013022F0010254
:10852000C3F8F8000A60EBE70400001010B40C4C2C
:108530006368002B11DD002004F1080C0146DCF813
:10854000A03003F1C00259600C339342FBD1636841
:10855000013083420CF5807CF1DC5DF8044B704700
:1085600004000010F0B5494C04EB401C9CF8242496
:1085700002B9F0BD464B4FF08C0E0EFB003E93F857
:10858000DC6493F8DD249EF87E708CF80A749642C1
:108590004FF0000C4FEA40158EF87EC00ED002EB73
:1085A000420C03EBCC0C57009CF8E0C40CF1FF3EEE
:1085B000BEF1010F5CD9BCF1030F53D06019A0F8D4
:1085C0000814EFF31182902383F3128890F80A3491
:1085D000B0F8081443EA41030021D2B29BB280F8FC
:1085E0000A1482F311881A09217882EA13225A4068
:1085F000D9B1D0F82044D0F80C14D4F8A040D2431C
:108600001B019BB202F00F0201208840134304F1CA
:10861000C0015A0013F4004F93B202D162680243C2
:1086200062600C348C42F4D1F0BDD0F82014D0F844
:108630000C04D1F8A0401B0100F110019BB202F024
:108640000F0201208840134304F1C0015A0013F4C3
:10865000004F93B202D16268024362600C34A142BF
:10866000F4D1F0BD02F1010C0CF0030CB445A5D01F
:108670003A4403EBC202131893F8ED1400299DD07D
:108680006319012283F80A2498E700BF0400001050
:10869000B01A0020704700BF024B03EB401090F867
:1086A00025047047040000104368B0F8502010B44F
:1086B0001A83EFF31182502383F312884168446CCC
:1086C0000B6823EA0403C46C2343D2B20B6082F329
:1086D0001188D0E907418268036912681C605961FA
:1086E000D0E909415C60C46A9960B0F86010DC6050
:1086F0000023D1625DF8044B0376704710B4037D0C
:1087000001681F2B09D94C68203B202202FA03F391
:108710001C4215D15DF8044B70470C68202202FA08
:1087200003F31C42F6D00D4A4068002482F840450D
:1087300002685DF8044B22F0010202608B60704712
:10874000064A4068002482F8404502685DF8044B00
:1087500022F001020260CB60704700BFB01A002017
:10876000704700BF0B4890F83C1589B101EB4101FF
:10877000002310B4490000F244501C4650F8232056
:10878000063302B114608B42F8D15DF8044B704798
:10879000704700BF040000100B4890F83C1589B1E9
:1087A00001EB4101002310B4490000F244501C4683
:1087B00050F82320063302B114609942F8D15DF8D5
:1087C000044B7047704700BF040000100120704741
:1087D000034B00EB400003EBC00090F855057047D9
:1087E000040000101F4890F83C35002B39D00022BF
:1087F0002DE9F04300F244531B4E1C4D4FF0500E38
:108800004FF02C0C144607E053F8181B0C6090F83E
:108810003C150132914222DD197C0029F4D05F68B9
:10882000B90AA1F5801105EB010952294FF0FE08A4
:1088300098BF99F8F483EFF311898EF31288796A5F
:108840000CFB08680131C8F86C15B98A89B241F08F
:1088500001015FFA89F8B98288F31188D4E7BDE88D
:10886000F083704704000010B01A00208CCA06087C
:1088700007EE900AB8EE670A704700BFBCEEC00A68
:1088800010EE103A98B270470D4B0E49DB68DB438F
:10889000C3F30223C3F104030122DBB202FA03F3A0
:1088A00001EB000C1B0103F0F0038CF800334309CB
:1088B00000F01F0002FA00F041F82300704700BFEB
:1088C00000ED00E000E100E0037D1F2B08D9026805
:1088D000203B5168202202FA03F3194214D1704759
:1088E00001682022096802FA03F31942F7D00D4A01
:1088F00041684FF0000C82F8ACC70A68006822F0AB
:1089000001020A6083607047064A41684FF0000C1C
:1089100082F8ACC70A68006822F001020A60C360EE
:10892000704700BFB01A0020122301480B80704727
:1089300088010020042301480B8070479C0100201F
:108940002048D0F8E837D0F8EC2730B59B184FF026
:108950001A040C8001D11C4830BD1B4AD0F8EA171C
:108960004FF0000E10467546B3F1204F4FEA137CCE
:108970000CF130040EF1020E2ABF0CF1370C84709A
:1089800080F802C0BEF1100FC5704FEA031300F16A
:108990000200E9D100200446B1F1204F4FEA1173E3
:1089A00003F1300C00F102002ABF373382F812C005
:1089B00093740828D4744FEA011102F10202EBD13A
:1089C000014830BD00F0FF1FA0010020B4228280CA
:1089D0002A224FF4A57C4FF4EB7102814FF4877289
:1089E0000023A0F802C0C1804FF4E17C962182816F
:1089F00044220370A0F80AC0C181028243827047FA
:108A000082B01F4B002201920193019B1D4A043347
:108A10000193019B1968936803F00C03042B07D0A2
:108A2000082B0AD0184B194AC3F8B02702B0704778
:108A3000154BC3F8B01702B070475368506813F471
:108A4000800F00F03F00536813D1C3F388130F4920
:108A5000B1FBF0F101FB03F30A4A0B495268C2F380
:108A6000014201325200B3FBF2F3C1F8B03702B059
:108A70007047C3F38813B1FBF0F101FB03F3EBE79D
:108A80005028004000380240B01A00200024F400B2
:108A90000123437700207047D0E90B2108B5836993
:108AA0000B4483610AB108469047002008BD00BF0F
:108AB000436A1B681B6A5B685B78024613F001001F
:108AC00008BF5077704700BF70B5224A224C234B35
:108AD00094B00546CDE90042214A0992A4F108026A
:108AE0000A922A7F0493201D0023CDE905039A42B0
:108AF000CDE90E330B931093139314BF052004207C
:108B000011936B6A0C9002200122029018688DF874
:108B10000C200E4607928DF820208DF834208DF819
:108B2000482060F089FF2B7F93B1330E04F8073C97
:108B3000063C320C330A22706370A670686A69467C
:108B400011F0C2FC6B6A186860F076FF14B070BD5B
:108B5000073CEEE764220020C4010020B18A00082F
:108B6000918A000810B5044694B050220649684620
:108B700063F0C4FE606A694611F0A6FC636A186877
:108B800060F05AFF14B010BDD4CE0608C2628161F5
:108B9000704700BF2DE9F0410446406A00681E4658
:108BA0000F46904660F048FF237F002B3FD02A4DB0
:108BB000A0690523EB67030E85F8453005F14603F0
:108BC0009870020C000A58701A703B68C5F888301B
:108BD0000020D8F80030C5F89030012E2363C5F886
:108BE000A0002BD0022E20D1D8F80420C5F8980080
:108BF000796885F89400C5F89C1013441749C5F8A6
:108C0000A4200120236385F8A800C5F8AC10144BFC
:108C1000617F606A03F11402002914BF19461146EE
:108C200011F052FCE36A8BB1206BBDE8F0810A4D74
:108C3000A0690423EB6705F14503C1E7074B85F8FD
:108C40009460C5E92630C5F8A400E0E7636A1868B7
:108C500060F0F2FEE8E700BF88010020998A000872
:108C6000D4010020704700BF00B583B0816101923C
:108C7000049A0093C26201236A4601A9FFF78AFFA2
:108C800003B05DF804FB00BF043070470D4B93F850
:108C9000BC27D3F8B8170244D2B283F8BC2793F8A4
:108CA000BC2708441206C3F8B80705D593F8BC27BB
:108CB00082F0800283F8BC27034B012283F8C42092
:108CC000704700BFB01A0020880100202DE9F0474E
:108CD000144FD7F8C057ED0A1ED00026B04607F54E
:108CE000FF69D7F8C4371048D3F828A0C7F8F08731
:108CF000AC19641010234A46E102D0470F280BDD5F
:108D00000A4B03F1100C53F8041B013107D16345E2
:108D1000F9D12546B542E4DCE802BDE8F087661CDF
:108D2000F8E700BFB01A002074220020A82200201B
:108D30001C4BD3F80818D3F80C288A1A322A16D8F4
:108D4000D3F820288A4200D37047D3F8142822B3DE
:108D50001068928810B444693231224218BF4283AD
:108D60005DF8044B08BF0283C3F82018704793F8DE
:108D70001028D3F8141802F0010219B132B90A68A8
:108D8000898811830022C3F8202870470A688988DF
:108D900051830022C3F8202870473231C3F82018CD
:108DA000704700BFB01A0020094A92F81038D2F874
:108DB000142803F001031AB123B9136892881A83A7
:108DC00000207047136892885A830020704700BFC4
:108DD000B01A00204FF40070034B1060D3F8303805
:108DE0000B600020704700BFB01A002000207047C1
:108DF00001207047012070470020704710B51C69A2
:108E000094420DD396468A188C469442996938BF8D
:108E1000A4EB0E0C71446246BDE8104063F06EBDD9
:108E200010BD00BF30B4194B00209C7B14B11D68ED
:108E30008D4206D001300B2803F11003F5D130BC70
:108E400070479AB1124B03EB40218A4219D0114B63
:108E500093F8E4278AB1104B01225A7000F5B170E3
:108E600003EB00100123837130BC70470A4B00F5FF
:108E7000B17003EB00108271E1E7012283F8E4276F
:108E8000E9E7022CE3D1183BE8E700BF0C590020CA
:108E90000C430020F4520020F442002030B41D4C5A
:108EA000002384F8D03604F5C36004E001330B2BB3
:108EB00000F1100015D005688D42F7D190F80EC072
:108EC000BCF1030FF2D1C2B1134901EB432082423E
:108ED00009D1A1F1180203F5B17302EB03130122CA
:108EE0009A7130BC704794F8E42712B9012284F8D3
:108EF000E4270A4A01215170EDE70849D4F8CC264D
:108F000003F5B17301EB0313013204219971C4F825
:108F1000CC26E6E7F45200200C430020F442002067
:108F2000A8B183681BB10E4B07229A7070470C4A98
:108F30001178D36003294FF004000CBF80214FF457
:108F40008071C2E901111361137590707047044A72
:108F500002F580510123537081F8E437704700BF58
:108F6000F44200202DE9F0430446406A344D006885
:108F700095B00E469146984660F05EFD314B0193E8
:108F8000314B049305F1D0030093217F0223029318
:108F900005F1C802012300278DF80C3005920697D1
:108FA000002936D08DF834308DF84830CDE9097776
:108FB000330ECDE90E77CDE9107785F8C93005235A
:108FC000CDF82C908DF82070CDF830801397CA35ED
:108FD0000793330C1D4F2B70330A6B70AE70D7F8AC
:108FE0006408656A11F028FC637FA88033BB05A97B
:108FF000284611F069FA636A186860F01DFDD7F819
:10900000680811F019FC636A9880404615B0BDE805
:10901000F0838DF834308DF848300423CDE9091100
:10902000CDE90E11CDE91011CDF82C908DF820105E
:10903000CDF830801391C9350793CAE76946D7E761
:109040008801002010230020B18A0008B01A0020F7
:1090500070B5224B93F8DC2493F8DD349A4237D173
:109060001F4D95F80436E3B195F808461D4B0020D6
:1090700040F20D3CB4B19A6899895160166819683C
:1090800046F001061660A1F848C08A8992B242F4FF
:1090900080728A8195F804260130824203F1180318
:1090A000E8DC70BD1A68118821F080010904090C00
:1090B00011809988D162118889B241F080011180B4
:1090C0005462998A9689314389B291819C82E1E701
:1090D0005FF042F80028C3D170BD00BFB01A002075
:1090E000040000101C2300202DE9F0411E4B93F8D2
:1090F000DC2493F8DD349A422FD11C4F7D68002D7B
:1091000012DD3846002410F8086BA046013416B171
:10911000037E012B1CD002691368AC4243F00103AB
:1091200000F580701360F1D112F074FFD7F80C468F
:10913000002C0BDD0E4A02EBC40411689388888969
:10914000083203439BB294428B81F6D1BDE8F08193
:1091500080F8F080FFF7A8FADDE75EF0FDFF002859
:10916000CBD1BDE8F08100BFB01A00200400001090
:10917000140600102DE9F04F037D02681F2B83B009
:10918000044609D95068A3F120052021A9400142D5
:1091900007D103B0BDE8F08F10682021994001424B
:1091A000F7D05149514D4968C5F8301695F8081661
:1091B000A7694F4E19BB8C2101FB0761D1F88400D0
:1091C000D1F8FCE0D0F800C0DEF80000B1F88880EB
:1091D00020F00100CEF80000BCF80C1089B221EAA2
:1091E0000801ACF80C10297801BB1F2B6FD9A3F133
:1091F000200120238B40D36003B0BDE8F08F8C2189
:1092000001FB0761D1F88410D1F810C00868DCF8C0
:10921000001021F00101CCF80010818921F4807147
:109220000904090C818129780029DED04FF08C08CF
:1092300008FB07F806EB08032E49D3F8FCA0D3F887
:1092400084200193504608F11809D2F800B08944EF
:1092500059F05AFC019BD5F838262649012083F89D
:10926000D000002A3AD0BBF800309BB243F0800314
:10927000ABF8003008F174084FF0FF334144CBF8ED
:109280002C30584659F0C6FD8C2303FB076600239B
:109290004946C6F8A030504659F0CCFCD6F8FC3010
:1092A00016225A601A6842F001021A60D6F8842029
:1092B000B6F88830126891890B439BB293810A49B2
:1092C000237D49682268C5F834161F2B8FD82021CA
:1092D00001FA03F3936003B0BDE8F08F12F09AFE39
:1092E0000449C5F83806BEE7001000E0040000108D
:1092F000B01A00202C1B00202DE9F04112F08AFE4C
:109300001F4F204E05464FF000087C68002C2ADDD8
:1093100000231A4607EB0321013391F8F9109C4210
:1093200042EA0102F6D142EA0804E4B290467368C8
:10933000C3F30803A3B9EFF311838BB912F0B8FE9E
:10934000431BB3F5FA6F02DCB8F1000FDDD124B195
:109350000D4B93F82C29542A09D02046BDE8F08102
:1093600012F02CFEECE744464FF00008DFE7B3F8BC
:1093700034290132A3F834292046BDE8F08100BF2A
:109380000400001000ED00E0B01A0020BC4B1B7878
:109390000BB9012070472DE9F04FBA4DBA49D5F805
:1093A0000828BA4BA1FB02125209A3FB023A4FEA6A
:1093B000DA0A0AEB8A0AA2EB4A0A85B0B04A5FFAD7
:1093C0008AF3039302F61C1302F23C670193002315
:1093D00007EB8A0A02F581699846A94BD3F8243A2B
:1093E000434540F31781D9F81830D9F80460D3E920
:1093F0003A34029312F00EFE029B95F82CC90290AB
:109400004FEA860E95F840090EF1085E04F180617E
:109410000EEB431E3939BCF1540F0EEB81110EEBEC
:10942000801301D1A5F83609994240F26A811A6881
:10943000002A00F05E811A6C002A00F07081D3F8D7
:109440008020002A00F06D81D3F8C02003F58073DE
:10945000002AE9D1A3EB0E0E99424FEAAE1E40F26C
:109460005081A4EB0E0145294FF0000428BF45218F
:1094700003EB81119B46204626460DE01A6C002A1C
:1094800040F0D080D3F88020002A40F0F680D3F856
:10949000C02003F580732AB9994206D91A68002AB8
:1094A000ECD04033994200F2C180112E344640F294
:1094B0002C81D6F1150200F128817549029ED1F860
:1094C000D4309E45D5F8443938BFC1F8D4E0F11AFC
:1094D000002919DB03F5F42303F590739E4288BF3E
:1094E000029B6B4988BF0533C5F84439684BD3F8F4
:1094F000D430052B86BF053BDBB2002385F840390D
:109500004FF0FF33C1F8D43042B100FA02F2C4F197
:109510001404012000FA04F444EA02005D4BC0F395
:10952000C43203EB8202D2F8981400F01F0203EB5E
:109530008202D2F8982442EA0131C0F3441203EBCC
:109540008202C0F3842003EB8000D2F8983441EA11
:109550000311D0F8983441EA032181EA112383EA08
:10956000131303F00F030F2B40F0B180B1F5803FD0
:1095700080F0AD80BCF1540F4FEA111104D1B5F861
:1095800030390133A5F830393D4AD2F82439B1F5E4
:10959000606F03F10103C2F8243900F0D480019B0D
:1095A000998197F858300398834210D0DAF8082050
:1095B0003B689B1A3B60DAF830207B689B1A7B6023
:1095C0000023CAF80830CAF8303087F858003B68E2
:1095D00001333B60DAF808300133CAF808304FF63F
:1095E000FF73994207D17B6801337B60DAF8303032
:1095F0000133CAF83030019B08F101081433B8F187
:10960000080F07F15C070AF15C0A019309F12009D0
:109610007FF4E3AE1A4A0123012082F8203A05B014
:10962000BDE8F08F803399427FF63FAF5A469A1AD1
:109630009211541C184A82FB04B2A2EBE472012A74
:10964000B8BF0122904001241644013A04FA02F204
:1096500010431C4622680AB3226C002A63D0D4F857
:109660008020002A61D0D4F8C02004F58074B2B103
:10967000A142EFD89B4623460EE7C03312E700BF56
:1096800004000010B01A00201F85EB51CDCCCCCCCB
:10969000880100208CCA0608565555554034A14211
:1096A000E8D9E31A9B115A1C2F4B83FB02B3A3EB9F
:1096B000E273012BB8BF012398401E440122013BF5
:1096C00002FA03F3184323469B462346E4E6BCF123
:1096D000540F2CD0254AD2F824390133C2F824394A
:1096E000224AD2F820390133C2F820394FF6FF71EF
:1096F00057E74033A3EB0E0E99424FEAAE1E3FF6FA
:10970000B0AE10B1013885F84009BCF1540F7FF4B8
:1097100072AFB5F832390133A5F832396BE78033CF
:1097200098E6C03396E68034B9E7C034B7E7B5F8B9
:1097300030390E4A0133A5F83039D2F824390133D3
:10974000C2F82439CCE795F8DD3403EB430305EB8D
:10975000C303434493F8ED340D2B7FF420AF019AFB
:10976000802393771DE700BF565555550400001020
:1097700010B5044662F04AFB81B22046BDE81040B5
:10978000FEF7F0BE38B50B4D00EB400005F2445338
:1097900003EBC00393ED027AD3ED037AE7EE007A90
:1097A000C4002C44B0EE670A62F030FBD4F84435B4
:1097B000186038BD040000100C4AF8B513685569EC
:1097C0002B4003EA000555617DB1094F0126B5FA2A
:1097D00085F4C4F11F0407EB840306FA04F4D3F8FC
:1097E000480903689847A543F1D1F8BD003C014002
:1097F000B01A0020038A2DE9F047B0F80C901FFA48
:1098000089F919EA03092BD005460E464FF00047A7
:109810004FF00008B9FA89F327FA03F2D24391B264
:109820001B3B298209EA0209042B16D8DFE803F062
:10983000352C231A0300B36A002B37D003F1FF3A0B
:109840001FFA8AFAC6F82880746A34B12368204661
:10985000514698476468002CF8D1B9F1000FD9D16E
:10986000BDE8F0877068696B036889B29847B9F101
:10987000000FCFD1F4E7B068A96B036889B29847AD
:10988000B9F1000FC6D1EBE7F068E96B036889B264
:109890009847B9F1000FBDD1E2E73069296C036840
:1098A00089B29847B9F1000FB4D1D9E7E96A1FFA34
:1098B00081FAC9E70A4608B5054920B9054859F0B3
:1098C000CFFB034808BD044859F0CAFB004808BD57
:1098D00038240020A85C0708D05C070810B5044CA9
:1098E00004480A46214659F0BBFB204610BD00BF84
:1098F00038240020F85C070810B5044C04480A46D8
:10990000214659F0ADFB204610BD00BF3824002091
:109910000C5D070810B5044C04480A46214659F06E
:109920009FFB204610BD00BF38240020185D0708AB
:1099300038B590F82830012B044604D0407F40B160
:109940000023637738BD406A03681A7B92B9637F4E
:109950000BB9012038BD0A4D0A49022305F68822B9
:1099600010F050FE95F8893A03F0010383F00100EE
:109970006377E7E71B6A002BE9D0002038BD00BF02
:10998000B01A0020600200202DE9F0410446154E77
:1099900090F82800637F144F06F68828012805D028
:1099A0000BB1002363770120BDE8F081606A056890
:1099B0002A7B82B9002BF6D002234246394610F0AA
:1099C00021FE96F8893A03F001036377002BEAD071
:1099D00094F82800E2E72A6A002AE8D1002BE2D0B6
:1099E000EAE700BFB01A002060020020F0B511F0D5
:1099F000010583B00AD190F82860012E044607D0F3
:109A0000C368B3F1807F01D90123237703B0F0BD90
:109A10000A4B476AD3F8640810F00EFFE368B88079
:109A2000B3F1807FF2D9B7218DF804102677334641
:109A30002A46384601A910F0E5FDE7E7B01A0020F4
:109A40002DE9F047089F884615460021202204464C
:109A50001E4662F0B6FF4FB13B68E3811B0C2382C8
:109A60007B687A89E3821B0C62822383404660F024
:109A70004DFBEB0619D4431EB8B108EB000701E01B
:109A8000013B12D317F801CDBCF12E0FF8D1C01A4B
:109A9000421E032AA8BF0322082B03F1010AA8BF14
:109AA00008239146C2441A4606E008280246C246E8
:109AB000A8BF08224FF000094FF020334146236031
:109AC000636004F10807204662F018FF174B2381FA
:109AD0005146BB704A46384662F010FF611EE31DD6
:109AE00011F801CFACF1610EBEF1190F9CBFACF1C2
:109AF000200C81F800C08B42F2D1384604F10B01F2
:109B000010F8013BA3F16102192A9CBF203B00F829
:109B1000013C8842F4D118232373330CA382E572ED
:109B2000099B6683E361BDE8F08700BF2020200029
:109B30002DE9F04FDFF88894D9F80808C9F80C0827
:109B400087B0002B00F0DA8001F5FE781344DFF8CF
:109B500074B40393164601F12007C24621E0002E9B
:109B600064D0D9F83C38B34200F0CC80D9F838380A
:109B7000B34200F0FF80D9F84038D9F84418B34216
:109B80004BD8B14200F29981711A20465DF080FCF9
:109B9000039B01369E4207F500770AF5007A00F034
:109BA000AD80D9F84858B542A7F12004D7D8751B25
:109BB000D9F8588805F00702EB080492D8F830204D
:109BC0000233934203D3D8F8382093420BD941464D
:109BD000184605935DF02CFC059B8046002800F09C
:109BE0008C81C9F8580898F80420002A40F0348184
:109BF000D8F82850002D00F07981D8F830209B1A31
:109C0000049A02EBC303D8F80C20204602EB43224F
:109C10004FF400714346A847BAE7B142B4D9204691
:109C20004FF40072002162F0CCFEB1E74FF40072F5
:109C30003146204662F0C5FE802387F89E310C2312
:109C400087F8A231D9F83838D44AD9F83018C4F88E
:109C5000C6319342C4F8CA1100F33481D04AD14CC2
:109C600082FB03021A44D817C0EB621284FB025431
:109C7000CD4D85FB03C5C0EB2530C2EB821587F8BF
:109C8000A1015B1B801020F03F000133034314440B
:109C900087F8A031D317C3EBE4142244BF4B87F8F5
:109CA0009F214A1E9A4200F31981BD4BBD4883FB98
:109CB00002311144D317C3EB611180FB0140BA4C50
:109CC00084FB0254C3EB2433C1EB811487F8A53124
:109CD000121B9B1023F03F0301321343084487F803
:109CE000A431CB17C3EBE010014487F8A31155232F
:109CF00087F8DE31AA2387F8DF3149E7002007B073
:109D0000BDE8F08F4FF0FF3384F8EC3184F8ED318B
:109D100084F8EE3184F8EF31D9F85038C4F8E831DE
:109D20005223237063706123A37084F8E7314123C9
:109D30000025E37084F8E631722384F8E43184F876
:109D4000E5314FF4F0722946A7F11C0062F039FEAC
:109D50005523C7F8D051C7F8D451C7F8D85184F863
:109D6000FE316FF0550384F8FC5184F8FD5184F8FE
:109D7000FF310DE700214FF40072204662F021FE12
:109D80008A4A03CA47F81D0CEB2007F8200C58201C
:109D900007F81F0C902047F8191C07F81E0C002329
:109DA00002220821F820E372227307F8131CA27321
:109DB000E37307F8102C07F80B0CD9F8380884F86F
:109DC0002C20D9F830286376121A2262D9F840087C
:109DD000D9F84428E376121A3F2020764FF0FF305E
:109DE000A0763E20207701206377A377E37784F87D
:109DF0002D3084F82E3084F82F30626284F83000E1
:109E000084F8313087F82610802187F82010292126
:109E100087F82210942187F823100E2187F8241048
:109E20000D21634A87F82510552187F8DE11AA21F4
:109E300087F8DF1103CA5F4BC7F82700C7F82B105C
:109E400003CB1388A7F82F309378C7F83200C7F8F0
:109E5000361087F831309BE64FF40072002120461F
:109E600062F0AFFD049B002B4ED1D8F84030002BA0
:109E700000F0AA80049AD8F830304F49CDE900228A
:109E800020461122FFF7DCFDD8F840301A6C002A7A
:109E900000F0AD80049A1B6BCDE9002247491122E6
:109EA0003846FFF7CDFDD8F8448007F120044FF481
:109EB000E075B8F1000F3FD16AE6F11A20465DF077
:109EC000E7FA65E6FF2387F89F3187F8A13187F825
:109ED000A031324B4A1E9A427FF7E7AEFF2387F844
:109EE000A33187F8A53187F8A43100E72946204639
:109EF0004FF4007262F065FD4AE6A7F1240343F8CF
:109F000004BF9A45FBD143E6D8F84030049AD8F80C
:109F10004480002B0CBF01230223C3EB02154346F0
:109F2000002B3FF435AE013D9B6CF9D198464FF4C0
:109F30000075002B3FF42CAE2544203423462035F9
:109F40004446049698460EE05CF81C1B236BCDF843
:109F500000C000260196FFF773FDA46C08F12008ED
:109F6000CCB1A84517D02379A44604F11C0E1122C8
:109F7000A8F12000002BE7D162792669236B2168C4
:109F800042F02102CDE900E6FFF75AFDA46C08F18A
:109F90002008002CE5D1049EFAE500BFFF03FB007A
:109FA000832008828180808097554541305D070875
:109FB0003C5D0708485D0708285D07082C5D070819
:109FC000B01A0020DEADBEEF049BD9F83418CDE9FD
:109FD000003320460822FFF733FDD8F84480B8F15B
:109FE000000F3FF4D5AD3C464FF4F075A4E7049B59
:109FF000CDE9003352E7084B10B5D3F88C3A18443A
:10A000000C46807D10F0DCFE18B1828803680CB12C
:10A010001A8310BD5A83FCE7B01A002010B42A49F5
:10A020002A4A91F804367BB3D2F86C48A04239D062
:10A03000012B29D0D2F88448844239D0022B23D076
:10A04000D2F89C48A04235D0032B1DD0D2F8B4489A
:10A05000A04231D0042B17D0D2F8CC48A0422DD04A
:10A06000052B11D0D2F8E448A04229D0062B0BD002
:10A07000D2F8FC48A04225D0072B05D0D2F81449CD
:10A08000844208BF07230ED003F1010C81F804C6F7
:10A0900003EB430102EBC1025DF8044BC2F86C080C
:10A0A000184670470023DBB218465DF8044B704732
:10A0B0000123F8E70223F6E70323F4E70423F2E79A
:10A0C0000523F0E70623EEE704000010B01A002095
:10A0D00038B5424C8C2303FB004393F88B3003B913
:10A0E00038BD94F8DCC494F8DD349C450ED003EB05
:10A0F000430204EBC20292F8E0E40EF1FF35012DB9
:10A100004FEA430246D9BEF1030F3ED08C2202FB38
:10A110000042A2F87C10EFF31181902383F31288A0
:10A12000B2F87C5092F87E3043EA45030025C9B26C
:10A130009BB282F87E5081F3118829491A090D7863
:10A1400082EA13225A4005B1D2431B019BB202F0AE
:10A150000F021A4391F808365BBB8C2303FB0044C3
:10A16000D1F8283AD4F8040101219847D4F8001115
:10A17000B4F888508A8AD4F8FC302A438A8258601E
:10A180001A6842F001021A6038BD5D1C05F0030533
:10A190006545BBD0134404EBC303034493F8ED14AB
:10A1A0000029B3D08C2303FB0043012283F87E20D7
:10A1B000ACE78C2303FB0044D1F8285AD4F8843050
:10A1C000D4F800115B79086903F0FC0318440421FA
:10A1D000A847D4F800318000988138BDB01A00201B
:10A1E0000400001043680B4A23F0407323F480738B
:10A1F00043F48073436083681A4042F00202826035
:10A20000C36A0139CAB223F4700141EA0251C16242
:10A21000704700BFFDF7FFC0704700BF0020FDF78B
:10A2200001BF00BF0120FDF7FDBE00BF0220FDF70A
:10A23000F9BE00BF10B1036882881A83704700BF5F
:10A2400030B1036882881B691A4214BF01200020C4
:10A25000704700BF10B1036882885A83704700BFFF
:10A2600010B404698269E468416814604024D460D1
:10A27000446900230C31C2E90433C2E90633C2E960
:10A280000833C2E90A33C2E90C3393609363516027
:10A2900084B1C269E0689363C2E90233C2E904335E
:10A2A000C2E90633C2E90833C2E90A33C2E90C3312
:10A2B000C2E900015DF8044B704700BF436800220B
:10A2C0001A60037D1F2B08D9203B2022016802FA67
:10A2D00003F343F01803CB6070472022016802FAB1
:10A2E00003F343F018038B60704700BF0268136AE2
:10A2F00011B1D96901B3143330B49C681D689169F8
:10A30000DDB14FF4806088618D60104640690C615A
:10A3100080B15968D369C9B10A464FF480619A6027
:10A320009961224312F0010F14BF00224FF4005232
:10A330001A621C6130BC704770478D61054D4FF04B
:10A34000FF0C05F8DACF00688D60DFE7024A9A60FB
:10A350009961E6E788010020402500200168F8B5F2
:10A36000D1E9042304465568002B49D09861107D3B
:10A370005E681F2831D81768202202FA00F040F0EA
:10A380001800B8601A7D1F2A32D91868203A202395
:10A3900003FA02F242F01802C26000232B6033601D
:10A3A0003368896943F010033360284658F042FC53
:10A3B00023683046D96958F03DFC2B68226843F089
:10A3C00001032B603368526843F0010333609388C4
:10A3D0009BB243F003039380F8BD17682038202216
:10A3E00002FA00F040F01800F8601A7D1F2ACCD85D
:10A3F0001868202303FA02F242F018028260CCE7C8
:10A40000137D90611F2B1CD81068202202FA03F3E1
:10A4100043F01803836000232B602B68896943F0A5
:10A4200010032B60284658F005FC2B68226843F087
:10A43000010352682B6093889BB243F00203938020
:10A44000F8BD1068203B202202FA03F343F0180302
:10A45000C360E0E72DE9F0417F4D804E07463C6840
:10A4600097F888806368B888012284F824201A88C5
:10A4700022F040021204120C1A802289824223D058
:10A48000198821F038010904AB424FEA114100F06C
:10A49000BF80734A934200F0BB800246B2F5807FD2
:10A4A000A8BF4FF48072022AB8BF0222002A92FA93
:10A4B000A2F2B2FA82F208BF4FF0FF32013A41EA4B
:10A4C000C20292B21A802081397BA27A8A420CD0D1
:10A4D0001A8822F003021204120C1A801A8892B20F
:10A4E000002900F092801A80A1721A8892B242F07C
:10A4F00040021A80226A9168002900F0A3804FF080
:10A50000000C1432E64652F8100C8E4400EA0601A4
:10A5100020B1B1F1805F23D0616909B352F8140C06
:10A52000143200EA060110B1B1F1805F18D052F880
:10A530000C1C0CF1010C0029E5D1227B82B1B8F191
:10A54000000F0DD0BCF1010F6FD8BEF1070F6CD812
:10A550000CEB8C018900226A11440A7B002A64D02A
:10A56000226A92684FF00008002A53D0B8F1000F19
:10A5700002D098F80C2022B1BA6812B11168928802
:10A580004A83226AD2F800E0226A5168226A9268FD
:10A59000501E9AB1BEF1000F23D01EF801CB1A89CC
:10A5A0009207FCD5A3F80CC01A89D207FCD59A896A
:10A5B00092B209B101F8012B0138EBD2236A1B7B5F
:10A5C000E3B9236A1B697BB1236AD7F894001B693E
:10A5D000984701280DD0022806D100232362BDE848
:10A5E000F0814FF0FF0CDAE7D4F82080236A1433AF
:10A5F0002362236A9B686BB16368B7E7BB68002B73
:10A60000DFD01A689B881383DBE742F003026AE716
:10A61000420843E7236A1B68DBB1236AD3E900726F
:10A6200022620022C3E9002219E700213846FFF721
:10A630005DFEBB6813B11A689B8853833846BDE83A
:10A64000F0418BE6227B002A8AD0B8F1000F82D13C
:10A6500086E72362C3E700BF003800400000FFFF29
:10A66000003C004038B5D0F8E0102B4B04465A6847
:10A67000D0F8D80071B1131A99420BDC94F8D0309D
:10A68000C4F8D820012B10D0D4F8D4300133C4F84A
:10A69000D43038BDD4F8E430C4F8D8200344C4F82A
:10A6A000DC3094F8D030012BEED16168201D04F12C
:10A6B000E805EFF3118C102383F3128863681B6A9B
:10A6C0000BB3D4F8F0302A461BB1D3691432002BF7
:10A6D000FBD10B6A6BB1996839B9934209D01968FB
:10A6E00029B15B6899680029F7D01433F3E7C3E90F
:10A6F00000055FFA8CFC8CF31188D4F8D430013358
:10A70000C4F8D43038BD0D625FFA8CFC8CF311882C
:10A71000FFF7A0FEB8E700BF001000E02DE9F04110
:10A72000826992F8DC30012B8AB005464CD0023B9E
:10A73000012B54D892F84C31D2F89C202E4C63F067
:10A740007F0313708669D6F8A030D6F8108003F125
:10A75000010E0FCCEC46ACE80F00D6F89C30CDE9EA
:10A76000003E0FCCACE80F0094E8030006F11007A0
:10A770008CE80300EFF31180102383F31288336910
:10A780001B6A002B2FD0029B6A461BB1D36914327F
:10A79000002BFBD1D8F8203073B1996839B99342B6
:10A7A0000AD0196829B15B6899680029F7D0143379
:10A7B000F3E71F60C3F804D0C0B280F31188AA6920
:10A7C00011690B6A002BFCD1D2F8A0305A8852BA1A
:10A7D000EA819A8852BA2A82DB885BBA6B820120AE
:10A7E0000AB0BDE8F081C8F820D0C0B280F311886B
:10A7F0003846FFF72FFEE2E7A4CF06082DE9F04127
:10A8000090F8DC30D0F8A050012B8AB0044672D00A
:10A8100016D8D0F89C304FF0FF321A605A609A6018
:10A82000DA60D0F8E0300522B3F57A7FC0F8F02086
:10A830007CD8032380F8DC3001200AB0BDE8F08129
:10A84000023B012BF8D890F84D31D0F89C20524EA5
:10A8500063F07F031370D0F8A030D0F8108003F1BC
:10A86000010E00F110070FCEEC46ACE80F00D4F853
:10A870009C30CDE9003E0FCEACE80F0096E8030017
:10A880008CE80300EFF31180102383F3128823690F
:10A890001B6A002B73D0029B6A461BB1D36914322A
:10A8A000002BFBD1D8F8203073B1996839B99342A5
:10A8B0000AD0196829B15B6899680029F7D0143368
:10A8C000F3E71F60C3F804D0C0B280F31188226997
:10A8D000136A002BFCD16B885BBAA4F8D030AB882C
:10A8E0005BBAA4F8D230EB8801205BBAA4F8D4306C
:10A8F0000AB0BDE8F08190F84C2190F84D319B1AD8
:10A900005B100133DBB205EB430235F813305BBA61
:10A91000A0F8D03053885BBAA0F8D23093885BBAE5
:10A92000A0F8D43001200AB0BDE8F08103691A7B99
:10A9300072B35B6963B390F898304BB390F84C31C5
:10A94000D0F89C20C4F8A40063F07F03137090F843
:10A950004C1190F84D31D0F8A0201048C4F80401F3
:10A960005B1A07330121C4F8FC30D4F89C3084F81A
:10A9700000110A44C4E93D3284F8DC105CE7C8F8F1
:10A9800020D0C0B280F311883846FFF763FD9EE700
:10A99000022384F8DC304FE7A4CF060801800008CA
:10A9A00008B51D2010F00CFA08B183794BB11E20B8
:10A9B00010F006FA08B1837903B108BD5523C380AE
:10A9C00008BD5523C380F2E7D3B2012B23D870B55D
:10A9D00002EB4202114C4FEA820E4FF0000C22466D
:10A9E0000EF10805634604E00133152B11D012F86F
:10A9F0001CCF6045F8D192F801C08C45F4D156596E
:10AA0000002EF1D0C3EBC3030EEB83030433E01835
:10AA100070BD002070BD0020704700BFCCCF06087D
:10AA200010B40C4C002304F6942C01E0152B0CD030
:10AA300003EB430201331CF802108142F6D1224499
:10AA40005DF8044B92F9960A70474FF0FF305DF8BD
:10AA5000044B7047B01A0020D3B2022B21D830B576
:10AA600002EB4202104D114C4FEA820C0CF10C0E1D
:10AA70002A46002304E00133172B10D052F82C4F44
:10AA8000A042F8D114798C42F5D152F80E40002C36
:10AA9000F1D02C2202FB03C30833E81830BD00209C
:10AAA00030BD0020704700BF8CCA0608000001407E
:10AAB000002838D030B51C4D90F804C0002305F6AE
:10AAC000942401E0152B2CD003EB43020133A15C4D
:10AAD0006145F7D12A44046892F9963A90F805E066
:10AAE000DAB2022A1DD803EB4303104810494FEA9B
:10AAF000830C02460CF10C05002304E00133172BF4
:10AB00000FD052F82C1F8C42F8D111797145F5D134
:10AB100051590029F2D02C2202FB03C308331844F8
:10AB200030BD002030BD7047B01A00208CCA060826
:10AB3000000001400348D0F8EC300BB1DC3018477E
:10AB4000704700BF880100200348D0F8103113B1CE
:10AB500000F5807018477047880100200348D0F83E
:10AB6000343113B100F59270184770478801002006
:10AB70000348D0F8583113B100F5A4701847704756
:10AB8000880100200348D0F87C3113B100F5B6707D
:10AB900018477047880100200348D0F8A03113B14E
:10ABA00000F5C87018477047880100200348D0F8A6
:10ABB000C43113B100F5DA701847704788010020DE
:10ABC0000348D0F8E83113B100F5EC70184770472E
:10ABD000880100200348D0F80C3213B100F5FE7054
:10ABE00018477047880100200348D0F8303213B16D
:10ABF00000F5087018477047880100200348D0F816
:10AC0000543213B100F511701847704788010020C5
:10AC10000348D0F8783213B100F51A70184770471E
:10AC2000880100200348D0F89C3213B100F523704E
:10AC300018477047880100200348D0F8C03213B18C
:10AC400000F52C7018477047880100200348D0F8A1
:10AC5000E43213B100F535701847704788010020C1
:10AC60000348D0F8083313B100F53E701847704719
:10AC700088010020094B0A4A013800EBC00003EBB1
:10AC80008000116BD0F8DC30064883420CBF4FF4D3
:10AC900000134FF480030B431363704788010020B7
:10ACA000003802400060024070B501383C4C3D4D18
:10ACB00000EBC00C04EB8C0C9646DCF8DC603A4AE6
:10ACC000AE420CBF4FF400154FF48005166B3543B0
:10ACD0001563CCF8EC10CCF8F4303449DCF8E030F3
:10ACE0008B424FEAC0023ED001F580618B423AD0E0
:10ACF000A1F57A718B4247D001F580618B4243D038
:10AD0000A1F57A718B4241D001F580618B423DD033
:10AD1000A1F57A718B4235D001F580618B4231D03B
:10AD2000A1F57A718B4233D001F580618B422FD02F
:10AD3000A1F57A718B422DD001F580618B4229D02B
:10AD4000A1F57A718B4227D001F580618B4223D027
:10AD5000A1F57A718B4221D0154D01F580618B42AE
:10AD600018BF002500E0134D104404EB8003CEF320
:10AD70008711C3F8FC5093F8F100BDE87040002241
:10AD80005CF0D6BD0C4DEFE70C4DEDE70C4DEBE75D
:10AD90000C4DE9E70C4DE7E70C4DE5E7044DE3E723
:10ADA000880100200060024000380240106002402C
:10ADB000008000282080001000800018008800100B
:10ADC00000802010208000200088002000802020AB
:10ADD0000D4B984214D0A3F58063984210D003F530
:10ADE000804398420CD003F58063984208D003F565
:10ADF0008063984204D0054BD3F8B00740087047F1
:10AE0000024BD3F8B007704700040140B01A00208D
:10AE1000800AA0F58010522808D8054B184490F8F5
:10AE2000F4330D2B02D8034AD056704700207047E8
:10AE30008CCA0608285E0708094910B54B6C094CF6
:10AE400043F480434B644022002104F6481061F033
:10AE5000B8FD4FF0FF33C4F8D43AC4F8D73A10BD68
:10AE600000380240B01A002058B183884FF00042E9
:10AE7000B3FA83F332FA03F303D002490A681343A7
:10AE80000B607047003C01400120FEF795BC00BFFD
:10AE90000220FEF791BC00BF0420FEF78DBC00BF6E
:10AEA0000820FEF789BC00BF1020FEF785BC00BF5C
:10AEB0004FF47870FEF780BC4FF47C40FEF77CBC0A
:10AEC00030B50C4683B0054618B3036803F13F4321
:10AED00003F57E039B0A104A134493F88C075CF039
:10AEE0005FFEA988009104F00303C4F381028DF88A
:10AEF000043028688DF80520C4F300136946C4F3B4
:10AF000041148DF806308DF8074057F04FFD03B01F
:10AF100030BD4FF0FF33DEE78CCA060800B1CFE743
:10AF2000704700BFF8B5CB7813B900252846F8BDA7
:10AF300000F110070C460646897838460FF0A6FC4B
:10AF400005460028F1D0E0780FF03AFFB061237891
:10AF50000133DBB210B1C371222383710921FFF7E2
:10AF6000DDFFB069FFF766F90D4AD2F80838632BA8
:10AF7000FBD90C480FF060FCB082384650F0D4FB8F
:10AF8000074630B9E0780FF01BFF0FF079FF3D4620
:10AF9000CCE7306986F8D8705EF052FDC6E700BF96
:10AFA000B01A002040420F000B4B10B5D3F88C3A7A
:10AFB00003440446987D0FF003FF60B12E22827196
:10AFC000621CC2710121FFF7A9FF20460021BDE8E4
:10AFD0001040FFF710B810BDB01A002070B50E4C2D
:10AFE000D4F8246A002E15DD04F58164002503E001
:10AFF000B54204F120040DD0237F0135002BF7D09A
:10B00000E0680028F4D0217DFFF75AFFB54204F133
:10B010002004F1D1012070BD04000010F8B5037DBB
:10B0200085691F2B04464DD90168A3F120024E68A3
:10B0300020209040064234D010239340C860CB605B
:10B040004B68D340DE0700F18380EFF31183502279
:10B0500082F312882A6C1168C9075AD4516889B2E0
:10B0600071B9D5E90960864250D0AF690744D7600D
:10B0700073D9301A80B25060AE62002185F8641036
:10B08000116841F00101DBB2116083F3118895F87A
:10B090006430002B44D1237D1F2B27D92168A3F1D5
:10B0A00020024C6808209040044200D0C8604C68E0
:10B0B000042000FA02F2224203D0203B00FA03F3FC
:10B0C000CB60F8BD026820201668984006421946F9
:10B0D0000ED010219940906091601168D940C80746
:10B0E000B3D5012101FA03F39360AEE72268194654
:10B0F000106808238B40184200D093601068042326
:10B1000003FA01F10142DCD09160F8BD012285F81B
:10B110006420DBB283F3118895F86430002BBAD039
:10B1200095F87C30002BB6D195F871000FF048FEF1
:10B130002A6E938923F008031B0401211B0C9381C1
:10B1400085F87C100028A6D02021FFF7B9FEA2E7E1
:10B15000012303FA02F2CA6077E72E69301A80B23F
:10B160005060A96289E700BF70B50C4682B01546F1
:10B170000646002839D0036803F13F4303F57E03F8
:10B180009B0A1B4A134493F88C075CF009FDB288B4
:10B190000092B2FA82F304F003028DF80420C4F3A3
:10B1A000810230688DF80520C3F11F03C4F300123B
:10B1B000C4F341148DF80740C3F3CC0400EB8404BE
:10B1C00003F007038DF806209B00226A0F269D409E
:10B1D00006FA03F322EA03032362226A154369464F
:10B1E000256257F0E3FB02B070BD4FF0FF33C8E7B4
:10B1F0008CCA060800B1B7E7704700BF2DE9F043DD
:10B20000774D05EB001683B0D6F8DC3A002B00F042
:10B21000938004464FEA001896F8E40A5CF0C0FCFC
:10B2200096F8E43A590903F01F0203294FF001038D
:10B2300003FA02F300F09880042900F085800229C7
:10B240007DD005EB0803013493F8E00A0FF0B8FD58
:10B25000E4B2814610B112238371C47105EB080377
:10B2600093F8E10A0FF0ACFD074610B11323C47147
:10B27000837105EB080393F8E20A0FF0A1FD06467F
:10B2800010B11423C47183714544484695F8E32AEC
:10B2900001924A21FFF7AEFF019A38462A21FFF7B3
:10B2A000A9FF019A0A213046FFF7A4FFD5F8DC2A4E
:10B2B0004C4B9A425DD04C4B9A424AD04B4B9A42EF
:10B2C00062D04B4B9A426AD04A4B9A4272D04A4B58
:10B2D0009A427AD049499088B1F81E43B1F81C339C
:10B2E000B1F826532343B1F820432343B1F8224356
:10B2F00020F003002343B1F824430004000C23434F
:10B30000B1F8284390802B4310882343B1F82A4397
:10B31000B1F82C1300F44150234303439BB2138034
:10B32000938B23F400631B041B0C938311821388FB
:10B330009BB243F04003138003B0BDE8F083304A72
:10B34000516A0B4353627CE72D4A11690B43136129
:10B3500077E703F50033196A41F480411962196AED
:10B3600021F480411962B5E7254A116A0B43136243
:10B3700067E703F58433596A41F480515962596A89
:10B3800021F480515962A5E703F5FE33196A41F4AF
:10B3900000411962196A21F4004119629AE703F524
:10B3A0008233596A41F400515962596A21F40051BB
:10B3B00059628FE703F56843596A41F48011596275
:10B3C000596A21F48011596284E703F56443596A8C
:10B3D00041F400115962596A21F40011596279E768
:10B3E000B01A00200030014000380040003C00400E
:10B3F0000034014000500140005401408801002009
:10B4000000380240431C00F074812DE9F04F00EB3E
:10B410008003BE4FDA0087B057F8029081000546DE
:10B42000019107EBC303B9F1000F05D09C68002C14
:10B4300000F02F81A17911B107B0BDE8F08FD3F8EA
:10B440000CA0BAF1000F00F0A2819AF80630002B90
:10B45000F2D11832B818D9F80480BB50691CC0E981
:10B460000133C3601523A371C9B21623E1718AF8B1
:10B4700007108AF8063099F818005CF091FBB8F8CC
:10B4800004302268A18823F440731B041B0CA8F825
:10B490000430DAF800301183BAF804201A8311213D
:10B4A0002046FFF70DFD11215046FFF709FD092643
:10B4B0004FF0330B05E0BBF1010B00F0158110F0EC
:10B4C00017FE0A20002CF6D02268A18813691942C1
:10B4D000F1D05183052010F00BFE2368A2881A8357
:10B4E000052010F005FE013EE2D1332604E0013EC6
:10B4F00000F0308110F0FCFD0A20002CF7D023680A
:10B50000A28819690A42F2D05A83052010F0F0FD92
:10B51000BAF1000F00F05D81DAF80030BAF80420CB
:10B520005A83052010F0E4FD002C00F024812368EC
:10B53000A2881A83052010F0DBFDDAF80030BAF893
:10B5400004201A83052010F0D3FD2368A2881B690C
:10B550001A4240F0D580019B2B4407EBC3039A7C31
:10B56000002A40F0CA801A7C12212046FFF7FCFD19
:10B57000019B2B4407EBC3039B7C002B00F0C48092
:10B580003221BAF1000F07D0019B2B4407EBC30314
:10B5900050465A7CFFF7E8FD5D4B984500F0288146
:10B5A0005C4B984500F02F815B4B984500F036814D
:10B5B000019B2B4407EBC3074FF47A73BC8A03FB50
:10B5C00004F4B8F8043023F440731B041B0CA8F8EF
:10B5D0000430B8F800309BB243F00103A8F8003003
:10B5E000B8F8045002A857F02BFA25F03F0504994B
:10B5F0004A4B2D04A3FB01232D0C45EA9345A8F8E3
:10B600000450B8F8002022F001021204120CA8F82D
:10B610000020434A980C9442034600F38380620062
:10B62000B1FBF2F292B20133042A38BF0422A8F827
:10B630002030A8F81C20B8F800309BB243F001037A
:10B64000A8F80030B8F8003023F4816323F0020337
:10B650001B041B0C4FF4804143F48063A8F80030B6
:10B66000A8F80810B8F8003023F080031B041B0C66
:10B670000022A8F8003099F81A0011465CF058F939
:10B68000002299F81900114607B0BDE8F04F5CF0B0
:10B690004FB9D3F80CA0BAF1000F00F0D4809AF89B
:10B6A0000630002B7FF4C8AE1832BB18D9F80480DE
:10B6B000BC50C3E90144DC6016238AF806306B1CD9
:10B6C0008AF8073099F818005CF06AFAB8F8043084
:10B6D000BAF8042023F440731B041B0CA8F80430B0
:10B6E000DAF800301A83DEE624B9052010F000FDF8
:10B6F000F6E67047A1882268EBE61A7C322134E72F
:10B70000DAF800301B6926E712213AE7B01A002068
:10B710000054004000580040005C004083DE1B43A2
:10B72000A086010004EB4404B1FBF4F18AB2C1F33A
:10B730000B0109B942F0010250494FF4967300FB26
:10B7400003F3A1FB03139B09013342F40042A8F861
:10B7500020306EE7002C40F08D80052010F0C8FCF2
:10B76000BAF1000F65D0DAF80030BAF804205A8335
:10B77000052010F0BDFC052010F0BAFCDAF800300E
:10B78000BAF804201A83052010F0B2FCF0E6183253
:10B79000BB18D9F8048047F802A0C3E901AAC3F88E
:10B7A0000CA01523A371431CE37199F818005CF0F9
:10B7B000F7F9B8F80430A28823F440731B041B0C7B
:10B7C000A8F80430236811211A832046FFF778FB7C
:10B7D0006DE6052010F08CFC2368A2881A830520F2
:10B7E00010F086FC052010F083FC23681B69B2E68C
:10B7F00003F5F2331A6A42F400121A621A6A22F44A
:10B8000000121A62D4E603F5F0331A6A42F4800299
:10B810001A621A6A22F480021A62C9E603F5EE334C
:10B820001A6A42F400021A621A6A22F400021A62C8
:10B83000BEE6052010F05CFC052010F059FC052048
:10B8400010F056FC94E61832BB18D9F8048047F87B
:10B8500002A0C3E901AAC3F80CA099F818005CF093
:10B860009FF9B8F8043023F440731B041B0CA8F8AC
:10B8700004301CE6A288236846E600BFD34D621060
:10B880002DE9F843074610F099FBDFF84C8007EBF1
:10B890008709044608EBC90542F20F7604E010F070
:10B8A0008DFB031BB3420ADC6B7E002BF7D108EB48
:10B8B000C90898F8180080F00100BDE8F883B8F8CE
:10B8C0000C3B013338469BB2A8F80C3BFFF79AFDBE
:10B8D0000020BDE8F88300BFB01A002010B582B088
:10B8E0008DF80730431C0CD00228044609DC0DF10A
:10B8F00007035CF0FBF820B12046FFF7C1FF02B060
:10B9000010BD002002B010BD70B500EB8003274DC4
:10B9100005EBC30255F833305C68A38A84B09BB250
:10B920000393039B13F4706F1CBF01231376039BD7
:10B9300013F4E06F4FEA80060CD1A38A304423F45D
:10B94000706305EBC0051B041B0C0022A3826A7602
:10B9500004B070BD238BA38823F480631B041B0CED
:10B96000A380039B9A05E8D423889B05E5D423880C
:10B97000D9050FD52388DA05FCD423889BB243F47C
:10B980000073238023889B05FCD40190FFF73AFDC8
:10B990000198D2E723889BB243F400732380A388E5
:10B9A00023F440731B041B0CA380C6E7B01A0020CD
:10B9B0000020A9E70120A7E70220A5E72DE9F84F1D
:10B9C0002F4F00EB800407EBC404D4F80480B8F1D7
:10B9D000000F04D09A46637E03F0FF0923B14FF0B5
:10B9E00000094846BDE8F88F0E469346054610F01C
:10B9F000E5FA0A9B7600F6B2C4E908330123A6767D
:10BA000084F81BB084F81D90A37784F81CA063769B
:10BA100084F81890B8F804209105064622D4B8F8A6
:10BA20000030DA0512D442F20F7404E010F0C6FAC6
:10BA3000831BA3421ADCB8F800309B05F6D4B8F893
:10BA400000309BB243F48073A8F80030B8F804309B
:10BA50009BB24FF0010943F44073A8F80430484604
:10BA6000BDE8F88F99464846BDE8F88FB7F80C3B1B
:10BA700001339BB22846A7F80C3BFFF7C3FCB0E7A5
:10BA8000B01A0020F8B590F871301C09013C052C63
:10BA90000FD81B4E06EB44020546B2F8940703F09C
:10BAA0000F0340FA03F2D20703D595F87C70012FFB
:10BAB00001D00120F8BD07FA03F3013B18403444DC
:10BAC0005FF050F894F8A0270E4C104454F8302042
:10BAD00004EBC0041069A3881840EBD0EB6E002281
:10BAE00085F87C2093F8212020460221FFF73CFBBB
:10BAF0002A6E93899BB243F0080338469381F8BDC0
:10BB00008CCA0608C0250020094BD3F8102ED3F8A4
:10BB1000141E40F62A00002350604B620B889BB233
:10BB200043F001030B80136843F001031360704777
:10BB3000B01A00201D4B1E48196C1E4A10B441F06B
:10BB400080510124196404625321FF24CA205462E5
:10BB5000506251625B6FDB0085B017D41648042336
:10BB6000002102910290029A1A440292029A04332E
:10BB70001C2B1160F5D103910390039B0393039B4E
:10BB80000E4A1A6005B05DF8044B70470A4B00225C
:10BB900001920193019B0193019A084B12689A420A
:10BBA000DCD105B05DF8044B704700BF003802409F
:10BBB00000000E42002800405028004031666542D7
:10BBC00010B5174C84B00139002389B2A042ADF8FA
:10BBD0000C30ADF806308DF80E30029113D0114BB9
:10BBE000984210D003F5804398420CD003F580634F
:10BBF000984208D003F58063984204D00A4BD3F8EA
:10BC0000B0375B0802E0084BD3F8B037B3FBF2F271
:10BC100001A9013AADF8042057F0AEF804B010BD08
:10BC20000004014000000140B01A002030B5044675
:10BC3000006EA268838923F400531B041B0C8381CC
:10BC4000637995B013F0040F4FF00001019214BF17
:10BC50004FF480520A46ADF808201A031B0203F481
:10BC60008063ADF80C302379ADF80E1002F4005269
:10BC7000ADF80A20DA0744BF0422ADF80E209B0776
:10BC8000ADF8101005D5BDF80E3043F00803ADF83F
:10BC90000E3001A957F082F96279236ED50700F1C1
:10BCA0008B8012F0080F9A8A48D092B242F00802B4
:10BCB0009A829A8992B242F400529A812279D007EC
:10BCC00032D5E06B002800F089800023E26D0893F4
:10BCD000CDE90C33CDE91033CDE912334FF4807543
:10BCE0000A936369E1680E9506920793626C059268
:10BCF0004FF480634FF480350B9309910F9556F004
:10BD000003FF05A9E06B56F095FFE26B216E136807
:10BD100043F0010313608B8A9BB243F040038B8294
:10BD2000536822799BB2636591070DD4226E938983
:10BD30009BB243F40053938115B030BD22F008024A
:10BD40001204120C9A82B4E7206C002852D02369A6
:10BD5000A26D0993A36CCDE90532402300254FF471
:10BD6000803108934FF480630B930F91CDE90C550C
:10BD7000CDE91055CDE9125507950A950E9556F067
:10BD8000C3FE206C05A956F055FF236C226E58693E
:10BD900040F080005861186840F0160018605D603F
:10BDA000938A9BB243F0800302F10C0193820B68EB
:10BDB00043F040030B60BAE71E498B4224D0A1F543
:10BDC0004C418B421ED001F580618B421ED1022076
:10BDD0000121FEF710F96279236E62E74FF6DF71F9
:10BDE0001980D96841F02001D960D96841F010016B
:10BDF000D96099E7226ED36843F0800302F10C0109
:10BE0000D360D4E70120E3E70020E1E701F580619A
:10BE10008B420AD001F580618B4208D001F5444184
:10BE20008B427FF43EAF0520D2E70320D0E7042009
:10BE3000CEE700BF001001402DE9F84F4D4C04EB58
:10BE40008004D4F82C4A002C7DD0E56E002D76D0ED
:10BE50001F46EB6A6361AB6AA3616B8EE3602B8E56
:10BE600023616B682366444B2360444BA160A36647
:10BE70000646204690460FF067FB94F871000EF0DE
:10BE80009FFF824695F8200094F870B0A1460028E4
:10BE90004ED102213A0784F87C1036D418F0020FF4
:10BEA00010D0BAF1000F0DD00B238AF80630731CA6
:10BEB0008AF807303B0648D495F8212050462221C5
:10BEC000FFF752F918F0010F04D1E26B9AB148461E
:10BED000BDE8F88F58460EF073FF0028F5D00C220D
:10BEE0000136C671827195F821202221FFF73CF9B5
:10BEF000E26B002AEBD195F8241095F8220089090D
:10BF00005BF016FD4846BDE8F88F0136F6B2BAF18F
:10BF1000000FDAD00B2317F0500F8AF807608AF869
:10BF2000063008D095F821205046FFF71DF9CCE7E0
:10BF30005BF036FEADE795F821201221F4E7A94623
:10BF40004846BDE8F88FA146C1E794F871000EF0AD
:10BF500037FF226E938923F008031B0401211B0C79
:10BF6000938184F87C100028ACD02021FEF7A8FF34
:10BF7000A8E700BF0400001034D2060885BA000804
:10BF8000BFF34F8F0549064BCA6802F4E0621343C2
:10BF9000CB60BFF34F8F00BFFDE700BF00ED00E0B7
:10BFA0000400FA0508B572B6FFF7EAFF00B583B0E2
:10BFB0000D49002200920091009B0C330093009BDE
:10BFC0001B68012B02D003B05DF804FB01920191C4
:10BFD000019B06490C330193019B1A600B6883F3A4
:10BFE00008884B689847FEE7502800400000FF1F74
:10BFF00038B5FFF79FFDFFF7D9FF012056F0ACFEE3
:10C00000714A936823F003039360936813F00C0F55
:10C01000FBD113686C49002842D143F0010313603F
:10C0200041F288330A6895075DD4013BFAD1674C29
:10C03000674D654B674AEA60596F674AC4F8301E1E
:10C04000AA60596B654821F080015963596F41F02E
:10C0500080715967196B41F4CE0119635A6B5A63A9
:10C060009A6B9A631A6C02431A64596C5C4A0A43CD
:10C070005A640FF05BFFD4F8B0375A4AA2FB03238F
:10C080009B09013BB3F1807F09D24FF0E022F02001
:10C0900053610021072385F823009161136138BDA6
:10C0A00043F4803313600A68940341F2883304D464
:10C0B000013BBCD00A689403FAD5444C4A4A4B4B26
:10C0C000B0FBF3F3B0FBF2F0B3EB400F18BF184630
:10C0D0004FF48002B3FBF0F3C4F82C2EC4F8180E12
:10C0E000C4F81C3E09E0394C002108220223C4F8A0
:10C0F0002C1EC4F8182EC4F81C3E022056F02CFE4C
:10C1000003280FD83A4BD4F81C1E03EBC0008588D7
:10C11000C2884388C4F8245EB3FBF1F3C4F8282E28
:10C12000C4F8203E284B33491A6C42F080521A64FE
:10C130000A6842F440420A609A689A609A6842F437
:10C1400000429A609A6842F4A0529A60D4F82C0E89
:10C15000D4F8182ED4F8201E024342EA8112D4F8F3
:10C16000241ED4F8280E490842EA0062013942EA46
:10C1700001425A601A6842F080721A601A6892018D
:10C18000FCD51D4A40F205711160996821F0030148
:10C190009960996841F00201A2F580629960936804
:10C1A00003F00C03082BFAD1D4F81C0E1349D82342
:10C1B000B3FBF0F39B0143F000530120C2F884303D
:10C1C0008866FCF71DFC33E700380240B01A0020F7
:10C1D00000ED00E00005FA0500000020FFC9FE3672
:10C1E000335F0700D34D621080841E0040420F0071
:10C1F00064D2060800700040003C02400000474244
:10C2000010B584B000230446ADF80C300068ADF8DA
:10C2100006308DF80E3003F18043013903F5823387
:10C2200089B29842029114D0A3F58063984210D04D
:10C2300003F5804398420CD003F58063984208D000
:10C2400003F58063984204D0204BD3F8B0375B08E5
:10C2500002E01E4BD3F8B037B3FBF2F301A9013B68
:10C26000ADF8043056F088FD2168194A0B8819484A
:10C270009BB243F001030B80002301E050F8332010
:10C28000914208D001330E2BF8D1002004B0BDE854
:10C290001040FCF7F9BA104A02EBC30393F8FD47CC
:10C2A0002046FCF7F1FA1B2C05D1192004B0BDE89B
:10C2B0001040FCF7E9BA2E2C08BF2C2004D104B0A2
:10C2C000BDE81040FCF7E0BA04B010BDB01A002081
:10C2D0000000014084D206088CCA060870B50468C4
:10C2E000A30AA3F58013522B51D83C4D2B4493F84D
:10C2F000F4530D2D4BD840798608002954D005EB16
:10C30000850305EB4303B4F80CE04FEA900C33448B
:10C310000220334E00FA0CF040EA0E0006EB830CCC
:10C3200080B2CCF84815CCF85825A081EFF3118CD9
:10C33000502383F312882C2305FB03F3F118D1F863
:10C34000442562B3274BC1F86825043226482C21C6
:10C3500005FB01F1084414310B4453F8041B19B1D7
:10C36000116053F8042C04329842F6D100235FFA8E
:10C370008CFC13608CF311882C2303FB0565D5F826
:10C3800068352BB1A3899BB243F00103A38170BD33
:10C39000A38923F001031B041B0CA38170BD03F1CF
:10C3A0002402104B1A44D1E7B4F80CC005EB850306
:10C3B000304605EB43034FF0020E33441FFA8CFC6A
:10C3C000074E0EFA00F02CEA0000A08106EB830075
:10C3D000C0F84815C0F85825A8E700BF8CCA060861
:10C3E000B01A0020F41F0020182000200149024844
:10C3F000FDF700BAF41F00200000014010B5064C04
:10C40000064804F24451FDF7F5F904F5DA610448F1
:10C41000BDE81040FDF7EEB9B01A00200000014061
:10C420000044014002494FF08040FDF7E3B900BFEE
:10C430002020002001490248FDF7DCB94C200020F3
:10C440000004004001490248FDF7D4B978200020DB
:10C450000008004001490248FDF7CCB9A4200020A3
:10C46000000C004001490248FDF7C4B92821002012
:10C470000004014010B5064C064804F5CF61FDF7F5
:10C48000B9F904F254710448BDE81040FDF7B2B99F
:10C49000B01A002000040140001C0040014902487D
:10C4A000FDF7A8B95421002000400140014902488D
:10C4B000FDF7A0B9AC210020004801400149024825
:10C4C000FDF798B9D8210020001800400149024822
:10C4D000FDF790B93022002000200040F8B5164D3D
:10C4E0001648174F00214FF41A7260F06AFA05F6E9
:10C4F00088064FF08041A5F18C043A46002301E004
:10C5000054F8332091420BD001330E2BF8D1002088
:10C510001C355BF045FBB5420CD055F81C1CECE714
:10C52000084A02EBC3031C3593F8FC075BF038FBA9
:10C53000B542F2D1F8BD00BF10D30608F41F0020A9
:10C54000000001408CCA060810B50C2937D8DFE876
:10C5500001F09736363666363636373636360700C9
:10C56000038C5488B2F80CE023F480531B041B0C9A
:10C570000384038CB0F804C0818B21F4E6414EEAB9
:10C58000040E0904148823F40053090C41EA042121
:10C590001B04754C1B0C43EA0E33A0421FFA8CFCA3
:10C5A0009BB289B200F0AE8004F58064A04200F036
:10C5B000A9809268A0F804C081830264038410BD3E
:10C5C000038CB2F80CC0548823F480731B041B0C3A
:10C5D0000384038CB0F804E0818B23F400731B0404
:10C5E0004CEA040C21F073011B0C43EA0C230904F0
:10C5F000B2F800C0090C41EA0C0C5B4988421FFAF2
:10C600008EFE9BB268D001F58061884264D092684A
:10C61000A0F804E0A0F81CC0C263038410BD038C22
:10C62000B2F80CC0548823F010031B041B0C0384C5
:10C63000038CB0F804E0018B23F020031B044CEAC8
:10C64000040C21F4E6411B0C43EA0C130904B2F874
:10C6500000C0090C41EA0C211FFA81FC42498842C2
:10C660001FFA8EFE9BB269D001F58061884265D0C9
:10C670009268A0F804E0A0F818C08263038410BD9B
:10C68000038C5488B2F80CE023F001031B041B0C4C
:10C690000384038CB0F804C0018B21F073014EEACF
:10C6A000040E0904148823F00203090C1B0421431F
:10C6B0002D4C1B0C43EA0E03A0421FFA8CFC9BB2CC
:10C6C00028D004F58064A04224D09268A0F804C069
:10C6D00001834263038410BDD189548A23F400632B
:10C6E00043EA0121138A2EF4405E23434EEA031EDF
:10C6F00094884FF6FF330B4043EA04231FFA8EFE63
:10C700009BB284E7148A2CF4804C4CEA841C1FFAF8
:10C710008CFC4EE7D489B2F810E023F008032343E1
:10C72000548A2CF4407C4EEA040E948823F00403CF
:10C730004CEA0E0C1FFA8CFC2343C6E7D189548ABD
:10C7400023F0800343EA0111138A2EF4406E234341
:10C750004EEA830E94884FF6BF730B4043EA0413EE
:10C760001FFA8EFE9BB283E7000001402DE9F04FD7
:10C77000A24BDFF8A49293F8463EA14EA14F8FB092
:10C78000CDE90139013BDBB200930025DFF88CB223
:10C79000DFF88CA25B46D3469A464FEA9A23A3F56C
:10C7A0008013522B4CD8334493F8F4330D2B47D8D5
:10C7B000FC56019B012B40F00181012C35D14FF03B
:10C7C00000084146204610F08BFA10F017FB037862
:10C7D00013B1542B40F0F98008F104081FFA88F8CF
:10C7E000B8F1100FEDD14FF0000E8DB34946002087
:10C7F0000CE0334493F8F4330D2B0ED8FB56A342D0
:10C800000ED00130A84201F580711EDA8A681368E3
:10C810009B0AA3F58013522BEBD90023A342F0D13E
:10C8200053799BF805209A42EBD1774B5B454BD06F
:10C830005BF81CAF4FEA9A23A3F58013522BB2D9B1
:10C84000009B012BF1D90024B9E7BEF1000FECD118
:10C850005846FBF797FDC3B2022B9BF805C000F2C8
:10C860003483431C5BB203EB43034FEA830E644BF8
:10C87000664903F5727004E0984200F0268353F88D
:10C880002C1F5145F8D11A796245F5D153F80E4065
:10C89000002CF1D05E4800234268A24203F101035C
:10C8A00000F08980102B00F12400F5D14FF0FF3308
:10C8B000584A03EBC30302EB830393F8F830002BD1
:10C8C000B3D1029BC3F808B0029B013503F5807316
:10C8D000042D02937FF45AAFDFF848B10BF59E7335
:10C8E0000027ABF5816A9846DAF8243ABB425FDD4F
:10C8F000DBF80C50002D5BD09BF81030A888029319
:10C900002B68DAF80460019303F13F41B0FA80F339
:10C9100001F57E010393002EC3F11F034FEA91211D
:10C92000009340F38480002302E00133B3427BD0C4
:10C930001C0259F804208A42F7D14C440099029B0A
:10C940008BF8103003260137CBF80410CBF80C50CD
:10C95000CBF81840AE71EF71636CE26C0D46490084
:10C960008E401E43012303FA01F111439AF800207F
:10C970006664E1647AB303FA05F11A46236D0B434A
:10C980002365019B89B21883D4F8A000FBF736FD1C
:10C990002046FBF789FE0123082F8BF81C308BF80B
:10C9A0001D3088F811300BF1200B08F118089BD1CD
:10C9B0000FB0BDE8F08FDBB2013B79E7022B7FF4CB
:10C9C000FEAE082C3FF4FBAE2FE74FF0010E002D1A
:10C9D0007FF40CAF29E70399C1F12F05009903FA01
:10C9E00005F58B4099B2236D2B432365019B58833A
:10C9F000D4F8A000FBF702FDCAE700BFB01A002080
:10CA00008CCA0608285E07085CDC060800000140A6
:10CA100064020020880100200C0000100004014086
:10CA20007CDB06080C040010032B00F31F820AEBCA
:10CA30000623320218690492002800F03F829960B0
:10CA40000131CAB283F805210692542283F80421E9
:10CA50000136026805924479CAF80460FBF792FC3B
:10CA6000934AC3B2022B92F85DEE844600F22D8207
:10CA7000461C76B206EB46068E498F48059AB600EC
:10CA8000002305E00133172B00F01F8251F82C0F13
:10CA90008242F7D10879A042F4D188590028F1D018
:10CAA0002C2101FB03F30CEB4C0C03EB8C0C814BA6
:10CAB00063441969049B5344C3E906017F4B002179
:10CAC0001E461C466368984216D00131102904F1B5
:10CAD0002404F7D17A4B93F8D420002A00F0E781A0
:10CAE0007849794A794BCAF8681ACAF8602ACAF8AC
:10CAF000703A0FB0BDE8F08F01F1010C5FFA8CFCC9
:10CB00006F4B07960CF1FF3C0CEBCC0C03EB8C0C41
:10CB10009CF8F8300593002BE2D1049E069B8CF81C
:10CB2000F930F31103EB262000EB001368488C2446
:10CB300000EB83003112674B04FB01F103EB410171
:10CB40000AEB0603C3E93C145421019E8CF8F8104B
:10CB50003321C3F8AC10DE60C3F8A8005E4B049923
:10CB60009A4209EB010400F07681534B9A4200F09F
:10CB7000728103F580439A4200F06D8103F5806372
:10CB80009A4200F0688103F580639A4200F0638165
:10CB9000474BD3F8B007BEF1060F4FEA500000F044
:10CBA00061814E4B4E49BEF1070F18BF9C464D4B5D
:10CBB00008BF8C464C4918BF1946B0FBF1F1B0FBD9
:10CBC000FCFC1046049A01390AEB020389B20CF10D
:10CBD000FF3CA3F8B0C0A3F868104FF00006019323
:10CBE000A165002302F154014944A4F85C60636527
:10CBF00056F0C2F8019B3D4A1B69019318680388EF
:10CC00009BB243F080030380038809920A210B91B1
:10CC10004FF48072022123F00103CDE90C121B04B2
:10CC2000ADF828601B0C019E0380717909AAFFF7FB
:10CC30008BFC3079002840F02281049B079E0AEB90
:10CC4000030200231069D2F818C001680A8892B262
:10CC500042F001020A807268944503F1010300F07A
:10CC60000A81102B06F12406F5D14FF0FF33144A48
:10CC70001F4E03EBC30302EB83031E4AD3F8DC30E1
:10CC8000B3420CBF4FF400134FF48003166B3343D1
:10CC90001363427918480C2A9BBF184B03EB4203DD
:10CCA0000026B3F8F460049B53449E8200232EE0D8
:10CCB000B01A00208CCA060800000140640200205F
:10CCC00088010020ED7C0108E97C0108F57C010861
:10CCD00010290020402C0020000401404495080049
:10CCE00010552200D0DD060040771B0060000100D7
:10CCF00000600240003802401406001084DB060881
:10CD0000914200F0E0800133042B00F0E18050F804
:10CD10003320002AF4D1DAF80C260132CAF80C26A6
:10CD20000AEBC302DB00C2F8101603446A499A8872
:10CD3000059816439E80049B0AEB03069022234627
:10CD4000FDF7B2FFB0690268002342F010020260F2
:10CD5000C4E92533A367C4F88830C4F89C30F2696D
:10CD600062664FF48062E26704214FF40032C4E946
:10CD7000232140222267D6F8AC206267F268049B28
:10CD80001832A2664FF48052C4F88020D6F8A8204A
:10CD9000E26603F164014FF480424944C4F8842000
:10CDA00055F048FFB069049BD0F800E0C4F81CE0DF
:10CDB000D0F814E0C4F820E0D0F804E0C4F824E08F
:10CDC00003F1AC01D0F808E0C4F828E00023D0F863
:10CDD0000CE0C4F82CE0C4E93733C4F8B830C4F828
:10CDE000C030C4F8D030C4F8E430F369C4F8AC30D3
:10CDF0004FF48063C4F8C4304FF4403C0423C4E9CA
:10CE000035C3D6F8F430C4F8BC30F3681033C4F836
:10CE1000B0304FF40063C4F8C830D6F8F030C4F82E
:10CE2000B4304FF48042C4F8CC20494455F002FF9E
:10CE3000B369A8881A6822635A6962635A68A26350
:10CE40009A68E263DA6822641A6842F010021A6093
:10CE50002B68019372E5214BBEF1060FD3F8B007A2
:10CE60007FF49FAEDFF87CC01D49A6E61B4A032372
:10CE700082F85C3E34E6DBB20593013BF7E60DF049
:10CE80009FFF069038B1019B0221DA79FEF76CF919
:10CE9000069B5422DA80019B1A68B2F844306FEA8C
:10CEA00043436FEA53439BB2A2F84430C5E6542291
:10CEB00083F8D420069A83F8D52011E6074A022386
:10CEC00082F85C3E0CE6DB002FE700235B68FFDEA8
:10CED00000239B88FFDE00BF45840008B01A0020B5
:10CEE000A0BB0D00882A11000C2911D8DFE801F041
:10CEF0002310101019101010111010100700838B40
:10CF000023F400631B041B0C43EA022292B28283C7
:10CF10007047838B23F008031B041B0C1A43828386
:10CF20007047038B23F400631B041B0C43EA0222AB
:10CF300092B202837047038B23F008031B041B0C7F
:10CF40001A430283704700BF2DE9F04FDFF870B23B
:10CF50009BF8004087B024B90124204607B0BDE803
:10CF6000F08F934ED6F808580FF054F89BF8B43A67
:10CF70000390002B00F058828E4AA2FB05328E4BA4
:10CF80005209A3FB0213DB0803EB8303A2EB430369
:10CF9000DAB204920BF23C6202EB830300930BF6CD
:10CFA0001C1306F1DC0401934FF00009924635E0B2
:10CFB0003B680293009B5C330093019B3046143323
:10CFC000019355F0A1FD7A4B02988C2202FB0933A4
:10CFD000002583F8D05079792A46FFF785FF22464D
:10CFE0007979FFF7B1FA79790822FFF77DFF4023BD
:10CFF00044F83C3CA4F14801304655F01BFE336830
:10D0000043F0100333609BF8B43A09F101099945E4
:10D010000AF15C0A04F18C0480F2D480DBF8383623
:10D02000039AD31A04D454F8082C9342C0F2AB816B
:10D030005F4B54F8587C266A8C2202FB093393F824
:10D04000D030002BB4D03968736834F8542C029176
:10D050001FFA83FE8B89CEF1160E9BB223EA0203E0
:10D06000BEF1070F8B81A5D9DBF824390133CBF84A
:10D070002439A36A05939C4600225CF8045B0121D5
:10D0800090461BE0DCF80000B8F1140FA0EB05039C
:10D090001DDC13F1080548BF03F117052B1108EB40
:10D0A00025180546581E013102FA03F30122824079
:10D0B0008E4542EA03020CF1040C08D38E45E1D8F8
:10D0C000C8F11503DCF800504FF01508EAE7B8F195
:10D0D000150F60D13948C2F38423C2F3441100EB29
:10D0E000830300EB8101D3F81031D1F810111B023A
:10D0F00043EA011302F01F0100EB8101C2F3C432C5
:10D1000000EB8202D1F81011D2F810210B4343EA50
:10D11000023383EA132282EA121202F00F020F2A6C
:10D1200039D1C3F30F134FF6FF72934233D0B3F5E7
:10D13000606F00F03681019A93819AF85820049D1F
:10D14000AA4211D00098DAF800208168521ACAF871
:10D150000020016BDAF80420521ACAF804200022D9
:10D16000826002638AF85850DAF800200099013290
:10D17000CAF800208A6801328A604FF6FF72934233
:10D180007FF418AFDAF804300133CAF804300B6BBF
:10D1900001330B630EE7DBF820390133CBF820397C
:10D1A000B9F1000F00F0E5804FF6FF73C5E700BF4F
:10D1B000B01A00201F85EB51CDCCCCCC84DB060807
:10D1C0000400001001228BF8202ACBF83856002BDF
:10D1D0003FF4C2AE974890F88C10890700F1BE80EA
:10D1E000D0F88410086849798A40018C92B289B2DB
:10D1F00021EA02010184018C89B20A43012B0284D5
:10D200003FF4AAAE8B4991F81821970700F1C0802E
:10D21000D1F8102110685479018C012289B2A24002
:10D2200092B221EA02010184018C89B20A43022BE5
:10D2300002843FF491AE7F4991F8A421960700F152
:10D24000C180D1F89C2110685479018C012289B2E7
:10D25000A24092B221EA02010184018C89B20A4300
:10D26000032B02843FF478AE724991F8302295077F
:10D2700000F1B180D1F8282210685479018C012284
:10D2800089B2A24092B221EA02010184018C89B2E2
:10D290000A43042B02843FF45FAE664991F8BC2236
:10D2A000940700F1A180D1F8B42210685479018C60
:10D2B000012289B2A24092B221EA02010184018CCA
:10D2C00089B20A43052B02843FF446AE594991F8CE
:10D2D0004823900700F19180D1F8402310685479D9
:10D2E000018C012289B2A24092B221EA020101849A
:10D2F000018C89B20A43062B02843FF42DAE4D49BE
:10D3000091F8D423920700F18180D1F8CC231068E2
:10D310005479018C012289B2A24092B221EA020121
:10D320000184018C89B20A43082B02847FF414AE75
:10D33000404A92F860349B0771D5D2F858240423F0
:10D34000116850790A8C83409BB292B222EA0302A0
:10D350000A840A8C92B213430B84FDE5354AD2F855
:10D36000842010685479018C0422A24089B292B2C0
:10D370003EE70599304858225FF0C0FA3B680293B7
:10D380004FF6FF73D9E60024204607B0BDE8F08FC2
:10D39000284AD2F8102110685479018C042289B2ED
:10D3A0003DE7244991F8DD2402EB420201EBC20281
:10D3B0004A4492F8ED240D2A7FF4BDAE01998022F3
:10D3C0008A77BAE61B4AD2F89C2110685479018CFE
:10D3D000042289B23CE7174AD2F82822106854790F
:10D3E000018C042289B24CE7124AD2F8B4221068A8
:10D3F0005479018C042289B25CE70E4AD2F84023AA
:10D4000010685479018C042289B26CE7094AD2F879
:10D41000CC2310685479018C042289B27CE7054B37
:10D42000D3F8582401238BE701228BF8202ACBF86C
:10D43000383692E5B01A0020CC0900102DE9F04FE3
:10D44000002299B02F2107460FF02EFD00B3BE4EEB
:10D45000D0F80080C6F8148E0446FDF729FB02467A
:10D46000B0B1D0F804C0C6F810CEBCF1000F0FD098
:10D47000B64D002329464868844501F1240103F193
:10D4800001030FD0102BF6D1B14B93F8D40018B193
:10D49000002019B0BDE8F08F2F2283F8D42083F844
:10D4A000D500F6E7DBB2DFF8A892013B03EBC3033C
:10D4B00009EB830393F8F8A0BAF1000FE8D13846DE
:10D4C0009768DFF8C0B22F22A3F8F8200DF078FC9F
:10D4D0002F220346CBF8FC0420B1DA80E2792A211E
:10D4E000FDF742FE9B4A9C49002301E051F833209E
:10D4F000904500F0228101330E2BF7D100205AF025
:10D500004FFBD6F8140E954A038823F001031B0441
:10D510001B0C9042038000F070818E4B984216D015
:10D5200003F58043984212D003F5806398420ED0F1
:10D5300003F580639842D6F8B0270AD08849B1EB4A
:10D54000520F4FEA520340F2528100210AE0D6F80E
:10D55000B027834B9A4280F017814FF0010C0021D5
:10D56000B2FBFCF37F4AADF804101B0A7E49A2FB14
:10D5700003231A09A1FB021252084FF000081B09ED
:10D58000ABF8FA2401A952000293ABF8F824ADF8E5
:10D590000C80ADF806808DF80E8055F0EDFBCDE9DE
:10D5A0000688CDF82080A379ADF81480602204921B
:10D5B0009A0740F1AF80DB0003F00803ADF81E309E
:10D5C0000423ADF81430D6F8140E617904AAFEF7DE
:10D5D000BBFF61790822FFF787FCB0F84430D6F82A
:10D5E000108E6FEA43436FEA53439BB2A0F8443076
:10D5F00003889BB243F080030380A3796179028C96
:10D600009B074CBF042301238B409BB292B222EABA
:10D6100003020284028C92B21343038403889BB2F8
:10D6200043F0010303802A4600235168884502F134
:10D63000240203F101037DD0102BF6D14FF0FF330C
:10D6400003EBC30309EB8309484AD9F8DC304849A6
:10D650008B420CBF4FF400134FF48003116B0B434C
:10D66000136300236A68904505F1240503F1010363
:10D670005DD0102BF6D13F49602200235046FDF7C4
:10D6800013FB404655F040FAD6F8100E036823F01D
:10D6900001030025036055F037FACDE91455CDE9B3
:10D6A0001655D6F8143E0E9512956279D6F8100EDE
:10D6B000099734331344304A0B9240220A930C9258
:10D6C0004FF480434FF48052CDE9102340F62A01F5
:10D6D0004FF440330D91139309A94FF480630F93D6
:10D6E00055F0A8FA6379D6F8141E0C2B04D8234AF7
:10D6F00002EB4303B3F8F4508B89D6F8102E9BB29B
:10D700001D438D811368012043F01003136019B08D
:10D71000BDE8F08F5B0003F00203ADF81C3001237D
:10D72000ADF812304FF48073ADF820304BE75FFA5C
:10D7300083FAA0E7DBB2013B82E7114A02EBC303A5
:10D7400093F8FC07DBE600BFB01A0020640200205B
:10D75000880100200000014084D206080004014036
:10D76000006CDC02598B4F01ABAAAAAA0038024018
:10D7700000600240FD8600086C80002084DB060803
:10D780008CCA0608A82B0020254B98420BD003F525
:10D790008043984207D003F58063984203D003F595
:10D7A0008063984222D102F1B7731E4903F55853A2
:10D7B000A1FB03139B0D013B99B2194B984201F158
:10D7C000010C3FF4CDAE03F5804398423FF4C8AE60
:10D7D00003F5806398423FF4C3AE03F5806398423B
:10D7E0003FF4BEAE5308B3FBFCF3BBE6530803F1B2
:10D7F000B7730C4903F55853DAE7D6F8B0270A4B4C
:10D800009A42FFF4AAAE074902F1B77303F55853E1
:10D81000A1FB03139B0D013B99B201F1010C9FE6A3
:10D8200000000140819F5E16006CDC02F0B50C46E2
:10D8300089B03C49BDF838609DF83C70013B054615
:10D8400020689BB2049388424FF00003ADF8143077
:10D85000ADF80E308DF8163013D0334B984210D0FF
:10D8600003F5804398420CD003F58063984208D0BA
:10D8700003F58063984204D02C4BD3F8B0375B0893
:10D8800002E02A4BD3F8B037B3FBF2F203A9013A16
:10D89000ADF80C2055F070FA20686179A3790FB1CA
:10D8A00083F001030022CDE90622ADF810206022AA
:10D8B00003929A0729D5DB0003F00803ADF81A306C
:10D8C0000423ADF8103003AA01910596FEF73CFE43
:10D8D00001990822FFF708FB2268B2F844306FEA8A
:10D8E00043436FEA53439BB2A2F844301388114676
:10D8F0009BB243F0010321F8343B63796A60C81896
:10D9000000222860CA5009B0F0BD5B0003F002039A
:10D91000ADF818300123ADF80E304FF48073ADF838
:10D920001C30D0E70004014000000140B01A002084
:10D9300010B4104A92F8AC3703F0FF01002BF9D174
:10D940000D4B0E4CD3F8000554F89C4CB3F814352D
:10D950004FF0010C82F8ACC74360616223889BB230
:10D9600043EA0C03238003685DF8044B43EA0C038D
:10D9700003607047B01A0020A82B0020A03C0020B4
:10D980000B4B13F8842C53F8943C3AB113B11A683A
:10D990009B885383074B00221A827047002BF9D0D3
:10D9A0001A689B881383034B00221A82704700BFBA
:10D9B000A03C0020001000400B4B13F8842C53F8BF
:10D9C000943C3AB113B11A689B881383074B002229
:10D9D0001A827047002BF9D01A689B885383034B37
:10D9E00000221A82704700BFA03C002000140040B3
:10D9F00070B5384C14F8785C84B00DB904B070BDC3
:10DA000014F8773C04F8843C28460DF0D9F944F822
:10DA1000940C08B13823C38014F8806C6EB3012EC7
:10DA2000ECD13146FDF77AFA14F8843C002B49D149
:10DA300054F8943C13B11A689B881383264D4FF415
:10DA4000E072D5F8903144F8882C03A8012204F83C
:10DA5000982C039355F042F8D5F89431029302A81C
:10DA600055F03CF81D491E4C0B6C1E48002243F03B
:10DA700030030B6422850285C0E7284632463821F0
:10DA80000FF012FA05460028B8D0C27954F8940C69
:10DA90000221FDF7AFFB144A14F8843CD2F8B027FA
:10DAA000124801935208802329460096FFF7BEFED4
:10DAB00054F8901C8023012244F8883C0B6004F841
:10DAC000982C9BE754F8943C002BB7D01A689B889D
:10DAD0005383B3E7A03C002084DB060800380240F3
:10DAE0000010004000140040B01A0020103C00203C
:10DAF0002DE9F0415A4CDFED5B7A34F87E3CDFEDE6
:10DB00005A6A14F8805C04EB400007EE103A30F8D3
:10DB1000763C34F87A0C6422B8EEC77A02FB03F341
:10DB200027EE277A07EE903AF8EEE77A02FB003309
:10DB300027EE277A07EE903AF8EEE77A002687EE8E
:10DB4000270A0F4644F86C6C20EE260A4DB3012DCF
:10DB500001D0BDE8F08154F8888C07EE908AF8EE89
:10DB6000677A27EE800A5EF051F980BB14F8843C96
:10DB7000002B64D054F8943C13B11A689B8813832B
:10DB800034F87C0C38440EF0EDFC14F8843C002B87
:10DB90005DD054F8943C002BDBD01A689B885383EB
:10DBA000D7E754ED227AF8EE677A27EE800A5EF026
:10DBB0002DF954F8902C2D4B1060D3F8083834F818
:10DBC0007C1C1944394444F8681CBDE8F081284A9B
:10DBD000284B5062C2F82C805E62C3F82C80EFF3B1
:10DBE0001181502080F312881580C9B21D8081F305
:10DBF000118895811D4A9D81D2F8083834F87C1C23
:10DC000019443944D2F808389942FBD81849194ABE
:10DC10000B8854F8940C23F001031B041B0C0B809D
:10DC2000138823F001031B0400241B0C13808C8138
:10DC3000948100288DD0036882881A8389E754F87C
:10DC4000943C002B9CD01A689B88538398E754F827
:10DC5000943C002B3FF47DAF1A689B88138378E7D0
:10DC6000A03C00200AD7233CCA269B3EB01A0020C5
:10DC70000010004000140040034B13F8982C12B120
:10DC8000042800D834E77047A03C00201648174A03
:10DC9000174938B5174C184D121A5EF02FFED4F8FC
:10DCA0008820164B164842F47002C4F888201A687F
:10DCB000002142F001021A6099601A6822F0847211
:10DCC00022F480321A6058601A6822F480221A60A6
:10DCD0000C4AD960521B28460B495EF00FFEA56026
:10DCE000BDE83840FAF78CBE0000001004000010B8
:10DCF0002B18080800ED00E000000020003802406A
:10DD00001030002488010020000000080548D0F8E9
:10DD1000C43723B1DB6A13B100F2C470184702485C
:10DD2000704700BFB01A00201CDD060838B5184C3B
:10DD300054F8643C1B8843B9164D002304F8583C42
:10DD400085F8BC37C5F8B83738BD54F8602C002AC0
:10DD5000F2DD012A09D054F85C3C59880D4D24F8B5
:10DD6000561C012304F8543CE7E754F85C1C8A88ED
:10DD700049880132521A9A42F0D1064DD5F8C4377B
:10DD800000221B69C5F8F02705F2C4709847D4E754
:10DD9000A03C0020B01A00200748D0F8C0371BB1C3
:10DDA000064B13F8543C0BB100207047D0F8C43731
:10DDB00000F2C4705B681847B01A0020A03C002035
:10DDC00030B4154A154D92F8BC37A5F150042344E0
:10DDD000036015F8583C446092F8BC07834292F8FF
:10DDE000BC0712D8834204D3002030BCC1E9000034
:10DDF000704792F8BC27002BC2F180020CBF0120B3
:10DE0000022030BCC1E9002370471B1A0022012008
:10DE100030BCC1E900327047B01A0020A03C00209D
:10DE20000E4B0F4A93F8BC1712F8580C93F8BC2706
:10DE3000904293F8BC270CD8904238BF93F8BC2787
:10DE4000D3F8B8373ABFC2F18002801800201844D6
:10DE50007047D3F8B837801A18447047B01A0020BA
:10DE6000A03C002030B51C4C1C4D94F8BC3794F8F5
:10DE7000BC1785B0A5F150021344029315F8583C25
:10DE800003928B421DD894F8BC27934211D294F888
:10DE9000BC170193C1F180010091D3B9012208B9E7
:10DEA0003F2906D90023694602A85CF0DDF815F881
:10DEB000583C94F8BC07C01AB0FA80F0400905B08D
:10DEC00030BD94F8BC170022591A0192009101222A
:10DED000E5E719440222E2E7B01A0020A03C002046
:10DEE0002DE9F043164685B0002936D0441E254D55
:10DEF000254F04EB01084FF0000901E0A0452CD0AC
:10DF000015F8580C14F8013F411C2844C9B200F818
:10DF1000503C0B0648BF002097F8BC3705F8581C4A
:10DF20004ABF0146084605F8589C8B4297F8BC3713
:10DF30008ABFC3F18003C01AC0183F28DED997F802
:10DF4000BC378B42DAD0114B93F8C430002BD5D0BC
:10DF50000020FFF787FFA045D2D1694602A8FFF74E
:10DF60002FFF20B1DDE9003213443F2B02D805B06A
:10DF7000BDE8F0830246334602A85CF075F805B0B0
:10DF8000BDE8F083A03C0020B01A002088010020EA
:10DF900030B585B0694602A8FFF712FF58B9094CA1
:10DFA00004F2C475D4F8C43728465B689847002843
:10DFB000F8D005B030BD0246012302A85CF054F849
:10DFC000EDE700BFB01A002070B5124E1546D6F826
:10DFD000C0370A46411999420F4988BF1D1A11F8E6
:10DFE000581C96F8BC37994282B0044603D001927F
:10DFF000FFF7CEFF019AD6F8C41708480023C6F8E9
:10E00000F0372B468D6A2146AC4602B0BDE8704021
:10E01000604700BFB01A0020A03C002074220020FE
:10E020008C461346014662461846CDE738B524486B
:10E03000244C0023C4F8C03702461178022902F1AB
:10E0400006022CD00133062BF7D11F4DD4F8C4376C
:10E05000002245F85C2CF3B1DA6AE2B11B48904724
:10E0600055F85C3C45F8640CA3B19A885B88D21AD9
:10E07000436802FB0333C4F8C037FAF727FE15F8EC
:10E08000582C94F8BC379A42054601D0FFF780FF20
:10E09000C4F8B85738BD0E4B45F8643C38BD0A4D3E
:10E0A000D4F8C42703EB430300EB430345F85C3C7F
:10E0B00012B1D26A002AD1D1054845F8640CD4E7E0
:10E0C000D03C0020B01A0020A03C00207422002088
:10E0D0001CDD060810B50A4CD4F8C4375B6A13B1CE
:10E0E00004F2C4709847074AD4F8B83752F8642C41
:10E0F0005288013B134452421340C4F8B83710BD54
:10E10000B01A0020A03C00202DE9F043DFF8E89091
:10E11000374F93B0FFF70AFEFFF788FF99F8BC3737
:10E1200017F8582C9A4201D0FFF732FFD9F8C08770
:10E130000025C9F8B857B8F1000F11D02D4E6C4624
:10E140002A463146204603F08BF920465BF0DEFF7D
:10E150002035014601222046FFF7C2FEA845EFD830
:10E1600099F8BC3717F8582C9A4201D0FFF710FFE6
:10E1700057F8643C9B7B012B33D099F8BC3717F8D8
:10E18000582C9A4201D0FFF703FF0027C9F8B8774F
:10E19000B8F1000F28D0DFF85C903D466C462A4667
:10E1A000494609A803F05CF92122002120465EF0CF
:10E1B00008FC202221462846FFF706FF20220646BB
:10E1C00009A9204615445EF039FC08B9202E00D07C
:10E1D0000137A845E3D8B7FA87F0400913B0BDE886
:10E1E000F083FFF777FFC8E7012013B0BDE8F083A5
:10E1F000A03C0020545D0708B01A0020032108B598
:10E200000546084654F098FD72B6104BD3E9162324
:10E2100052EA03010AD100242146042054F08CFD67
:10E220002146052054F088FDFDF7AAFE0848D0F8E5
:10E23000084829B24EF6602000FB01F1A41843F112
:10E2400000030C1943EBE171E7E700BFA03C00209D
:10E25000B01A002008B50021032054F06DFD72B6FD
:10E26000FDF78EFE08B5174C226E94F866004AB191
:10E270001168938809690B40F0B9003B18BF01236E
:10E28000002BF4D114200EF06DF900BF236E63B1A2
:10E290001A689B88116994F866200B4042B9003BCC
:10E2A00018BF01230BB1FFF7D5FFFAF741FDECE7EB
:10E2B000B3FA83F35B09F5E7B3FA83F35B09002B49
:10E2C000D5D1DFE7A03C002008B555F099FA0C49FC
:10E2D0000C4B91F86D0029220128A3F86E2BA3F8AE
:10E2E000762B01D0012008BD0748086700F1200106
:10E2F0004C3059F01FF9054B002083F8230008BD6E
:10E30000A03C0020B01A0020B804002000ED00E07E
:10E310002DE9F04F41F62C728BB00021AE485EF033
:10E3200050FB042054F018FD0446052054F014FD61
:10E3300050EA040340F03F81A84B0393039BA84994
:10E34000A548D3F8C843E4225EF0D8FAA24BC3E94B
:10E350000744C3E91A445C621C67C3F8B440C3F8BD
:10E36000B840C3F8BC401F465AF020FDFFF75EFEE0
:10E37000002108460CF0B4FDFAF7A8FCB0F1000A41
:10E3800040F38F81974D984B984E0193002407F1ED
:10E39000E40902942746A34605F1740804E00BF54E
:10E3A000006BDA4540F3AE80019AD2F80838C2F823
:10E3B0000C38FAF7BDFC202241465846FFF704FE10
:10E3C0008B49122240465EF039FB0028E7D1BB455D
:10E3D00022D00299874BCDF8149001EB410203EB58
:10E3E00082004A1C84490292049003F039F8DDE966
:10E3F0000403D9F81C2043F84C0BC9E908227F4AD2
:10E40000C9F80C70C9F82820ABEB07070122C9E94D
:10E410000477C9F808209946039BD3F8C833C9F894
:10E420001C305F461222A918335D91F8741099428E
:10E4300002F101020BD00024202AF4D12037BA4582
:10E440004146384654DBFFF7BFFD0022EBE70134BD
:10E45000152CF1D1D0196A492022FFF7B5FD002310
:10E460000A2209A96648CDF8248003F081F90490B6
:10E470000998002301300A2209A9099003F078F9CC
:10E4800007900998002301300A2209A9099003F096
:10E490006FF906900998002301300A2209A9099012
:10E4A00003F066F90590099809A9013000230A22B2
:10E4B000099003F05DF907460998002301301946D9
:10E4C0000A22099003F054F9049989B1DDE9063272
:10E4D00043EA4212059B7F0147EAC323A1F2BC71C4
:10E4E00043EA600342EA412243EA0243C9F81C308E
:10E4F000029B642B00F0F6805F460BF5006BDA455B
:10E500003FF752AF029A642A00F0EC80BB4500F05E
:10E51000C080384C38490C2303FB0244531C1A4674
:10E520002046029302F09CFFD9F81C30C9F8004045
:10E53000ABEB0705C9E90375C9E90833C9F81450FD
:10E5400001232E4DC9F82850C9F80830029BDC1C65
:10E550004C22214E02FB04F43319184600215EF0D0
:10E5600030FA4C2200215EF02CFA039A0299D2F87C
:10E57000C823034623483051C3E904AAC3E907224C
:10E580005A62012204319D629A604FEA4A03B3F154
:10E59000805FC0F28780104A95682DB913791BB14E
:10E5A0001368002B40F0A880002108460BB0BDE89E
:10E5B000F04F0CF095BC4FF47A72002321465CF0CA
:10E5C00069FA114B40F26D11A3FB00231B0C0224CE
:10E5D00040F2B2720D4622E04C5B00208801002020
:10E5E00030DD0608A03C0020B01A0020985D070826
:10E5F000745D0708343D0020885D070821E00008AD
:10E60000143D0020B05D070807452EC2013212F00C
:10E610000304A3EB01030CBF4FF4B77129468B42EF
:10E62000F4DA8B49002C61D003910399D1F8981347
:10E630008B42C0F29480874D01245B1A55F8041F69
:10E64000994204F10104F8DD013343EA4413A2F2D4
:10E65000BC7243EA4223804A039DB0FBF2F102FB05
:10E6600011024FF461603C24B2FBF0F100FB112277
:10E670001C20C5F89C03B2FBF4F004FB10225210DE
:10E6800042EA401242EAC12242EA0343C5F8C833D3
:10E6900054E6029B0321DC1C002B3FF476AF6F4D48
:10E6A00056E703214C226E4D02FB01F42B1918464C
:10E6B00000215EF086F94C2200215EF082F9039978
:10E6C000CAF100620346520066482851D1F8C813C7
:10E6D0005962C3E9042202225A710122C3E90711D7
:10E6E0009A6058E764235D4D02932FE70C4603912F
:10E6F0001D21C4F89C1398E7C2E911551564D56330
:10E7000029462E46D46C02F14C0354B39C681E6417
:10E71000481E8442C3E91166DE6312D0481C84425D
:10E7200016D08C427FF440AF084600283FF43CAF3F
:10E73000116CCC6B0134CC631964936401461A46A6
:10E74000E0E700293FF430AF884253F80C2CECD1BD
:10E75000117900293FF428AF53641A64EEE70124CD
:10E7600072E73F490222264613E0CB6B0A635B0146
:10E770001DBF03F6FF7702F1FF3303EB1733134698
:10E78000C1E90466C1E90D3351F84C0F5A1C01353B
:10E79000C8B10B79002BE8D10F690A63002F4AD169
:10E7A0004F691046531E4863002F4DD007F6FF7780
:10E7B00003EB1733201A8B63C41851F84C0F5A1C03
:10E7C00001350028E5D128492848C1F85C583E2287
:10E7D0000D46C1F838283F22013BC1F83C284022B1
:10E7E000C1F840280191C1F84C38C1F850489A004E
:10E7F000990FC5F834084BB340F2FF10121841F1DD
:10E800000001520A42EAC152019C02F140010A444D
:10E8100002EBC303C4F84828C4F84418144A10494A
:10E82000C4F85418C4F858185802D90D42E9020126
:10E83000C4F83038B8E607F6FF77531E03EB1730FD
:10E840004F694863002FB1D11346B3E70122DBE7DC
:10E8500088010020200500208051010021E00008EF
:10E860004C5B0020C05D0708B01A0020CC5D070893
:10E87000E02200200A4AD2F8983573B119689888C6
:10E88000096992F8953508401BB1B0FA80F040094B
:10E890007047003818BF012070470120704700BF43
:10E8A000A03C00200020704700231B6AFFDE00BF51
:10E8B0000378022B12D00F4943680269D1F8480847
:10E8C00010B41840D1F84048D1F83C18931E400AC3
:10E8D00004FB030008445DF8044B7047054B426895
:10E8E000D3F83418D3F8300800EB410000EB522085
:10E8F000704700BFF45200202DE9F04F83B012F0B2
:10E90000020701930FD070B9864D95F8E437A5F54D
:10E91000805613B9012385F8E43701230220737070
:10E9200003B0BDE8F08F7F4DD5F83848D4BB4FF029
:10E93000FF3E7D4C7D4EF146F046F2464FF0000C16
:10E940002368984200F0BC8094F80EB0BBF1000F31
:10E950003DD0BBF1010F15D10CF5B17B06EB0B1BC4
:10E960009BF807B01BF0010F0CD11BF07E0F09D1F3
:10E970005FEADB1340F0B280D4F808B0D34501D28F
:10E98000DA46E1460CF1010CBCF10B0F04F1100466
:10E99000D6D1BEF1FF3F29D1B8F1FF3F20D0634E61
:10E9A000C64624E0D5F84068D5F83C3806FB043468
:10E9B000A042BCD395F8E43713B9012385F8E437B6
:10E9C0005A4B012200205A7003B0BDE8F08FE64692
:10E9D0000CF1010CBCF10B0F04F11004B0D1D8E71D
:10E9E000B9F1FF3F18BFCE4600F082804F4ED5F8F8
:10E9F000C84606EB0E1841F21869013448F80900C0
:10EA000041F21C600EF5B17C48F800404FEA0C1052
:10EA1000C5F8C846345006EB0C100024446006EBE1
:10EA20000C108079042876D8DFE800F0031B621B05
:10EA30002F0012F001046BD106EB0C10019B90F833
:10EA400007904FEAE20868F3C719032B80F8079094
:10EA50005CD94FF6FF70834228BF034606EB0C10CB
:10EA6000838097B1D5F8CC06D5F8C8360130C5F803
:10EA7000CC0641F21C6406EB0E1001330351C5F8BD
:10EA8000C83606EB0C1304209871500705D506EB29
:10EA90000C10C37943F00103C371D30608D506EB0C
:10EAA0000C16F379C3F34502013262F34603F371A6
:10EAB0001F4B012003EB4E230B6003B0BDE8F08F2A
:10EAC0001A4E0CF5B17406EB041E4FEA04189EF8BA
:10EAD00006E0BEF1000F0FD1E64688E7E0460CF1F4
:10EAE000010CBCF10B0F04F110047FF429AF50E7C7
:10EAF000002003B0BDE8F08FD5F8C8060130E64627
:10EB000046F80800A446C5F8C80688E72346A5E7E6
:10EB100000239B68FFDE95F8E437002B3FF4FAAE44
:10EB2000FBE600BFF45200200C590020F442002004
:10EB30000C43002070B5104E3378022B0F4B0BBFE7
:10EB4000020AC0F3D412C4B200F07F04D3F8300834
:10EB500082B010440D460023032201A9FFF7CCFE2A
:10EB6000012807D13378022B019B0CBF23F81450E6
:10EB700043F8245002B070BDF4420020F45200204B
:10EB80002DE9F04FDFF82C8198F80060032E85B056
:10EB90000C46154643D001288CBF00220122022ECC
:10EBA0000B68019269D14FEA1329DFB24FF4807AE2
:10EBB0000138012820D84FF0010B9D4217D93C4E57
:10EBC000D6F8A8271AB1D6F8C417994258D0D6F863
:10EBD000300800234844092203A9FFF78DFE0128CD
:10EBE0002CD0022817D020B123689D42E8D8256098
:10EBF000032005B0BDE8F08FF7B12D4B93F8E42763
:10EC000012B9012283F8E4270123022088F8013099
:10EC100005B0BDE8F08F022005B0BDE8F08F0128F7
:10EC20008CBF0023012301930B684FF0800AC3F3CC
:10EC3000D41903F07F07BBE7D346BEE798F800205E
:10EC40000399DDF804C0022A14D0032AE3D151F855
:10EC5000273023F07043B3FA83F35B0963455F44C5
:10EC6000236821D05B4457452360ECD309F10109A7
:10EC70000027BAE731F81730EDE74FF4807AD6E78E
:10EC8000D6F84018013A02EB41224902B2FBF1F2F8
:10EC90001344B3FBFBF20BFB12320AB15B449B1A29
:10ECA0009D4223608CD8A2E7AB42A2D39FE700BF6E
:10ECB000F4520020F44200202DE9F04FDFF86CB14F
:10ECC0009BF800C0BCF1020F894683B009688246F8
:10ECD000174640F08C800BF58053CEB2D3F83058F5
:10ECE000A6EB010805EB112590444FF4807398447E
:10ECF000B94208F1FF38B8FBF3F84CD2A844BCF194
:10ED0000030F07EB06040CBF80224FF48072641AD5
:10ED10009442A8EB050328BF144666B994422CBF61
:10ED20000A220B2201A92846FFF7E6FD012809D097
:10ED300003B0BDE8F08F0B2201A92846FFF7DCFDE8
:10ED40000128F5D19BF800C0D9F80010BCF1020FE2
:10ED500001F1010323D0B44210D9019906F1804298
:10ED6000013A01EB8202043901EB840142F8043FCD
:10ED7000914203F10103F9D1D9F80010A61B3144E7
:10ED8000BAF1010FC9F8001021D08F4205F1010539
:10ED90004FF00006B3D8012003B0BDE8F08FB442B5
:10EDA000ECD9019806F10042013A00EB4202023828
:10EDB00000EB440022F8023F904203F10103F9D135
:10EDC000A61B3144BAF1010FC9F80010DDD1B942D8
:10EDD000DBD1BCF1020F1DD004F18044019B013C4A
:10EDE0004FF0FF3243F82420D9F80010CDE70BF59F
:10EDF000805301F07F06D3F83038BCF1030FC1F324
:10EE0000D415A6EB01081D44904414BF4FF4807341
:10EE100080236CE704F10044019B013C4FF6FF7234
:10EE2000504623F8142003B0BDE8F08FF4420020D0
:10EE300030B50446C06983B010B9012003B030BDBD
:10EE40000D460023032201A9FFF756FD0128F5D145
:10EE5000B4F92030002B0ADA144B93F8E4270AB9EE
:10EE600083F8E407124B01225A700220E6E7019A68
:10EE7000012D4FEA431102EB431303D0022D11D1B0
:10EE8000E5255554A268DA612278032A04D10022CC
:10EE90001A775A779A77DA77626A5A83120C9A82CB
:10EEA00003B030BDE268DA61EEE700BFF452002043
:10EEB000F44200202DE9F04190F83C30002982B066
:10EEC000044614BF02210021042B7BD8DFE803F0A5
:10EED000030C3D486900FFF7ABFF012870D1626B5E
:10EEE000002A75D184F83C00404EDFF808814FF6C7
:10EEF000F77706F5805516E0BA424FD858F06EFA0B
:10EF000001284FF000011DD1206BFFF713FE0128EF
:10EF100018D1019AD5F844382263511E8B4228BF7C
:10EF20000B46C5F844383278236B032A01A91846EA
:10EF30009AB2E1D1434531D858F050FA01284FF048
:10EF40000001E1D002B0BDE8F081426B04F1300174
:10EF50000020FFF7B1FE012832D1032384F83C30B2
:10EF60002348E16AD0F8C437D0F84028C0F8C41765
:10EF70005B1A02FB03F3D0F8A82702EB4322C0F888
:10EF8000A827D0F8AC2702EB4323C0F8AC37002108
:10EF900000F5F460FFF74CFF012811D1042384F839
:10EFA0003C3094F82830042B04BF002384F8283028
:10EFB000A36B8BB120469847012002B0BDE8F081D9
:10EFC0000228BFD194F82830042B09D00220B9E7D9
:10EFD000022384F83C30B9E7012002B0BDE8F0819B
:10EFE000002384F828300220ACE700BFF442002060
:10EFF000F4520020F7FFFF0F38B590F83430044684
:10F00000052B43D8DFE803F01E033C0F185E006BAE
:10F010004FF0FF31FFF78EFD012837D1E06AB8BB12
:10F02000032384F8343000212046FFF701FF012834
:10F030002CD1042384F8343094F82830082B2BD0BA
:10F04000012038BD204DD5F8382800F130010232BA
:10F050000120FFF795FD012823D00238C0B2012816
:10F0600014D8052384F8343094F82830082B04BFD2
:10F07000002384F82830012385F8E537022038BDC5
:10F08000C06A216BFFF756FD0128C9D0002038BDAA
:10F09000022384F83430F4E7002384F82830012078
:10F0A00038BDE368D5F84018D4E90B2003EB4123C1
:10F0B000C5F84408C4E9033002B96062012384F84A
:10F0C0003430A5E7004DCFE7F452002010B590F89A
:10F0D00038300446032B59D8DFE803F0022F3843B9
:10F0E0002B4AC068117802F580530329D3F84018E1
:10F0F000D3F8C4270CBF4FF0800C4FF4807C01FB89
:10F100000CF100EB4120C4E90302D3F8A807A0EBFF
:10F110004120C3F8A807D3F8AC07A0EB4121E06A6F
:10F12000C3F8AC1702EB0C01C3F8C417C4E90C21F7
:10F1300040BB6262012384F8383016480021FFF793
:10F1400077FE012811D1022384F83830626B04F174
:10F1500030010120FFF7B0FD012806D1032384F818
:10F16000383000212046FFF763FE431EDBB2012B3F
:10F1700000D910BD94F82830062B04BF002384F872
:10F18000283010BDA2EB0C022263D3E70220ECE78B
:10F19000F4420020945A00202DE9F0434368C3F361
:10F1A00008020A44B2F5007F83B004460D4605D23A
:10F1B0002B446360012003B0BDE8F08390F91A206E
:10F1C000501C0AD0414902F5B17201EB0212D1790B
:10F1D0006FF30001D171FF22A27694F91B20511C1C
:10F1E0000FD03A4902F5B17201EB0212FF26D17934
:10F1F000C1F34500013820EAE07060F34601D171A7
:10F20000E67694F800C0BCF1020FD1D0DFF8C480DC
:10F21000D8F84028B5EB422F4FEA422915DCD8F840
:10F2200048781F407A42AA420FDCEA194A4510D2B8
:10F2300020690028BED0254A1278032A40D080B227
:10F240004FF6F7729042B3D9B4E7002003B0BDE89F
:10F25000F083227E206912F0080626D0D8F8C42751
:10F26000411C8A4213D300D100214B44A5EB090570
:10F27000DB1BBCF1020F60613D4421616360084605
:10F28000D7D1D8F85028B3EB422F91D392E798F812
:10F29000E42722B9012388F8E437636820690B4A20
:10F2A0000126567094F800C0DFE701A958F096F8DF
:10F2B0000128CAD10199636894F800C02069D4E795
:10F2C000034A90427FF674AF74E700BFF442002017
:10F2D000F7FFFF0FF45200202DE9F04790F8384077
:10F2E00082B00546032C00F2AB80DFE804F002197F
:10F2F000710BFFF781FE012810D002280AD10323E9
:10F3000085F838302B6C002085F82800002B6FD052
:10F3100098470224204602B0BDE8F08785F83800FF
:10F320002B78022B60D0474A6B68D2F8482803EA52
:10F330000208C8F34F282846FFF7BAFA414F06469D
:10F34000A8EB0008A7F5805901A902220023304646
:10F35000FFF7D2FA08EB060401281FFA84FA4FF4EB
:10F3600000724FF000010446D4D101985DF029FBF2
:10F37000EB694FF40071284613B16B68002B3BD04A
:10F38000D7F84038013B9A4506F101060DD2FFF748
:10F3900003FF0028D8D197F8E43713B9012387F881
:10F3A000E437012389F80130CEE7C3EBC353590298
:10F3B0002846FFF7F1FE40B997F8E43713B9012367
:10F3C00087F8E437204B01225A70022385F8383041
:10F3D0002B6C002285F8282063B128469847012429
:10F3E000204602B0BDE8F0876B68C3F34F28A2E760
:10F3F00002248FE701248DE7019B4FF020324FF06C
:10F400002E0E4FF0100C1A605A6083F800E0C3F81B
:10F4100007206C6A1A625A6283F80BC0C3F827206F
:10F4200083F820E083F821E0EA6B5C835A8724FAB2
:10F430000CF422FA0CF29C8283F82BC09A869FE788
:10F44000002467E7F4520020F44200202DE9F04147
:10F45000B1F904300F2B82B00E460446174635D062
:10F460002046FFF725FA94F91B80B8F1FF3F3ED004
:10F47000554B41F2186203EB08118A58904211D1A2
:10F48000183303EB4825B38801331BB205EB431552
:10F49000B38020463D60FFF70BFA3060012002B0D8
:10F4A000BDE8F08103F5805292F8E41700296AD094
:10F4B00001225A702278022A69D02369002B50D188
:10F4C000002301203B6002B0BDE8F0814FF40071E1
:10F4D000FFF762FE002852D04FF6FF73B38020463C
:10F4E000FFF7E6F994F91B80B8F1FF3FC0D122780D
:10F4F000022A54D02369002BDDD03349097803292F
:10F500000EBF32499BB24FF6F7718B4294BF002376
:10F510000123002BCFD138B92D4A92F8E437002BC4
:10F520004ED0294B01225A700023112201A9FFF766
:10F53000E3F9012842D1019D264BEB1A48BF03F2A3
:10F54000FF13B3F5B05F4FEA632230D3204A92F83D
:10F55000E43713B9012382F8E4371B4B01225A70B8
:10F5600027E0194A1278032A0EBF184A9BB24FF6B9
:10F57000F772934294BF00230123002BA0D10020F7
:10F5800002B0BDE8F081012182F8E41790E7104A4B
:10F590006368D2F85028B3EB422F91D2EFE70C4AC0
:10F5A0006368D2F85018B3EB412FB4D3F1E74FFAA8
:10F5B00082F884F81B80002D7FF465AF22787AE70B
:10F5C000012382F8E437ACE7F4420020F7FFFF0F95
:10F5D000F45200200C4300202DE9F04790F8303021
:10F5E00088B00446042B4BD8DFE803F0030C4DD160
:10F5F0004600C54859F0CCFC4FF6FF720123228427
:10F6000084F83030DFF8008304F11C0501AE04F10A
:10F610003109324629464046FFF718FF012800F01D
:10F62000DB8002282CD1B94901F5805595F90228D3
:10F63000531C0AD002F5B17201EB0212D3796FF3B9
:10F640000003D371FF2385F8023895F903385F1C56
:10F650000FD003F5B17301EB0313DA79C2F345015F
:10F66000013921EAE17161F34602FF21DA7185F87F
:10F670000318042384F830300020E36A2070984790
:10F6800008B0BDE8F087A24D95F81038002BF7D1EF
:10F690009D4F04F11C0901AE4FF00908324649465E
:10F6A0003846FFF7D3FE012840F0E8800198002893
:10F6B00000F0C2800378E52B01D0002BEED1954AF3
:10F6C000821A48BF02F2FF12B2F5B05F4FEA62231E
:10F6D00080F00E818D491B018F4A13449A7B042AC6
:10F6E0000CD0D5F8C8260132C5F8C8265A600422C5
:10F6F0009A73D5F8CC360133C5F8CC3695F9023873
:10F700005E1C0AD003F5B17301EB0313FF2285F8E9
:10F710000228DA796FF30002DA7195F903385A1C7E
:10F720000FD003F5B17301EB0313FF21DA7985F8EC
:10F730000318C2F34501013921EAE17161F3460280
:10F74000DA71202200215DF03CF9019BD4F83120D0
:10F75000D4F8351059601A60B4F8392094F83B1089
:10F7600099721A81019B627EDA7205A802F0B4F9DF
:10F77000BDF81430002B40F0058144F28171019AEC
:10F7800003201182D3811183D38284F83000237E39
:10F79000980608D5E0690023112205A9FFF7ACF807
:10F7A00001287FF46DAF204659F0F2FB2369002B4E
:10F7B00068D0237E03F0F70213F0040322766ED1A3
:10F7C000122A00F083800022E36A84F82820204671
:10F7D000984708B0BDE8F087019F002F00F09E8099
:10F7E0003B78002B00F09A8097F80BA01AF0080FD6
:10F7F0007FF40FAF0B22494638465DF01FF9002811
:10F800007FF407AF637E8AEA0303DB0640F1FB80E7
:10F810003E4901F5805595F902385E1C3FF415AF5D
:10F8200003F5B17301EB0313FF2285F80228DA799F
:10F8300060F30002DA7108E795F8E837022B3FF42D
:10F8400018AF95F81038002B7FF413AF85F82038E7
:10F85000C5F82438C5F8283885F81C38D5F8FC37A1
:10F86000C5F81438D5F8443885F81088C5F8183824
:10F870003846FFF731FD01283FF410AF02283FF46E
:10F88000F8AEFDE6237E19079DD5214B93F8C827D6
:10F89000002A7FF4F5AE072283F8C82793E7A5680E
:10F8A000E66A002384F8283029462046FFF774FCD6
:10F8B000002840F0A28094F82830002B7FF4E0AEBE
:10F8C0000223C4E90B6584F82830D9E6626AE16A4C
:10F8D000A163042084F82800C4E90B22C4E90233A0
:10F8E00084F83C3063636362204659F051FBC7E6FD
:10F8F00095F8E43713B9012385F8E4370349012368
:10F900004B706FF00F03E7E6DC5A0020F442002052
:10F91000F45200200C4300200C590020584901F5F6
:10F92000805595F902385E1C0AD003F5B17301EBDE
:10F930000313DA796FF30002DA71FF2385F80238D6
:10F9400095F90338581C0FD003F5B17301EB03137D
:10F95000DA79C2F34501013921EAE17161F3460226
:10F96000FF21DA7185F80318237EDA067FF581AE70
:10F97000444859F00DFB4FF6FF720223228484F8AD
:10F98000303081E6404B05A8B3F9A08501F0CEFFE9
:10F990004FF47A72002306460F465BF07BF83C2357
:10F9A000054608FB0355394630464FF47A7200236A
:10F9B0005BF070F84FF47A7192B20023C5FB01231B
:10F9C00002A801F0E9FF9DF80A209DF80B109DF8B0
:10F9D0000C3041EA4211BDF80820A2F2BC7241EAA3
:10F9E00042219DF80D20DB0243EA42139DF80E20D0
:10F9F00043EA520389B29BB2C1E6002E3FF440AE07
:10FA00002046B0473CE6BA8A7B8B204D43EA02434E
:10FA10006362D5F84028FB69A3605202B3FBF2F1A0
:10FA200002FB113109B113445B1AE36084F819A099
:10FA300095F902381249581C0AD003F5B17301EB4D
:10FA40000313DA796FF30002DA71FF2385F80238C5
:10FA500095F903385A1C0FD003F5B17301EB03136A
:10FA6000DA79C2F34501013921EAE17161F3460215
:10FA7000FF21DA7185F80318032384F8303086E615
:10FA8000F4420020DC5A0020A03C0020F452002068
:10FA900010B5037890F818C0023B012B044602D938
:10FAA0001CF0060F5DD11CF0200F3CD194F91A30E8
:10FAB000591C0AD0314A03F5B17302EB0313FF213D
:10FAC000DA796FF30002DA71A17694F91B305A1CCF
:10FAD0000FD02A4A03F5B17302EB0313DA79C2F3AC
:10FAE0004501013921EAE17161F34602FF21DA7132
:10FAF000E1761CF0080F0DD0214B93F8C827072A98
:10FB000005D093F8E427A2B31C4A012151700022CA
:10FB100083F8C827E26A0023237084F82830FAB1FA
:10FB2000BDE81040104700231649E0691A018A58C1
:10FB3000904206D001330B2BB8D01A018A5890425C
:10FB4000F8D10E4A03F5B17302EB0313DA79C2F36D
:10FB50004501013921EAE17161F34602DA71A5E755
:10FB600010BD0121FFF764F90128F9D194F818C0FC
:10FB700099E7012283F8E427C6E700BFF44200209A
:10FB8000F45200200C5900204FF0FF3C10B41A4AE8
:10FB90001A4C6046002304E001330B2B02F11002E3
:10FBA00017D011780429F7D103F5B17104EB0111D5
:10FBB000C979C907F0D4B0F1FF3F52F80A1C01D04F
:10FBC0006145E9D2184601330B2B8C4602F1100235
:10FBD000E7D1431C03D101205DF8044B7047074B6C
:10FBE00000F5B17003EB001083880BB91B69FFDED1
:10FBF0000023DB68FFDE00BF1A590020F44200201A
:10FC00002DE9F04F90F82830013B83B00446082BD3
:10FC10000BD8DFE803F0383C1E2305290A2E3300F9
:10FC20000121FFF747F9012802D003B0BDE8F08FAA
:10FC30002378002284F82820002BF6D0D4E9011381
:10FC40008B4238BF0B46226CA360032184F8281036
:10FC5000E262204603B0BDE8F04F19E7002103B08F
:10FC6000BDE8F04FFFF726B903B0BDE8F04FFFF74E
:10FC70002DBA03B0BDE8F04FFFF7BEB903B0BDE841
:10FC8000F04FFFF729BB03B0BDE8F04FA4E4534F9A
:10FC90004368D7F84858016BD7F840281D406818CA
:10FCA000B0EB422F4FEA42269C46C0F0938094F876
:10FCB00000E0DFF82C91A7F5805A4FF6F778BEF1F7
:10FCC000020F14D02069002857D1D4F804C0A368CB
:10FCD000E26A634538BF63460021A36084F82810B8
:10FCE000002AA2D0204603B0BDE8F04F1047D4F858
:10FCF00004C0D7F85028BCEB422FE8D22069227EFE
:10FD000012072CD5D7F8C42700F1010C624522D286
:10FD100097F8E42722B9012387F8E4376368216B59
:10FD200001228AF8012094F800E0891B2944334419
:10FD30005B1B8E42C4E904C0636021639C464FF0A4
:10FD40000005BCD9BEF1020F3ED020690028BED00C
:10FD5000DFF890B01FE0E8D14FF0000CE5E701A913
:10FD600057F03CFB01287FF460AF2069DDF804C048
:10FD700094F800E06368216BD7E79AF80020032A23
:10FD8000D3461AD082B2424594BF00220122002AF3
:10FD9000B5D0D4F804C09BF80030032B0EBF104B35
:10FDA00080B24FF6F773984294BF002001200028DC
:10FDB0008DD18C44C4F804C089E7484594BF002223
:10FDC0000122002A9BD0E4E7D7F85028B3EB422F5A
:10FDD000EFD37CE794F800E0B4E700BFF4520020D2
:10FDE000F7FFFF0FF442002010B5194C19484422C8
:10FDF00000215CF0E6FD237804F580544FF6FF7097
:10FE0000D4F84C28A4F80208022B4FF0030118BFC5
:10FE100003234FF0100C84F8001804F5FD60002156
:10FE2000C4F8F82784F8E837C4F80C2884F801C827
:10FE3000FFF7B2F948B994F8103833B9022284F8C0
:10FE40001028C4F81438C4F81838012010BD00BFB9
:10FE5000F4420020DC5A0020012143F20102002379
:10FE600043F2012C017202804FF47F41FF22A0F87F
:10FE700004C043818381C38101828274704700BFC3
:10FE8000154BFF224FF0FF3CF0B5C27002710272B9
:10FE900042724273827303F10C07664617251624DB
:10FEA0004FF0150E002202EB820281189F4200F8EB
:10FEB00002E04C708D70CE7081F804C00BD093F9C5
:10FEC000062093F807E01C7A5D7A93F90A6093F9AB
:10FED0000BC00633E7E7F0BD44E806084FF0000C1E
:10FEE00001210222032380F805C08171C2710372CF
:10FEF000704700BF00230222037043708370C370F9
:10FF0000027170472C22022302704370704700BFB9
:10FF10004FF0010C45210322002380F800C04170FE
:10FF20008270C370704700BF40F22E4C4FF4F071E6
:10FF3000A0F81EC001804FF4FA6C4FF47A71A0F85B
:10FF400020C0418440F2262C4FF4F561A0F81CC07B
:10FF5000818442F2267C42F220110023A0F808C0DE
:10FF600041814FF00E0C0221072280F826C0437118
:10FF70008371417440F2012C40F20341438240F20C
:10FF800005638270A0F814C0C18203838276704733
:10FF90008388C3F30B039342A8BF134670B51A4678
:10FFA0001D460C46064680685CF0A8FC6219944227
:10FFB000B569074B08D0074814F8011B00FB03F391
:10FFC000A24283EA0103F7D12B60012070BD00BF7C
:10FFD000C59D1C8193010001FF2303704370837052
:10FFE000C370704700220123027042708270C27099
:10FFF000037143718371C371704700BF00230370A5
:020000040801F1
:1000000043708370C3707047002303704370837024
:10001000C3707047002306214FF47A72C0E90123B0
:1000200001700373704700BF00230372704700BF65
:1000300037230370704700BF00234370C370037001
:100040000371704710B50023411CFF2200F81320F4
:1000500001F8132001330B2BF8D10B4B4FF0FF317C
:1000600003F10F0400228C4605E093F904C093F9D4
:10007000051013F8032F00F812C000EB420E9C424B
:100080008EF80110F1D110BD58E806084FF0260C8B
:1000900080F800C04FF0270C80F803C04FF0200C10
:1000A00080F806C04FF0210C022180F809C04FF003
:1000B000180C00230122C171817280F80CC0372115
:1000C0004FF02A0C42708370027143710372C37245
:1000D0004273837380F80FC0027443748174C274D6
:1000E0000375704703230370704700BF002303703C
:1000F0004370C37083700371704700BF0A4491421C
:1001000019D000B501F1FF3C02F1FF3E41F221019F
:100110001CF8012F082380EA022010F4004F81EA26
:1001200040020ABF400090B280B2013BF5D1E645E3
:10013000EED15DF804FB7047704700BFD0ED007A48
:10014000D0ED016A30EE677AE6EE877AB0EE670AA4
:10015000C0ED007A704700BFD0ED017AD0ED026AA1
:1001600030EE677A90ED000AE6EE877A37EEC07AD5
:10017000C0ED017AA6EE870A80ED000A704700BF45
:1001800090ED017AD0ED036AD0ED027A30EE470AA5
:10019000A6EE807A90ED000A80ED017A37EE676A6C
:1001A000E6EE867A37EEC07AC0ED027AA6EE870ACE
:1001B00080ED000A704700BFDFED277AB4EEE70A52
:1001C000F1EE10FA0CDDDFED256A9FED257AF0EEF9
:1001D000407AF4EEC77AF1EE10FA30EE660AF6DCF9
:1001E000DFED207AB4EEE70AF1EE10FA0CD5DFED80
:1001F0001B6A9FED1D7AF0EE407AF4EEC77AF1EEBD
:1002000010FA30EE260AF6D4DFED187AB4EEE70ADB
:10021000F1EE10FA14DDDFED107A37EEC00A60EE71
:10022000006A9FED136A9FED137ADFED137AA6EE55
:10023000867A20EE266AE6EE877AA6EE270A7047CF
:10024000DFED0E7AB4EEE70AF1EE10FA44BFDFED0F
:10025000057A37EEC00AE2E7DB0F4940DB0FC94001
:10026000E4CB1641DB0F49C0E4CB16C1DB0FC93F1D
:1002700092E741B99730083C15A82ABEDB0FC9BFE9
:10028000D0ED056AD0ED017A90ED007A90ED066A26
:10029000D0ED025A90ED035A80ED050A66EEA77A7A
:1002A000C0ED066AE7EE007A90ED077AE5EE867A11
:1002B00090ED086AD0ED045A80ED087AE5EE477AB1
:1002C000E5EEC67AB0EE670AC0ED077A704700BF68
:1002D000D0ED057A90ED006A90ED067AD0ED035AE4
:1002E000E6EE007A90ED016AF0EE406AA6EE267A1C
:1002F000B0EE670AD0ED047A90ED026A67EEC07A3C
:10030000A5EEC07AE6EE267A80ED057AC0ED067A93
:10031000704700BF2DE9F047089F3C460E4614F891
:10032000011B002B054614BF4FF030094FF0200988
:1003300041B3002A2CDD234600E0B2B113F8010BD3
:100340009046013A0028F8D1A8F102086AB1C246E5
:1003500049462846B0475346002B0AF1FF3AF7DCDE
:10036000397828EAE872013249B1D71B2846B047EC
:10037000E01914F8011B0029F8D1BDE8F0871046F8
:10038000BDE8F087002A02F1FF38E0DC0846F4E718
:100390000022EAE703685A1C02601970704700BF28
:1003A000024B186803681B68184700BF14A100209F
:1003B000884210B54FF001043ED301FB04F4B0FBBA
:1003C000F4FC8C45F9D2CCB122BB08E0A14203F881
:1003D00001EBB4FBF1F211D8B0FBF2FC1446BCF116
:1003E000090F0CF1570E0CF1300204FB1C00EDDC80
:1003F000A14203F8012BB4FBF1F2EDD900221A70EF
:1004000010BDA14203F801EBB4FBF1F2F6D8B0FB4A
:10041000F2FC1446BCF1090F0CF1370E0CF130025E
:1004200004FB1C00EDDCA14203F8012BB4FBF1F24C
:10043000EDD900221A7010BD8446002AEAD1CEE719
:10044000002870B503DA2D2301F8013B404209284A
:1004500086464FF0010307DD03EB83035B00B0FB2F
:10046000F3F2092AF8D8EBB1104CBEFBF3FCA4FB65
:100470000320C008BCF1090F0CF130060CF1570540
:10048000024607D8092B01F8016B03FB1CEE09D9C2
:100490000346EAE7092B01F8015B03FB1CEE01D9D7
:1004A0001346E2E700230B7070BD00BFCDCCCCCC6F
:1004B0000378202B024600F10100F9D0092BF7D078
:1004C0002D2B28D02B2B03BF5378B7EE000A024602
:1004D000B7EE000AA3F13001C8B209289FED567AA1
:1004E00010D8F2EE046A07EE901AF8EEE77A12F8E6
:1004F000013FE7EE267AA3F13001C8B20928B0EE39
:10050000677AF0D92E2B5ED003F0DF03452B07D09E
:1005100020EE070A70475378BFEE000A0246D9E77B
:1005200010B451782D2978D02B296AD0A1F130034D
:10053000092B02F101026BD80024002303EB830393
:1005400001EB430312F8011FA1F130000928A3F1C8
:100550003003F3D9B3F59A7F1A4628BF4FF49A7245
:10056000072B66D9DFED356A1346F7EE007A083BB4
:10057000072B67EEA67AFAD802F00702DAB1F2EE9C
:10058000046A012A67EEA67A15D0022A67EEA67AD7
:1005900011D0032A67EEA67A0DD0042A67EEA67A58
:1005A00009D0053A67EEA67A05D067EEA67A012A49
:1005B00018BF67EEA67A6CB387EE277A5DF8044B16
:1005C00020EE070A70475378A3F13001C8B209281A
:1005D00002F1010298D8F2EE046AF0EE665A07EED4
:1005E000901AF8EEE77A12F8013F87EEA66AA3F1B7
:1005F0003001C8B2092866EEA56A37EE067AEED950
:1006000082E79178A1F13003092B02F1020293D91C
:10061000F7EE007A27EE277AD0E79178A1F1300340
:10062000092B02F1020288BFF7EE007AC4D8012438
:1006300083E7F7EE007AA1E70000000020BCBE4C83
:10064000F8B5164D6B78BE2B25D1022229464FF600
:10065000FF70FFF753FD124FAC1C22884AB1A61859
:10066000BE4218D2052A16D92146FFF747FD344667
:10067000F3E721460222FFF741FD0222A118FFF70E
:100680003DFD0634074B641B9C8041F60F53C31A93
:1006900058425841F8BD0020FCE700BF0040000868
:1006A0000080000814A10020F0B5067906F0E003F0
:1006B000402B03D145794FF0FF3406E0602B4FF01B
:1006C0000105F8D1447905FA04F40023012006F06D
:1006D0000706AB4200D1F0BD052E0FD8DFE806F0CB
:1006E0000308101D242448B1C85CD75C78400FE093
:1006F00020B1C856D756C71B784278410133E8E786
:100700000028FBD031F8130032F81370784080B223
:1007100020420CBF01200020F0E70028EED031F984
:10072000130032F91370E6E70028E7D051F82300F0
:1007300052F82370DAE7037903F01803102B1CD06A
:1007400004D82BB1082B06D000207047182BFBD102
:10075000B0F80B007047104BB0F80B0093F9003065
:10076000591C06BF0D4B1B7ADBB203EB830203EB74
:10077000C20300EB830080B27047074BB0F80B0058
:1007800093F901305A1C06BF044B5B7ADBB2C3EB12
:10079000031300EB4300EEE77805002014A10020CE
:1007A000114A002330B50360838002F10C054FF439
:1007B00048744FF0290E4FF0280C03EB430300EB75
:1007C000430100F813C081F801E0D3788B70AA428E
:1007D0008C8008D092F9063092F807C092F808E0B1
:1007E00054890632E9E730BD6CE80608092900D0D3
:1007F00001B9704701394B0003F00802930001F082
:100800000301A3EB9203C1EB0111C3EB0313C1EB93
:10081000011100229B0089000260818043807047A3
:1008200084B04FF46173ADF804300199ADF80C1049
:10083000BDF80CC0A0F80CC041F2014100234FF4F8
:1008400000724180012100930280C2808360C181D7
:1008500004B07047144B154910B5044618681B794D
:10086000206284F82430152204F125005CF0FAF8A7
:100870000F4B1A7E4FF0010E84F83AE012B984F85B
:100880003B2010BD03F11C0CBCE80F002060616030
:10089000A260E360BCE80F0084F83BE02061616186
:1008A000A261E36110BD00BF3C5E0708445E07081B
:1008B00014A1002010B50021382204465CF081F814
:1008C0000D490E4A0E482061C4E905120D480E4A32
:1008D000E061012341F61E614FF0090CE18484F8C8
:1008E00008C0A37384F82130A26221460748BDE8FE
:1008F000104036F091BE00BF1A046C070019750352
:100900006400DC0543080E001E7D0101585E0708E7
:10091000B5EEC00ADFED347AF1EE10FACCBF30EE5E
:10092000270A30EE670ADFED317A20EE270A70B52C
:10093000FDEEC07A86B017EE904A054684EAE47070
:10094000002303A9A0EBE470CDE90033029353F038
:100950009BFD002CACBF20232D2303A88DF8003075
:1009600059F0D4FB01286E4628D0022832D0032843
:100970001CD003A930465CF02CF8304659F0C6FB79
:100980000338C4B22246314628465BF0B7FF002345
:100990002B55284659F0BAFB2E232B540130311920
:1009A00028445CF032F8284606B070BD302303A915
:1009B00030468DF801305CF00CF8DEE743F230028F
:1009C000302303A93046ADF801208DF803305CF0E8
:1009D00000F8D2E743F2300303A93046ADF8013006
:1009E0005BF0F7FFC9E700BF6F12033A00007A44DB
:1009F00009F082BC13B568B14C1E14F8011F21B96F
:100A000002B0BDE8104009F08BBC019009F074FC05
:100A10000198F2E702B010BD08B520215BF0E8FFB5
:100A2000034620B11A78202A00F10100F8D01846B8
:100A300008BDF8B5D0B1104B0138C70003EBC000BA
:100A4000CA4390F8406090F8415002F0010282EAF7
:100A50000604A5420AD0C06B28B185880068B2425E
:100A600014BF058345833B4483F84140CB0701D441
:100A7000FBF798FAF8BD00BF14A100202DE9F3415F
:100A8000124D134F002305F85C3F044600EB81062E
:100A9000B44203D10F4802B0BDE8F0813946284680
:100AA0005BF097FF214668465BF0AFFF4FF0000810
:100AB000202168465BF09CFF28B9694628465BF018
:100AC00088FF0434E4E780F80080F1E714A10020F7
:100AD000D8B1070870A10020024BD3F8800046F07F
:100AE0004FBB00BF14A10020704700BF084B09494D
:100AF0008B4202460AD2184602E01C30884205D2D8
:100B00000388C3F30B039A42F7D170470020704764
:100B100034F30708F0FC070870B50546B0F8090083
:100B2000FFF7E4FF064B93F8846004462846FFF77E
:100B300002FE16B1E368184470BDA368FBE700BF6E
:100B400014A1002038B505460C46FFF7E5FF2B79C8
:100B500003F0E002602A03F007032AD1052B0CD82A
:100B6000DFE803F0030B0F0B1B1B6A790123934093
:100B7000DBB2027814B11343037038BD22EA0303D9
:100B8000FAE76A79012393409BB2028814B11343B8
:100B90000380F2E722EA0303FAE76A79012303FA02
:100BA00002F2036814B113430360E6E723EA020389
:100BB000FAE7052BE1D8DFE803F003030505070793
:100BC0000470DAE70480D8E70460D6E770B585885A
:100BD0000B460446C5F30B052A46002118465BF078
:100BE000F0FE6169084A9142034602D3074A9142E6
:100BF00005D319B1BDE870401846084770BD2A46B4
:100C0000BDE870405BF07ABEF0FC070807FF0708FC
:100C100038B5064C064DAC4206D2A16820461C34BD
:100C2000FFF7D4FFAC42F8D338BD00BF34F3070858
:100C3000F0FC07084840082310F0800F82EA4001CA
:100C40000ABF4000C8B2C0B2013BF5D1704700BF37
:100C500030B505688D4219D901F1FF3E6C1E0023A5
:100C60001EF801CF082183EA0C0313F0800F82EAFB
:100C7000430C0ABF5B005FFA8CF3DBB20139F4D19D
:100C80007445EDD16A1C02602B7030BD00236A1CD4
:100C900002602B7030BD00BF07EE901AB8EE677A85
:100CA000DFED7C7A27EE000A60EE277ABDEEE77A68
:100CB00017EE103A2033402B00F2DB809FED767A5E
:100CC000B4EEC70AF1EE10FAB0EE677A0CDDDFED94
:100CD000735A9FED736AF0EE476AF4EEC66AF1EE5E
:100CE00010FA37EE657AF6DCDFED6E6AB4EEE67A7E
:100CF000F1EE10FA0CD5DFED695A9FED6B6AF0EE5C
:100D0000476AF4EEC66AF1EE10FA37EE257AF6D4A9
:100D1000DFED666AB4EEE67AF1EE10FA00F39D803C
:100D2000DFED636AB4EEE67AF1EE10FA44BFDFED70
:100D30005D6A36EEC77A27EE075ADFED5E5A9FED01
:100D40005E6ADFED5E6ADFED5E4AA5EE256A27EE9C
:100D5000054AE5EE066AF7EE005AA4EE267AF0EEB2
:100D6000656AE7EE646AE7EE245A86EEA54A9FEDCF
:100D70004F7A77EE877ABDEEE77A17EE103A203396
:100D8000402B6FD89FED4F7AB4EEC70AF1EE10FA00
:100D90000CDD9FED426ADFED426AB0EE677AB4EE99
:100DA000E67AF1EE10FA77EEC67AF6DC9FED3D7A40
:100DB000F4EEC77AF1EE10FA0CD59FED386ADFED4C
:100DC0003A6AB0EE677AB4EEE67AF1EE10FA77EEB0
:100DD000867AF6D49FED357AF4EEC77AF1EE10FA02
:100DE0004CDD9FED397A77EE677A67EEA74A9FED83
:100DF000317A9FED315ADFED316AA4EE875A67EE02
:100E0000A43AE4EE856AB7EE006AE3EEA67AB6EE9F
:100E1000007A36EE676AB8EE005A67EE857A26EEFB
:100E2000077AB7EE005AC5EE256A00238361436155
:100E30000362C36180ED044A26EE877A26EE866A55
:100E400066EEA77A80ED095A80ED007A80ED016A9E
:100E500080ED027AC0ED037A7047DFED1B6A36EE53
:100E6000C77A68E7DFED197AB6EE007AB7EE006A66
:100E7000D7E7B7EE004AF0EE445A78E79FED0C7AD8
:100E8000F4EEC77AF1EE10FA44BF9FED067A77EEE2
:100E9000677AAAE727D4D2360024F448DB0FC9408A
:100EA000E4CB1641DB0F49C0E4CB16C1DB0FC93FD1
:100EB000DB0FC9BF92E741B99730083C15A82ABE9D
:100EC000F304353F00247448DB0F49400000000064
:100ED0009FED2E7A70EE077AFDEEE76A16EE903AF5
:100EE0002033402B4FD8B4EEC70AF1EE10FA0CDDD8
:100EF0009FED276ADFED276AB0EE677AB4EEE67AF7
:100F0000F1EE10FA77EEC67AF6DC9FED237AF4EE76
:100F1000C77AF1EE10FA0CD59FED1D6ADFED1F6A5E
:100F2000B0EE677AB4EEE67AF1EE10FA77EE867AF2
:100F3000F6D49FED167AF4EEC77AF1EE10FA1DDCC6
:100F40009FED177AF4EEC77AF1EE10FA44BF9FEDE9
:100F5000127A77EE677A27EEA76ADFED125ADFED95
:100F6000126A9FED127AE6EE256A67EE865AA6EEC1
:100F7000267AE5EE877AB0EE670A70479FED0C7A25
:100F800077EE677AE7E79FED0B0A7047DB0FC93F03
:100F9000DB0FC940E4CB1641DB0F49C0E4CB16C1DF
:100FA000DB0FC9BF92E741B99730083C15A82ABEAC
:100FB000DB0F494000000000F0EEC07AB0EEE07AAE
:100FC000B4EEE77AF1EE10FAB4BFB0EE676AB0EEB5
:100FD000476AB5EE406AF1EE10FA46D0B4EEE77A11
:100FE000F1EE10FA8CBFF0EE675AF0EE475AC5EEFC
:100FF000866ADFED1F2ADFED1F3ADFED1F4A9FED06
:101000001F5A9FED1F3A9FED1F4ADFED1F5AE6EE74
:10101000E23AA6EE834AE6EEA34AB7EE006AA6EEEF
:10102000A45AA6EE846AE6EE855AC5EE866AB4EE48
:10103000E77AF1EE10FA48BFDFED147AF5EEC00A58
:1010400048BF77EEE66AF1EE10FA48BFDFED107A9E
:10105000B5EEC00A48BF77EEE66AF1EE10FA48BF77
:10106000F1EE666AB0EE660A7047DFED076ADEE70A
:1010700039094E3DE3B59E3E88FA163E45FE7F3F58
:1010800099FB243F69A2163EA7DFA834DB0FC93FB6
:10109000DB0F494090ED005A9FED4C0A35EE000AF7
:1010A00008B5FDEEC07A17EE903A2033402B7BD87E
:1010B000FFF782F8F0EE403AFDEEC57A17EE903A6F
:1010C0002033402B7FD8B0EE450AFFF775F8B0EE1D
:1010D000405AD0ED014A9FED3D0A34EE800AFDEE04
:1010E000C07A17EE903A2033402B69D8FFF764F8A6
:1010F000F0EE405AFDEEE47A17EE903A2033402BA2
:101100005BD8B0EE640AFFF757F8F0EE404A90ED76
:10111000023A9FED2E0A33EE000AFDEEC07A17EE7A
:10112000903A2033402B45D8FFF746F8B0EE404ABE
:10113000FDEEC37A17EE903A2033402B37D8B0EE4D
:10114000430AFFF739F8F0EE407A24EE233A27EE0F
:10115000A36A24EE057A67EE856AB0EE462AF0EEC1
:10116000432AA7EE242AE6EEE42AA6EE247AE3EE4A
:10117000646A24EE254A65EEE77A25EE655A65EE47
:10118000A35A81ED004AC1ED017AC1ED024A81ED19
:10119000032AC1ED042A81ED055AC1ED066A81EDED
:1011A000077AC1ED085A08BDDFED093A84E7DFEDA3
:1011B000087ACAE79FED064ABAE7DFED054AA6E7D7
:1011C000DFED035A96E79FED025A82E7DB0FC93F36
:1011D000000000002DE9F04389B0541C03941478FA
:1011E000002C00F007810025074688461E46A946C8
:1011F00009E021463846C047039A0135531C039342
:101200001478002C3DD0252CF3D1931CCDE9033963
:101210005078302800F09480A0F13003DBB2092B25
:101220004FF0000440F297806C2838D0782822D8FC
:1012300057282AD9A0F15803202B1CD8DFE803F047
:10124000B41B1B1B1B1B1B1B1B1B1B959D1B1B1B59
:101250001B1B1B1B1B1BAF1B1B1B1B111BA71B1BC8
:10126000B40056F8043B049A0093002341463846E4
:10127000FFF750F80544039A531C03931478002C8D
:10128000C1D1284609B0BDE8F0830028F9D025284F
:10129000F1D125213846C0470135039AAEE7039BBB
:1012A0005A1C039219787829A8D8572958D9A1F13E
:1012B0005803202BA2D801A050F823F0C113010835
:1012C000FD110108FD110108FD110108FD110108C2
:1012D000FD110108FD110108FD110108FD110108B2
:1012E000FD110108FD1101086B130108D913010854
:1012F000FD110108FD110108FD110108FD11010892
:10130000FD110108FD110108FD110108FD11010881
:10131000FD110108A1130108FD110108FD110108CB
:10132000FD110108FD11010863120108FD110108FA
:10133000E5130108FD110108FD110108C1130108A1
:10134000D31C03939078A0F13003DBB2092B4FF04C
:1013500001043FF669AF04AA03A956F00FFB63E747
:1013600000298ED0252994D048E756F8041B38462A
:10137000C9B2C0470135039A40E756F8040B05A9E6
:10138000FFF75EF805AB0093049A23466EE756F824
:10139000040B05AB00220A21FFF70AF8F2E7039AD3
:1013A00056F8043B1D6029E7A0F15802B2FA82F218
:1013B00056F8040B520905AB1021FEF7F9FFE1E7DF
:1013C000A1F15802B2FA82F256F8040B520905ABA9
:1013D0001021FEF7EDFFD5E756F8040B05A9FFF73E
:1013E0002FF8CFE756F8040B05AB00220A21FEF7D1
:1013F000DFFFC7E7254644E773B5144C0192064664
:10140000D4F888000D46C0B11149FFF7F3FAD4F8BB
:1014100088003146FFF7EEFA0E49D4F88800FFF74E
:10142000E9FA0D49019BD4F888002A46FFF7D2FE5D
:101430000A49D4F88800FFF7DDFA94F88C3013B12C
:10144000012384F88D3002B070BD00BF14A10020CC
:10145000D0A1070871A60708F1090108DDA1070856
:101460000EB400B584B005AB019053F8042B0649C7
:10147000039301A8FFF7AEFE019B00221A7004B08F
:101480005DF804EB03B07047950301082DE9F043C4
:10149000002483B0064604802146304601343FF0E4
:1014A000A5FA082CF8D10023DFF8688086F8EA3026
:1014B000C6F8EC30C6F8F030C6F8F430C6F8F830AC
:1014C0001F46FC3699463A46414601A8FFF7C8FF39
:1014D0003546032401AA12F8013B6BB1013C05F823
:1014E000013BF8D10137082F85F8009006F104067A
:1014F000E9D103B0BDE8F0832846224620212544E7
:1015000001375BF05EFA082F85F8009006F10406BB
:10151000D9D1EEE7645E0708F7B5114E07463046AD
:10152000002300F88E3F0C460E4B0F49002F08BFDA
:10153000194615465BF04DFA0C4F04EB45058E3607
:10154000AC4202D10A4803B0F0BD394634F8022B50
:101550006846FFF785FF694630465BF03AFAEFE7E9
:1015600014A10020EAA10708E1A10708F3A10708D8
:10157000A2A10020F7B50C4E0C4F002306F8BF3F88
:10158000044600EB4105AC4202D1094803B0F0BD6E
:10159000394634F8022B6846FFF762FF6946304649
:1015A0005BF017FAEFE700BF14A1002027ED070852
:1015B000D3A10020F8B5084F4E1E054601F11F04C7
:1015C00016F8012F28463946FFF74AFFA64205F1D3
:1015D0000205F5D1F8BD00BFF8A1070803685A1C41
:1015E000026019700368090A5A1C0260197070477A
:1015F00002681146531C036011F802CB0160D31C32
:101600005178036093781B0443EA0123111D0160A4
:10161000D07843EA0C0343EA00607047A0F130033E
:10162000092B07D920F02000413819288CBF002051
:101630000120704701207047303809288CBF0020F6
:1016400001207047413819288CBF002001207047C5
:10165000613819288CBF002001207047202805D050
:10166000093804288CBF00200120704701207047F2
:10167000A0F14103192B98BF20307047A0F16103FE
:10168000192B98BF2038704710B500F1004402466E
:10169000013C04E0B3EB0E0015D1A24214D012F8C5
:1016A000013BA3F14100192811F8010BA0F1410CF5
:1016B00098BF2033BCF1190F00F1200EEAD91B1A94
:1016C00004D10028E9D110BD002010BD184610BD7E
:1016D00002B310B58446841804E0B3EB0E0014D1B5
:1016E000A44513D01CF8013B11F8010BA3F14102F2
:1016F000192AA0F1410298BF2033192A00F1200EC7
:10170000EBD91B1A04D10028EAD110BD002010BD6E
:10171000184610BD1046704770B5044608460D4681
:1017200058F0F4FC064602E014F8013F43B12046AD
:1017300032462946FFF7CCFF0028F5D1204670BD80
:101740001C46204670BD38B507490546FFF7E4FF43
:101750000649041E284618BF0124FFF7DDFF08B123
:1017600044F00204204638BDFDA10708BFB80708B1
:101770002DE9F041044686469EF800C0BCF1200FDA
:101780007046ACF109050EF1010EF5D0042DF3D928
:10179000BCF12B0F5BD0BCF12D0F3BD1102A4FF0C9
:1017A000010600F1010E58D19EF800C0BCF1300FC7
:1017B0005FD04FF010086FF070450F2742460EF1D2
:1017C000010E00200DE0ACF1300C5FFA8CFC94456A
:1017D0000FDA854274462DD32AD008FB00C01EF8CC
:1017E00001CBBCF1390FEED94CF0200CBCF1600FED
:1017F0000BD801B10C600EB323B1B0F1004F28BF7C
:101800004FF000404042BDE8F081ACF1570C5FFA68
:101810008CFCDCE7102A864649D04FF0FF35B5FB3B
:10182000F2F502FB05F7FF43FFB290460026C6E73C
:101830006745D2D21E404FF0FF30D0E7002BE2D0F8
:101840006FF00043984228BF1846BDE8F081102A87
:101850004FF0000600F1010EA6D04FF0FF35B5FBAA
:10186000F2F502FB05F7FF4390F801C0FFB2904686
:10187000A5E79EF801C0ACF1410019280EF1010462
:10188000624601D80CF12002782A4FF0100805D0EA
:10189000A6466FF070450F27424690E79EF802C0BB
:1018A0006FF070450EF1020E0F27424687E70026C3
:1018B0007AE700BF01230A22002159E770B50D46DF
:1018C0001446FFF7A9F80646A0B1FFF7F3FF40F66C
:1018D00034039842A8BF1846B0F5617FB8BF4FF4F3
:1018E0006170A0F561731920B3FBF0F32B702378BE
:1018F000013323703046FFF78FF80646A0B1FFF79B
:10190000D9FF40F634039842A8BF1846B0F5617F6E
:10191000B8BF4FF46170A0F561731920B3FBF0F309
:101920006B70237801332370304670BD10B4028889
:10193000C378174CA2F5FA6202F0030140F2B55CDD
:101940009208013B0CFB0233827801EB4101013A22
:1019500002EB810204EB420102798C8F417923442E
:1019600003EB430302EBC30384790A4A0089C3EB08
:10197000031301EB8303C3EB0313224402EB830243
:1019800000214FF47A73C2FB03015DF8044B7047EA
:1019900044E8060880436D382DE9F04117461E469D
:1019A00005464FF47A7200233846314659F072F8F2
:1019B0004349444A014482FB0143C8170B44C0EB2E
:1019C000631382FB03021A44D8173F4CC0EB621228
:1019D00084FB02044FEAE27C3C48CCEBA40C80FB85
:1019E0000C404FEAEC74C4EBE010C3EB0314A1EB22
:1019F0008401A971C2EB0211A3EB81036B710CEBA3
:101A00004C03A2EBC30240F2B55303FB10CCBCF570
:101A1000896F2A714FEA800044DA40F2DA239C454C
:101A200047DCBCF5B77FB4BF00220122284B02EB94
:101A3000420103EBC1034FEA4208B3F8523091B2BE
:101A4000244C08EB020E04EBCE0416344FF00B0EC0
:101A500001E034F8023D63451FDDBEF1010EF8D10F
:101A60001B4B424403EBC2024FF0010E938F85F8EB
:101A700002E000F5FA600CF1010C0844ACEB030C39
:101A8000288085F803C04FF47A7200233846314627
:101A900059F000F82A81BDE8F0810EF1010E5FFADD
:101AA0008EFEE4E7032140F296530A464FF0060803
:101AB000C6E7022140F229430A464FF00408BFE777
:101AC00080BC92C789888888ABAAAA2A73B06D1691
:101AD00044E8060880E8060808B50C4BD3E9002363
:101AE00052EA030C09D1002340F2011242808380A4
:101AF000837103800381184608BD054909688A1867
:101B000043F10003FFF748FF012008BDF83C002027
:101B1000B822002090422DE9F0410B4604461546BC
:101B20000AD2B0FBF5F6134A05FB16441846135DBE
:101B300000F8013BBDE8F081B0FBF2F69642B6FB3F
:101B4000F2F706D20B4A05FB1767D15D03F8011BBC
:101B5000EAE7BA42B7FBF2F807D9064A05FB18785C
:101B600012F8081003F8011BEDE74046FFF7D2FF1B
:101B70000346F2E76C5E070830B5874CB4F8F433DF
:101B8000B4F8F803B4F8FA13B4F8FC23B3F57A7F89
:101B900084BF4FF47A73A4F8F433B4F8F633B3F592
:101BA0007A7F84BF4FF47A73A4F8F633B0F57A7F66
:101BB00084BF4FF47A70A4F8F803B1F57A7F88BF38
:101BC0000021B4F8FE3388BFA4F8FA13B2F57A7F87
:101BD00084BF4FF47A72A4F8FC23B3F57A7F84BFF4
:101BE0000023A4F8FE3388429CBF0021A4F8F81318
:101BF0009A4298BF0023B4F80A2498BFA4F8FC3393
:101C0000B4F80C349A4284BF0023A4F80A34634B1E
:101C10001B8883B02BB3627B614D012A48D9AA7817
:101C2000062A97BF5F499FED607A01EB820191ED33
:101C3000277A2979002940F08A8094F8141407EE55
:101C4000903A06EE901AF8EEE77AB8EEE66AAB79CB
:101C5000C6EE276A002B72D1B4EEE67AF1EE10FAE6
:101C600037DC637A032B14D8504AC3EB031302EB1F
:101C70004302237AC4F81C24032B12D84C4A03EBEA
:101C8000830103EBC10302EB8303C4F8203403B0E8
:101C900030BD00236372237A444AC4F81C24032B0A
:101CA000ECD9434BC4F820340022227203B030BD7B
:101CB000AA79002AB3D0AA78072A2AD0B3F57A6F76
:101CC000AED994F814140229B8BF022184F8141470
:101CD000A6E767EE277ABCEEE77A8DED017A9DF8EC
:101CE000042007EE102AB8EEC77AF4EEC77AF1EEB8
:101CF00010FAC4BF0132D2B2002A3CD0102AA8BFC9
:101D00001022D2B28A42134638BF0B4684F81434EC
:101D1000A7E70622B3F57A6FAA702ED82A79002A8F
:101D20009FD194F8141407EE903A07EE101AF8EECB
:101D3000E77AB8EEC76A9FED1F7AC6EE276A37EEDC
:101D4000077AB4EEE67AF1EE10FA8ADDC1E7042AEA
:101D500002D8002A85D002E0053A032A81D9B7EEDD
:101D6000000A80EE070A5AF051F82B88984228BFE3
:101D70001846288075E70122C3E794F814242979CE
:101D8000022AB8BF022284F8142400297FF469AF24
:101D90009FED087A51E700BF14A10020C00A00108F
:101DA000E428002044E806086F120338FCA1002054
:101DB00074A2002017B7D1382DE9F04FAC4E85B092
:101DC00096F82434A3F11702022A00AF00F2C18270
:101DD000A84BBB60DFF8BC9296F83C14DFF8B8B2B1
:101DE000A54D09F16C0A4C464FF0000834E010F0A4
:101DF000010C4ED1142A00F0A8824308820802F098
:101E0000333203F077331344C20802F01132C31A9D
:101E10009B1A03EB131303F00F33ABFB03E2D2095E
:101E2000C2EB02229A1A830302D5012A00F08D82A6
:101E3000012A0ED9082A00F28882BCF1000F01D0D5
:101E4000284206D1F96057F063FBF968002800F0DA
:101E50007C820C34544521D094F904202068A2F1EE
:101E60001E03DBB2012BC2D8A379022BA8BF022329
:101E7000A371E379022BA8BF0223E371237A022B1B
:101E800020F04100A8BF0223206023724FF0000C15
:101E9000B3E708F101085FFA88F8AEE708F1FF3808
:101EA000B8F1020F00F251820024022086F8DC44CF
:101EB00010F072F896F8E034022B00F0F782002858
:101EC00000F05E836D4B96F8AD8503F5247B4FF4EF
:101ED0007A7E4FF0000C5A88B2F57A7FB3F846202C
:101EE00088BFA3F802E0B2F57A7F9A8888BFA3F88A
:101EF00046E0B2F57A7FDA8888BFA3F804E09988D3
:101F0000B2F57A7F84BF0022A3F806C09142B3F8ED
:101F10005A10B3F85C2098BFA3F804C0914293F81C
:101F20006B2088BFA3F85AC0013A632A84BF642299
:101F300083F86B2093F86C200132D2B2092A88BF53
:101F400083F86CC003F16600194600228D7A10F800
:101F5000014B0132A54238BF00F801CC032A01F140
:101F60000601F3D1B8F1010F18BF83F885C0A4337F
:101F70009B45B0D1424B9B78042B00F0D4823BB9F7
:101F80003F4A1388B3F5F07F84BF4FF4F07313809A
:101F9000FFF7F2FD3B4896F8C015FEF727FC96F8D0
:101FA000DF151030FEF722FC96F8ED150E30FEF727
:101FB0001DFCB6F8FA25B6F8F8351343B6F8FC253B
:101FC00013431BB213B10123A6F8FE35D6F89C3596
:101FD0002D4A1A40002A00F0E982D90700F1438215
:101FE0005A0440F1D4812949D6F8A0250B400A4073
:101FF000C6F89C35C6F8A025180440F116820022C8
:1020000086F8432486F85324D90440F1198296F8BF
:102010000B36DFF87CB0022B04BF012386F80B36A9
:102020000BF178045B4602E006339C420CD01A7830
:10203000072AF9D19978DA78914202D35A79002A9D
:10204000F2D0072026F054FF00234FF4806086F87A
:10205000DC340FF0A1FF002800F07F820C4DA84671
:1020600098F8051029B398F8000000B35B4618E013
:1020700014A1002044E80608BC02020074A200205B
:10208000E4280020E4A6002009600002F6DFFFFD3E
:1020900024A7002080A500208180808006339C42F8
:1020A00007D01A788A42F9D15A79002AF6D026F058
:1020B0001FFF08F106084445D2D1B74B93F802B090
:1020C000BBF1080F00F0DD8196F8AD35D6F8A025FC
:1020D000A3F10103B3FA83F35B0986F8883696F817
:1020E000AE35A3F10103B3FA83F35B0986F88C36AE
:1020F00096F8F133032BC2F3C03188BF002386F872
:102100008A1688BF86F8F133A449D6F89C350A4070
:102110000B40B17DC6F89C35C6F8A025002900F01B
:10212000E981B6F8A036002B40F0F081D6F8A4364D
:1021300013F07F4F1CBF0023C6F8A436D6F8AC3688
:1021400023F4007323F002031BB140F20223C6F80C
:10215000AC3696F8A836013B042B84BF012386F8E1
:10216000A836ABF1050B8E4BBBF1030F93F890151E
:1021700040F2528111B30023FB60874B7C606FF00B
:102180000702A2EB0308444603F1080B884604E06B
:1021900004EB0B03434580F015811BF8010B00286D
:1021A000F6D00AF065FD0028F2D083799B07EFD5C1
:1021B000FA687C680123002A40F00A81764B9B79FB
:1021C00013B1754A00239371B6F8B63613F00C0FAD
:1021D00003D1C3F30313022B03D94FF42063A6F8F2
:1021E000B636B6F8B83613F00C0F03D1C3F30313A9
:1021F000022B03D940F60123A6F8B83696F83537F6
:1022000096F829279A4296F8283705D9002286F8A9
:10221000292753B1A6F82C2796F834279A4204D2DE
:10222000002386F82837A6F82C3796F81E3896F83B
:102230002A275C49FC609A4288BF0023BC6888BF9B
:1022400086F82A3701F1780B11F8013C03EB4303C0
:1022500023444FF0030893F870E293F871C293F8A7
:1022600072020B461A787245A8BF724603F8012B1A
:102270005A796245A8BF62465A719A788242A8BFCD
:102280000246B8F101089A70ECD11E318B45DBD1C2
:10229000D6F86424FC68002A00F026810020012181
:1022A0002B78282B07D16B78043301FA03F3134200
:1022B0001CBF9A4301200635AC42F1D108B1C6F8E3
:1022C0006424394D05F108042B4613F8012B072A25
:1022D00000F28B809C42F8D1EB4688B06B46FF2120
:1022E000184620225AF06DFB2F49034611F8012BA6
:1022F00053F8220001307FD18C4243F82220F5D1DF
:10230000B6F8A625B6F8A4359A42DD4602D3274B87
:10231000C6F8A435FF23264986F8503899F90430C9
:10232000142B05D0D9F8002031EA020200F0F88021
:1023300009F10C09D145F1D11E4B5A79022A00F05E
:10234000AB801437BD46BDE8F08F1B480FF0E0FDB1
:10235000AAE51A4ABA601146DA0001EBC30393F802
:10236000B81021B1D3F8BC30002B00F0F280BB686C
:10237000134493F8B920002A3FF42CAD93F8983118
:10238000002B7FF427AD182386F8243422E51D079F
:1023900072D50B4928E600BFE4280020FFDFFFFDCF
:1023A000C00A0010FFA10020F7280020AE014A015A
:1023B00001000200083D002080A5002044E8060836
:1023C000FE9FFFFDFA687C680023002A3FF4F6AE0A
:1023D0007C494A7C002A7FF4F7AE4A79012A3FF40F
:1023E000EDAE002B7FF4EAAEEEE6EB4688B020229D
:1023F000FF2168465AF0E5FA05F8018B08F101085B
:10240000B8F1080F3FF47CAF05F8018B08F1010823
:10241000B8F1080FF0D173E76A4A0023137100295D
:1024200000F0BB800123FB60A7E696F84324002A56
:1024300000F0A0800022D90486F853243FF5E7ADD0
:102440001A067FF5E4AD96F82414182906D85E4BD9
:1024500001228A401340002B7FF4D9ADDFF87CB114
:102460000BF17804F0E55949D6F8A0250B400A4055
:10247000C6F89C35C6F8A0259C047FF5BDAD54492F
:10248000B2E51A469B79002B3FF41EAE537C012B1C
:1024900004BF0223537417E696F85828002A7FF4E5
:1024A00050AF14375A71BD46BDE8F08F00283FF495
:1024B00009AD484B96F82D1590F904504FF0FF0CDC
:1024C00003F16C0093F90820AA4204D1013983F882
:1024D00008C0C9B201240C338342F3D1002C3FF46D
:1024E000F1AC86F82D15EDE4282026F001FDD6F894
:1024F0006424D3E638490B43C6F89C35B6F8A036B9
:102500000A43C6F8A025002B3FF410AE96F89C06AF
:102510000AF0AEFB00287FF409AEA6F8A00605E697
:1025200086F8503808E7D6F89C35264A23F48053BD
:10253000C6F89C35D6F8A03523F48053C6F8A035EC
:10254000538CB3F57A7FBFF423AD4FF47A73538481
:102550001EE5172386F8243409E7D6F89C3523F0C6
:102560000063C6F89C35D6F8A03523F00063C6F8A2
:10257000A03573E542F2010213427FF45BAF43E5FD
:10258000D6F89C25D6F8A03522F0800223F08003EF
:10259000C6F89C25C6F8A03594E4537C002B7FF444
:1025A00013AE5379012B7FF40FAE07E6D6F8A025C2
:1025B00043F0080342F00802C6F89C35C6F8A0258F
:1025C0000BE500BFE428002000410001F79FFFFD5C
:1025D000F6BFFFFD44A600202006370024A70020F8
:1025E0002DE9F04F884F97F85C38013B012B83B001
:1025F00040F2F280D7F89028844B02F2DC52C7F800
:102600009028834A934280F0FB8003F11C059B468F
:10261000804B814E4FF0010A03F102087D4B5A882E
:10262000002A00F0C28008EB0203B34280F0BD80B4
:10263000444608E01A881C461344002A00F0B5807E
:10264000B34280F0B280052A40F2AF8035F81C2CEE
:102650006188C2F30B029142ECD162799207E9D111
:10266000238855F8141C94F8049001935846FEF7FB
:10267000ADFA35F81C2CB9EB123F00F09E804FF0FC
:10268000000A35F8181C55F8140CC1F30B0153F06F
:10269000C1FF55F8043C18605D4B0BF11C0B9B45CA
:1026A00005F11C05BAD3D7F89C35C7F8A035FFF75C
:1026B00083FB3B7A594D5A4C03EB830203EBC20375
:1026C0007A7AA5F17801C2EB021201EB420205EB26
:1026D0008303C7F81C24C7F8203425F007FC4FF00B
:1026E000FF33D7F8200463602EF0EEFD26F054FC93
:1026F00005F5966305F5A56102E006338B4266D0C9
:102700001A78002AF9D19D78D878854202D3587971
:102710000028F2D097F80836227203EB830303EB0C
:1027200083039B00632BD8BF6423B7F80C26C7F83C
:102730008838642303FB02F2632AD8BF1A4639495A
:10274000CCBFC7F88C28C7F88C38C7F8A42800235A
:10275000354AC7F89038C7F89438C7F89838C7F89A
:102760009C38C7F8A038A7F8A83887F8AA38C1F865
:10277000402734F0FFFF97F8AE18B7F8AC0827F001
:1027800093FA44F0ABFD1BF017FB97F85C38013B64
:10279000012B2DD9254A1268C7F8902801235046ED
:1027A00087F8A93803B0BDE8F08F55F8141C5846D7
:1027B000FEF70CFA4FF0000A63E7019BA11D9A1F78
:1027C0005846FDF7E5FB00287FF45BAF57E7FA7D3D
:1027D000003A18BF01229DE709F01CFC00F5B71074
:1027E00000F558700223C7F87C0887F8803801E7A5
:1027F00009F010FC0223C7F87C0887F88038C9E785
:102800004FF0010A4FE700BF14A1002034F307087E
:10281000F0FC0708004000080080000874A20020B7
:1028200078050020C00A00100CA70020B822002064
:102830001C4B0122032870B51B4D83F84827064620
:102840001ED9711CC9B249004029184A28BF40212D
:10285000002302244FF0140ED454023302EB030C75
:1028600099420CF801ECF7D8FF2E08BF0221294449
:10287000FF2381F8B038BDE870400E200FF010BD86
:1028800000EB800005F5B07306EBC00003EB8000A1
:10289000C5F820042E722EF017FD2AF0C3F92AF095
:1028A00097FACEE7C00A001014A10020C4A90020A6
:1028B000054BD3F8F428012142F4001283F8F118F3
:1028C000C3F8F428704700BF14A10020F8B50468CD
:1028D000C4F30D0406460F460CB335683F6850F04C
:1028E000D7F9092840F08780444C236923F44073CA
:1028F0002361236943F400732361236943F00103D7
:1029000023612F6050F0C4F92369092823F00103E3
:10291000236170D1336804333360002034E0384BD6
:10292000384A93422AD302F58042934225D302F5D6
:102930008042934229D3344A934228D902F5803207
:10294000934226D902F50032934224D902F500328F
:10295000934222D902F50032934220D902F5003287
:1029600093421ED902F5802293421CD9B3F1016F24
:102970001BD355F0D3FE55F069F8082450F088F9C0
:10298000092814D04FF0FF30F8BD1024F6E71824C2
:10299000F4E72024F2E72824F0E73024EEE7382497
:1029A000ECE74024EAE74824E8E75824E6E7134D3B
:1029B0002B6923F440732B612B6943F400732B6163
:1029C0002B6923F0F8032B612B691C4344F00204AC
:1029D0002C612B6943F480332B6150F059F92B693A
:1029E00023F002032B612B69092823F0F8032B61E4
:1029F0003FF473AFC6E76FF00100C5E7003C02404B
:102A00000040000800400008FFFF00082DE9F041E9
:102A1000574F3B78B12B8AB06FD1FDF711FE80F094
:102A20000104E4B2534B544DB3F87F32534EADF82A
:102A3000003004F00104B54261D3002C00F0968010
:102A40001022002106A859F0BCFF4D4B0497DB1B58
:102A500005934C4B1A69002A04DA4B4A5A6002F17A
:102A600088325A6001228DF82420F322DA60694608
:102A7000022204A80025089556F0F6FF02226946B6
:102A80004FF6FF70FDF73AFB3B4F0446B74243D386
:102A9000022201A904A80025ADF8045056F0E4FF75
:102AA000022201A92046FDF729FB40BAC043ADF838
:102AB0000800022204A802A956F0D6FF079868B1C0
:102AC00006ABC0F104022946184459F07AFF089871
:102AD00018B906A904A8FFF7F9FE08909DF824305C
:102AE000089823B1274A136943F000431361B0FAF1
:102AF00080F040090AB0BDE8F081012492E7A9887E
:102B0000A868C1F30B0153F085FDAB691B681C3548
:102B1000834218BF01248EE7B7F804808DF80D506A
:102B2000C8F30B0808F10603ADF808303B88C3F37F
:102B30000B02ADF80A201B0B062202A904A88DF88F
:102B40000C3056F091FF062202A92046FDF7D6FA76
:102B5000B9680446424604A856F086FFB968204684
:102B60004246FDF7CBFA1C3704468FE70120C1E748
:102B70000040000844E8060834F30708F0FC0708A2
:102B800000800008003C02402301674510B5284C36
:102B9000FFF712F994F85C38013B012B21D9D4F8E6
:102BA0009038012203F2DC53C4F8903884F8F828F6
:102BB000FFF72CFF10B9FFF729FF50B11D4B1B7811
:102BC000B12B02D1FDF73CFDB8B955F0A7FD54F08B
:102BD0003DFFFFF71BFF0028F0D155F09FFD54F09B
:102BE00035FF09F017FA00F5B71000F55870022309
:102BF000C4F87C0884F88038D1E794F85C38013B4D
:102C00000022012B84F8F8280AD90B4B01221968FD
:102C1000C4F89018002384F8A92884F8F93810BD66
:102C200009F0F8F90223C4F87C0884F88038ECE74E
:102C300014A1002000400008B822002010B50B4A63
:102C40000B4C012382F84837A375FFF79FFFFFF76E
:102C5000C7FC41F20242FF23A4F8B02884F8B2383E
:102C60000E20BDE810400FF01BBB00BFC00A0010D3
:102C700014A1002090F88730DFED6A5A03EE903AF5
:102C800090F88B3006EE103A90F8893004EE103A46
:102C900090F88A30F8EEE33A04EE903A90F88D30EE
:102CA00063EEA57AB8EEC66A03EE903A26EE256A80
:102CB000B8EEC44AF8EEE44AF8EEE33A26EE276AA4
:102CC00024EE254A64EEA54A63EEA53AF0B5564DCA
:102CD00024EE064A64EEA74A63EEA73A00210626D0
:102CE000F7EE002AA5F10C0C00F1660E06FB01F2CE
:102CF000B7EE005AAC1890F886700244F0EE456AC0
:102D000015E0012904F1060402F10602EED190F863
:102D1000883007EE903A90F8903006EE903AF8EE50
:102D2000E77AF8EEE66A27EEA55A66EEA56A2378FA
:102D300007EE103A66EE867AB8EEC77A27EE277A63
:102D4000FDEEC77A17EE903AFA2BA8BFFA2323EAD2
:102D5000E3731372637807EE103A66EE847AB8EE86
:102D6000C77A27EE277AFDEEC77A17EE903AFA2B4C
:102D7000A8BFFA2323EAE37353725CF8213007EE0D
:102D8000903A002BF8EEE77A49DDA37807EE103A87
:102D9000B8EE477A90F88C3037EE677A03EE103A47
:102DA00087EE272AB8EEC33AB0EE627A23EE253AD0
:102DB000A2EE037A64EEA77A66EEA36A67EE857ADE
:102DC00027EE877AFDEEE77ABDEEC77A17EE103A66
:102DD000FA2BA8BFFA2323EAE373937217EE903A13
:102DE000FA2BA8BFFA2323EAE3730EF80130A38875
:102DF00007EE903AF8EEE77A013167EEA67AFDEE3B
:102E0000E77A17EE903AB3F57A7FA8BF4FF47A735A
:102E100023EAE3738F429381BFF673AFF0BDB7EE41
:102E2000007AC7E70AD7233C64ED060890F88E3095
:102E30006BB3B0F85A308BB190F88F2002EB82035D
:102E40006421C3EB0313B3FBF1F3A0F85A309623CC
:102E500012FB03F3B3FBF1F3A0F85C3043884BB1F2
:102E600090F88F3003EB8303C3EB03136422B3FBAF
:102E7000F2F34380B0F846304BB190F88F30962291
:102E800013FB02F36422B3FBF2F3A0F84630704761
:102E900090F821304BB3438B83B190F82230FA2263
:102EA00013FB02F203EB8303B3F57A7FA8BF4FF461
:102EB0007A7364218383B2FBF1F24283838843B146
:102EC00090F82230FA2213FB02F36422B3FBF2F3F0
:102ED0008380C3884BB190F8223003EB8303B3F5B2
:102EE0007A7FA8BF4FF47A73C380704770B50B4CDC
:102EF000002504F5247694F8863013B12046FFF7B8
:102F0000B9FE2046FFF792FF01353046FFF7C0FFBC
:102F1000042D04F1A404EED170BD00BF74A2002002
:102F2000034BD3F8E00F08B107F0FAB9704700BFC0
:102F300014A1002008B50B4605490246D1F8E00F60
:102F400028B10449FEF746F9BDE80840E8E708BDA6
:102F500014A10020F1090108024B0146D3F8E00F4B
:102F6000FDF748BD14A1002008B504460848FFF746
:102F7000F3FFFFF7D5FF074BD3F880000FF00EF9F2
:102F800009F09EFA012C01D154F060FDF9F70AF81E
:102F900005A2070814A100200048DDE747AE070896
:102FA0000CB4C30607B500D561B9049805A9019111
:102FB000FFF7C0FFFFF7F0FF012003B05DF804EB5F
:102FC00002B070470020F8E708B5FFF7C5FFBDE87D
:102FD0000840E1E710B504460348FFF7BDFF20466F
:102FE000BDE81040F0E700BF11A2070808B5094886
:102FF000FFF7F0FFFFF794FF074B002483F8E44F3F
:10300000064B43F8144C03F8104C2AF019F82046EC
:10301000FFF7AAFF16A2070814A100200CB2002097
:10302000034B0146D3F8E00F08B107F065B97047CC
:1030300014A100200CB407B510F020000BD079B912
:103040002320FFF7EDFF049805A90191FFF772FF18
:10305000FFF7A2FF012003B05DF804EB02B0704758
:103060000020F8E70FB407B504A951F8040B01914B
:10307000FFF760FF03B05DF804EB04B0704730B5B4
:103080002B4885B0FFF768FF2A4B93F8583823B9CF
:10309000294805B0BDE8304096E7FBF7EBFB08B9DF
:1030A0002648F6E7FBF7FEFB08B92548F1E7254B74
:1030B0001B68DB6998470028F7D0FBF7F5FB02682F
:1030C000037D81790446407C0290207C0190608AD7
:1030D000009052081C48FFF7C5FFE51D0C3415F899
:1030E000010BFFF79DFFA542F9D1184C1848FFF7D7
:1030F00033FF6378022B06D007D9032B10D1154874
:10310000FFF72AFF0CE01448FAE704F5805413484F
:10311000FFF722FF94F8E437022B05D0032B05D0EC
:1031200005B0BDE8304037E70D48E9E70D48E7E76F
:103130003DA2070814A1002047A2070856A20708CD
:1031400064A20708385E070873A20708F44200204B
:10315000A1A20708B1A20708B7A20708C4A20708DE
:10316000CAA20708E3A20708154B1B6870B52BB36A
:103170001448154EFFF728FFFFF7D2FEFAF7D6FDE9
:103180000025FAF709FE044640B113200FF088F835
:10319000FFF702FFBDE870400C4815E73046FFF727
:1031A00061FF782D06D80135FFF7BAFE642009F0DB
:1031B000D9F9E6E7FFF7F0FE2546F5E770BD00BF59
:1031C00070220020F5A2070890D407080FA3070873
:1031D0000FB407B504A951F8040B0191FFF7AAFE3B
:1031E000FFF7DAFE03B05DF804EB04B070472DE999
:1031F000F041037903F0E002402A50D004D85AB1DC
:10320000202A29D0BDE8F081602A4BD0802AF9D14C
:1032100082794179254812E003F00703052B16D87F
:10322000DFE803F0101510150309D0F80510204849
:10323000BDE8F041CCE7D0F8052051421D48BDE87B
:10324000F041C5E7B0F80720B0F80510F6E7B0F98F
:103250000720B0F90510F1E74679174D174805EB3F
:10326000C605FFF779FE95F8387500240123A742BB
:1032700002D8BDE8F0418FE6D5F8346556F8242031
:103280004FEA84084AB113B90D48FFF765FE56F8B6
:1032900008100C48FFF7E6FE00230134E7E7417908
:1032A0000948C5E7BDE8F041084891E764A307086D
:1032B00015A307082BA3070844E8060842A307083C
:1032C000BAA6070850B7070853A307087BA3070847
:1032D0002DE9F04387B0FAF719FD02698389018867
:1032E0000292826801924288009242681B4EDFF887
:1032F00080801B4FDFF87C9004461A48FFF768FF78
:10330000002515B94046FFF75FFE3B689D4213DA82
:1033100033781548052B96BF09EB83030022D3F8B9
:103320000C27B3880093294673880135FFF750FFB7
:10333000062D06F10606E4D154F046FB8188438849
:10334000CB1A616803FB01110591FAF769FD059934
:103350000246064807B0BDE8F04339E7D03C0020FC
:10336000403C002093A30708FDA307080CA407080E
:10337000F1A3070844E806080249034801F5216162
:103380000EC925E70070FF1F29A4070810B5752195
:10339000044634F0A5FC01460948FFF719FF1A213D
:1033A000204634F09DFC01460648FFF711FF1B2123
:1033B000204634F095FCBDE810400146024807E77E
:1033C0003DA4070850A4070863A4070838B50C4DAE
:1033D00095F8F30310F0FD0405D10A48FFF7F8FE55
:1033E0002046FFF7D3FF95F8F333013B012B06D8B6
:1033F0000548FFF7EDFEBDE838400120C6E738BDBF
:1034000014A1002076A4070881A407082DE9F04F35
:103410002DED028B794B7A491A687A4BB2FBF3F2A5
:1034200099B008EE100A7848FFF71CFE774BDFF8DA
:1034300050C20FCBDCF808700CAD85E80F00744B60
:103440000793BC08734B089314F00204C7F3810779
:1034500018AB18BFDCF8046003EB870318BFC6F392
:10346000805653F8301C002C00F0C68018AB03EBDC
:10347000860353F8442C684C6848694D694EDFF860
:103480000482DFF8C8A1FFF7EDFD34F80E2C4FF4ED
:103490007A73B2FBF3F103FB11220A2034F90C3CDE
:1034A00092B2B2FBF0F26048FFF792FE5F4A6049C9
:1034B0006048FFF7D7FDFFF76FFDA97D5E4A5F4BC0
:1034C0005F4806EB8101D31AD1F83417AA88FFF7B9
:1034D0007FFE5C48FFF740FD14F80A1C5A48FFF7CE
:1034E000C1FD5A48FFF738FD14F8091C5848FFF78A
:1034F000B9FDFFF751FD5748FFF72EFD00210A46A1
:1035000095F80F340B4113F0010F01F1010708D0BA
:1035100012B15046FFF720FD39464046FFF7A2FDA5
:103520000122072F3946EBD14B4F97F86A1507F563
:10353000EC7307F13C02012918BF134693F8DC3005
:10354000032B02D04548FFF78DFD454B97F86A15D0
:10355000A3F5CE72012918BF134693F8DC30012B76
:1035600002D14048FFF77EFD3D4B97F86A15A3F561
:10357000CE72012918BF13461B695B7B012B02D950
:103580003948FFF76FFDDFF800A1FFF705FD54F89C
:10359000083C03934FF000080AF1200B5AF8041B73
:1035A000002973D0012303FA08F9039B19EA030FDA
:1035B0001FD019F01F0F1CD02C4B5BF8282013F8DC
:1035C000080052F82020B8F1000F06D02848CDE9B5
:1035D0000412FFF7C1FCDDE904122648FFF742FDA3
:1035E000B9F1020F05D197F86D1A11B12248FFF712
:1035F00039FD08F10108D1E7204A3CE760220020AC
:1036000094A4070840420F0099A4070868EF060831
:10361000B6A40708BBA407080CB20020C0A4070882
:1036200014A1002044E80608C8A40708F0FF001011
:1036300000080000E9A40708008000080040000816
:103640000DA507083CA507084EA5070856A50708BD
:1036500058A5070860A50708C00A001079A5070843
:10366000980C001081A5070886A507089C05002076
:10367000BAA607088EA5070894A5070849AE07084B
:103680000038024070A5070880EF0608FFF784FCA9
:1036900095F8461ED5F8482E7B48137A527A06EBE9
:1036A0008101D1F87017FFF793FD784B78481968BE
:1036B0004FF47A73B1FBF3F1FFF7D4FC09A8FEF7DE
:1036C0000BFA38B109A910A856F0CAFA714810A926
:1036D000FFF7C8FCFFF760FCD4F88420002A00F054
:1036E0008F8007EE902ADFED6C6AB8EEE77AC6EEBF
:1036F000877AFDEEE77A17EE903AB4F87C0858B175
:1037000007EE900ADFED646AF8EEE77A86EEA77AB4
:10371000FDEEC77A17EE900A616859B107EE901A6C
:10372000DFED5D6AF8EEE77A86EEA77AFDEEC77AFE
:1037300017EE901AB7F8A87A642FCDE90001394640
:103740005648A8BF6421FFF743FD94F87E3894F8EB
:103750007F28B4F88018524806EB8303D3F88437E7
:10376000FFF736FD4F4B5048198889B2FFF730FDFF
:103770004E4918EE100AFFF782FCFAF7C7FA016902
:1037800021B182684A48120DFFF722FD4948FFF730
:10379000E3FBD5F8A0351B0662D594F8AC38032BB3
:1037A0008CBF45484548FFF7D7FB95F8E034022B1E
:1037B00028D14348FFF7D0FB94F8AC38042B46D807
:1037C0004048FFF7C9FB94F8BC38002B46D006EB05
:1037D000C303D3F8DC173C48FFF744FCFFF7DCFBDE
:1037E0003A4F3B48FFF7B8FBD5F8F4480125002CC9
:1037F0003AD1FFF7D1FB19B0BDEC028BBDE8F08FD9
:1038000013467AE702200EF0E9FB074608B9314873
:10381000D0E743F049FD97F9041006EB8000013131
:10382000D0F898272C48FFF71DFC95F8E334012BBE
:1038300004D12A48FFF790FB2948BBE7BB79294808
:1038400006EB8303D3F89817FFF70CFCF4E795F821
:10385000E2340BB92448B4E72448B2E72449BAE774
:103860002448FFF779FBB9E794FAA4F3B3FA83F39A
:1038700005FA03F206EB83033846D3F8101824EA5E
:103880000204FFF7EFFBB2E798A50708B822002073
:10389000AAA50708C4A5070800247449D7A50708E6
:1038A0001DA60708BC25002044A6070849AE070846
:1038B00053A607086EA6070874A6070880A607087F
:1038C00090A60708CFD60708CDA60708D9A60708EF
:1038D000E9A6070896A60708A0A60708B4A6070841
:1038E000B9A60708CEB00708BDA607084BA207086F
:1038F0008CA40708DDA607082DE9F04FDFF87881D2
:1039000098F80B3099B0002B00F098805148524E37
:10391000DFF868B1DFF86891DFF868A1FFF754FBC2
:1039200000252F460BA9E8B21AF0A2FC9DF834300E
:10393000002B53D0139C54B107EE904A9FED470AD9
:10394000F8EE677A80EE270A58F060FA04460B9A80
:1039500029465846FFF786FB109A002A70D002FBD2
:1039600004F04FF47A73B0FBF3F30993DDF848C029
:10397000BCF1000F66D00CFB04F142F21073B1FBF6
:10398000F3F198F80B30082D18BF7F18002B5BD08F
:103990001798079015980690169805900A23119885
:1039A0004FF47A7EB0FBFEFE0998CDF810E0B1FB33
:1039B000F3FE03FB1E11CDE902E10999B1FBF3F11E
:1039C00003FB1100CDE90010BCFBF3F32146504688
:1039D000FFF7FEFB0023C6E90D33B3620135222D4C
:1039E00006F140069ED198F80B3023B31C4C1D48BD
:1039F000D4F8C428D4F8C018D2084FF47A73B1FBB5
:103A0000F3F3D4F8C818FFF7E3FB0A221648B7FB14
:103A1000F2F102FB1172FFF7DBFB144B1B78432B17
:103A200006D1D4F8CC28D4F8D0181148FFF7D0FB31
:103A30000023C4F8C83819B0BDE8F08F0D4866E718
:103A4000099293E761469CE721464846FFF7C0FB91
:103A5000C0E700BFFFA6070808B200208096184BF9
:103A60000CB20020A6A70708C6A70708DC23002081
:103A7000EAA707085DA7070814A1002067A70708A1
:103A8000ECB6070876A7070813B52C48FFF764FAC9
:103A90002B4B93F85534002B4ED02A4C2A48FFF775
:103AA00093FA94F8403B2BB194F8423B13B194F84D
:103AB000413B83B9254B264893ED280A8DED010A39
:103AC000FFF74AFA234B9DED010AB3F87C3833BB6C
:103AD0002148FFF779FAB4F8441B2048FFF7C2FAEF
:103AE00094F8403B13B31E48FFF76EFAB4F8481B36
:103AF0001C48FFF7B7FA94F8423BCBB11848FFF7E0
:103B000063FAB4F8461B1848FFF7ACFA94F8413B47
:103B100083B1134802B0BDE81040FFF755BA58F022
:103B200075F981B21148FFF753FBD4E71048DBE782
:103B30000F48E4E70E48EDE70E48EBE714A8070846
:103B400014A10020C00A00102AA807086C15001054
:103B500031A807080CB200204BA807085AA807088C
:103B60007AA807088AA80708A4A8070855A807087C
:103B700083A807089DF007080EB403B503AA52F8FE
:103B8000041B0192FDF738FC064BD3F8E02F22B955
:103B90000549D3F88800FCF72DFF02B05DF804EB6F
:103BA00003B0704714A1002047AE07082DE9F04785
:103BB00098460B7903F0E004402C81460F461646E8
:103BC00031D1684DDFF8A081DFF8C091002422E0F8
:103BD0003B7903F00703013B042B04D8DFE803F033
:103BE00006080B0E2000315D28460AE03157FBE73E
:103BF00036F81410F8E736F91410F5E756F82410E3
:103C00004046FFF72FFA7B79013BA34202DD48468D
:103C1000FFF7A2F901347B79A342D9DCBDE8F08734
:103C200056F82410E0E703F00703052B58D8DFE827
:103C300003F0030C141619313578602C5ED045D88A
:103C4000002C66D0202C7CD0E8E796F90050602C40
:103C500054D03BD8002CF5D148E03588EDE7B6F9D3
:103C60000050F4E7D6F800A0202C554669D02BD898
:103C7000002CD3D151463C48FFF7F4F9D7F8051092
:103C80008A4518D8B8F1000FC8D03848BDE8F047C9
:103C9000FFF7E8B9202C356853D015D8002CBDD1DA
:103CA00029463048FFF7DEF9D7F80510A94202DBB4
:103CB0004B42AB42E6DDFFF76FF93A682C492B46E1
:103CC0004846BDE8F04757E7602C17D0802CA5D1B7
:103CD0003178284B2848002914BF31461946D5E7CA
:103CE000202C2DD007D8002C98D12546B7F90540B7
:103CF000B7F9076011E0602CE8D100257B7945FA1F
:103D000003F3DB07BDE8F0474CBF1C481C48FFF736
:103D1000A9B9B7F80540B7F8076012482946FFF778
:103D2000A1F9AC42C7DCAE42C5DBB8F1000F3FF4ED
:103D300075AF324621461348BDE8F047FFF792B908
:103D400000257A79104B03EBC20393F8382595428E
:103D5000B1DAD3F8343553F82500BDE8F047FFF762
:103D6000FBB800BF28ED070828A30708C4A8070868
:103D7000CAA807082CD5070850B7070890A307085A
:103D80009DF00708C0B1070844E8060856A50708D3
:103D900013B50446084601920091FCF7BDFEDDE92B
:103DA00000130246204602B0BDE81040FEE60EB405
:103DB00003B503AA52F8041B0192FDF71DFB054B46
:103DC0000549D3F88800FCF715FE02B05DF804EB56
:103DD00003B0704714A1002047AE0708014902460E
:103DE000E5E700BFE4A80708F8B5064608460C4614
:103DF000FDF760FD20210546204658F0F9FD0446F8
:103E000018B93046BDE8F840E8E7114F114E3B784D
:103E100032789A4201D0FAF7BBF80F4B20461D606A
:103E200056F074F9012201462046FAF759F83B781A
:103E300032789A4201D0FAF7ABF8204656F066F98C
:103E40002A460146BDE8F8400448FFF7C1B900BF63
:103E50006C220020483C002068220020FBA80708B4
:103E60002DE9F041064688B008460D46FDF722FDD3
:103E700020210446284658F0BBFD20B9304608B042
:103E8000BDE8F041AAE7FDF715FD224605460146CB
:103E90000F48FFF79DF985B1202D2A46694628BFB6
:103EA00020222046FAF790F8E84606460027B74257
:103EB00008DBAD1B3444002EEDD1FFF76DF808B0E0
:103EC000BDE8F08118F8010BFFF7AAF80137EEE71B
:103ED00011A9070810B504460748FFF775F8FAF767
:103EE00013F920B1BDE810400448FFF76DB8204633
:103EF0000349BDE810405AE729A9070833A9070874
:103F00003BA907082DE9F041144BD3F8303B88B0AA
:103F10000446F3B11A6804A9D56A18466A46A84748
:103F2000064688B1DFF8408004AC6D46002735F8BE
:103F3000022B34F8021B40460137FFF749F9BE4215
:103F4000F5DC08B0BDE8F08105492046FFF72FFFFA
:103F5000F7E7044908B0BDE8F04128E714A10020C4
:103F60005CA9070874A9070842A9070813B5044605
:103F70000846019156F0CAF8024670B1102804D1E3
:103F80000199094858F05AFD38B1074B074A0849CA
:103F9000204602B0BDE8104009E70349054802B0D9
:103FA000BDE81040FFF714B9445E07087BA9070875
:103FB00086A90708B0A9070813B504460846019169
:103FC00056F0A4F80199024668B1042803D10948C3
:103FD00058F034FD38B1074B074A0849204602B073
:103FE000BDE81040E3E60349054802B0BDE81040D3
:103FF000FFF7EEB83C5E0708BEA9070886A90708C8
:10400000CEA907082DE9F04306469BB008460C46AA
:1040100056F07CF8002705461C22394602A8019775
:1040200058F0CFFC25B3402D07D0394940232A460C
:1040300030461BB0BDE8F043B9E60DF1040804F1C9
:10404000400902222146684658F00CFD0023102248
:1040500009A968468DF80270FDF78AFB099B0DF1EE
:104060000202934222D10234A14508F8010BE8D1A3
:1040700000213D220AA8099158F0A3FC002D3AD056
:10408000244C257ED5B1202204F11C0101A858F052
:104090006EFC98B104F11C0109A8FDF78BFA1E4AC9
:1040A0001E4909AB3046FFF782FE04E01A781C492E
:1040B0003046FFF77CFE1BB0BDE8F08394F88430F7
:1040C000CBB9C5B901AD0FCD164C0FC495E80F00A3
:1040D00084E80F00144B012209A8A4F1100183F811
:1040E000D428FDF767FA1148FEF774FF104809A9B4
:1040F000FFF76EF8DFE70C4B93F8D4381BB9054B8C
:104100001B7E002BF2D0074909A8FDF753FAEDE713
:10411000E1A9070814A100201FAA070886A907081B
:1041200003AA070830A100200CB2002029AA070822
:1041300038AA07082DE9F74F834608460D4655F083
:10414000E5FF374F0446D7F89C95B8B93548364D4A
:10415000364FFEF701FF012655F8041B49B106FA58
:1041600004F313EA090F02D03846FEF77BFF01344F
:10417000F2E703B0BDE8F04FFEF70EBF02462C4950
:104180002846FDF7A5FA78B92A48274C2A4DFEF7AC
:10419000E3FE54F8041B0029EBD00B78002BF8D079
:1041A0002846FEF75FFFF4E72B782D2B1E4B03BF4D
:1041B000013504F1FF344FF0010A4FF0000A0026E8
:1041C00053F8048BB8F1000F06D11C492A46584613
:1041D00003B0BDE8F04FEAE5224641462846019388
:1041E000FDF776FA019BC0B90123B340BAF1000F85
:1041F0000DD029EA03031248C7F89C35FEF7ACFE40
:104200000D48414603B0BDE8F04FFEF7E1BF49EA73
:1042100003030C48C7F89C35F0E70136D0E700BF30
:1042200014A1002045AA0708BCF006084FAA0708F9
:1042300062A7070853AA0708D9A607085EAA0708B5
:104240006FAA070878AA07082DE9F74F81460846A4
:104250000E461746984655F059FF0446E8B93F48C0
:104260003F4DFEF7FFFE20460DF03AFC3B6818423A
:1042700006D020460DF046FC01462846FEF7F2FE29
:104280000134182CEFD13B6813B93648FEF764FEB1
:1042900003B0BDE8F04FFEF77FBE0246324930461C
:1042A000FDF716FA0546A8B93048FEF755FE2C462C
:1042B0002F4D20460DF014FC10EA080F06D02046C2
:1042C0000DF020FC01462846FEF7CCFE0134192CE7
:1042D000EFD1DDE733782D2B48F0807303BF013633
:1042E00004F1FF34012500254FF0000A01935046E8
:1042F0000DF008FC2246834601463046FDF7E8F9FA
:1043000000BB50460DF0ECFB019B03421AD08DB16F
:10431000BAF1180F1CBF3B6840EA03081548C7F8FC
:104320000080FEF719FE1248594603B0BDE8F04F71
:10433000FEF74EBFBAF1180F1CBF3D6885433D60C4
:104340000D48EEE70AF1010ABAF1190FCFD10B4976
:104350003246484603B0BDE8F04F28E580AA07087A
:10436000D8A607088AAA070862A7070853AA070859
:10437000D9A607086FAA070878AA07085EAA07083F
:10438000014A40F202235FE7C0A70020014A6FF014
:104390007F4359E7B8A7002010B5044633F0B0F9C1
:1043A00020B920460449BDE8104000E5BDE81040B2
:1043B0000248FEF70DBF00BF91AA0708A0AA070890
:1043C00070B5054608461646FDF774FA0D4B93F88E
:1043D00090259042044605D201460B48FEF7F8FEB0
:1043E000204670BD2EB1FF2803D10848FEF7F0FE2D
:1043F000F6E70749013A2846FFF7D9FC4FF0FF34AA
:10440000EEE700BFC00A0010ABAA0708BCAA070865
:10441000CFAA07082DE9F04F074691B08248834D97
:104420000E46FEF7D5FE8249C5F8D8D8002385F898
:10443000DC380622012391F890153046402485F897
:10444000DD4808F005F80A2008F08CF895F8DC380B
:104450000C2BDAB240F2E4809DF80C50FE2D30D0E7
:10446000FF2D0BBF15240F2401260026944240F097
:10447000D780611EC9B2684649F054FF04F1400379
:104480000DEB030414F8413C834240F0C48006F174
:10449000FF385FFA88F8B8F1010F9DF80D3012D996
:1044A00003F01F0761375C096248FEF755FD022ED5
:1044B0006AD0013C042C65D8DFE804F00B5E606430
:1044C00062000226D2E79DF80E709DF80F401D464F
:1044D000EAE75948DFF8BC91DFF8BCB1FEF774FD9C
:1044E0005648FEF739FD6C464FF0000A14F8011BE0
:1044F00048460AF1010AFEF7B5FDBAF10C0F49D1A1
:10450000FEF74AFD022E4FD06422B5FBF2F102FB0A
:1045100011524B483B46D2B2C9B2FEF759FEB8F130
:10452000010F71D8474A484B9DF810104748484D35
:10453000002914BF11461946FEF74AFE9DF81110D6
:10454000444B4548002914BF19462946FEF740FE52
:10455000022E59D19DF812404048FEF7FDFC4CB3A5
:10456000FF2C37D00A22B4FBF2F102FB11423C4887
:10457000D2B2FEF72DFE20E03A48ABE73A48A9E771
:104580003A48A7E73A48A5E700238DF83F300DF1F8
:104590001F009FE7374B03FB0AF2B2F1553FA5D846
:1045A0005846FEF7D9FCA1E733483A462946FEF7BC
:1045B0000FFEB7E72846FEF707FD9DF813402F488A
:1045C000FEF7CAFC44B1FF2C21D02D482146FEF74E
:1045D000FFFD04E02B48EEE71D48FEF7F5FC1C4EFE
:1045E000284FDFF870800DF11305002415F8013F06
:1045F0007BB1FF2B0CBF3A4642462146224801348C
:10460000FEF7E6FD042CF1D111B0BDE8F08F1D4896
:10461000E3E73246F1E71D493846FFF7C8FBF3E709
:104620001B48FEF7D1FCEFE715AB07080CB20020E2
:10463000C00A001026AB070831AB070857AB0708C4
:1046400069AB0708F5AA0708FEAA0708A0AB070888
:1046500005AB070892B80708B7AB0708BEAB070859
:10466000D2AB070838AB070840AB070848AB0708D0
:104670008CA40708ABAAAAAA85AB0708DAAB07087F
:1046800028ED070809AB0708EAAB0708F5AB0708F0
:1046900005AC0708F8A107082CD507082DE9F84F45
:1046A000DFF8A880DFF88890DFF8A4A007460C4662
:1046B000204655F02BFD064660B91D4B1D4893F86A
:1046C00024241D4B03EB8203D3F8F018BDE8F84F08
:1046D000FEF77EBD024641462046FCF7F9FF60B179
:1046E000DFF860B000255BF8041BB1B922463846FC
:1046F0001249BDE8F84FFFF75ABB1148114C124D53
:10470000FEF72AFC54F8041B19B12846FEF7AAFC50
:10471000F8E7BDE8F84FFEF73FBC32462046FCF70D
:10472000D7FF01350028DED189F824545446BFE76D
:1047300014A100200EAC070844E806085EAA07088A
:1047400053AA070838F10608D9A6070862A7070880
:1047500049AE070838B50D4604461A4905222846D1
:10476000FCF7B6FF68B9184B93F88C2022B90121E9
:1047700083F88C1083F88D20BDE838401348FEF78D
:1047800023BC134903222846FCF7A2FFA0B90E4D13
:1047900095F88C3063B195F88D304BB10D492046BA
:1047A000FFF705FB002385F88C3085F88D3038BD88
:1047B0000948FEF709FCF5E720460849BDE83840FE
:1047C000FFF7F5BAD3B7070814A1002018AC070803
:1047D0003BB907082EAC070865AC070879AC070899
:1047E000F8B5174C94F88C3005467BB194F88D30B1
:1047F00063B11449FFF7DBFA28461349FFF7D7FAEC
:10480000002084F88C0084F88D00F8BD0F4E96F8D7
:10481000D47897B1207E0028F7D10D4D0FCD06F545
:104820000E640FC495E80F0084E80F00012386F89A
:104830001B3908F083FB3846E7E70120E5E700BFB6
:1048400014A100202EAC070888AC07080CB2002089
:1048500030A1002008B5FFF7C3FF50B1054B01227E
:104860009A75FEF793F90448FEF7B4FB0020FEF7B3
:104870007BFB08BD14A10020A6AC070808B50346C1
:1048800010462AB1DB0600D511B1FEF7A3FB0020CC
:1048900008BDF8B50D4E96F88430054693B9F8BDBD
:1048A00025B12388C3F30B039D4204D0D4E9020150
:1048B000A28858F023F81C34BC42F1D3002386F8B8
:1048C0008430ECE7024C034FF6E700BF14A1002050
:1048D00034F30708F0FC07082DE9F04F85B01646C1
:1048E00001911A46824600213046FFF7C7FF324C3D
:1048F00006F0100305464FF000090293FEF710FB87
:104900002379019A03F01803934203D0002A48D177
:10491000182B46D1284B4FF00D0B0BFB0933B3F886
:104920000900FCF7E3F880462046FBF704FFD8E9CE
:1049300002210746024401442046FBF7B5FE80F001
:1049400001012A460390C9B23046FFF797FFDDE91F
:104950000223054602B123BB174A0BFB09FB52F8A1
:104960000BB0B2060FD573B9144803935946FEF73E
:1049700079FBD8F80820039B3A4421465046FFF7BC
:1049800015F9FEF709FB0E485946FEF76BFBD8F800
:104990000C2000233A4421465046FFF707F9FEF762
:1049A000FBFA09F1010940F27E23994504F10D0457
:1049B000A4D105B0BDE8F08FECFF0608ADAC070848
:1049C000AEAC07080149FFF7F2B900BFB8AC070861
:1049D00038B50C46054615492046FCF755FE30B95A
:1049E000FEF784FA1248BDE83840FEF7EDBA1149E7
:1049F0002046FCF749FEA0B90F4A82F8E60182F88A
:104A0000EE0182F88A0282F8920282F82E0382F87E
:104A1000360382F8D20382F8DA0382F811040748D9
:104A2000E1E72846BDE83840CCE700BFC7AC07083F
:104A3000CDAC0708E8AC070814A10020F0AC0708CB
:104A40002DE9F043064687B008460C4655F05EFB5C
:104A5000082843D1671E03AD073429463A46A846C5
:104A600012F8010FFCF70AFEA24201F8010BF7D180
:104A70000023DFF87C908DF8143017F8010FFCF755
:104A8000FDFDC1B205F8010B4846019157F0B0FF9A
:104A900020B10199284657F0ABFF28B13046FFF707
:104AA00091FF07B0BDE8F083A742E6D10F49404629
:104AB00032F0B2FD0D480E49082310F8012B11F811
:104AC000014B18326A44013B02F80C4CF5D10948FD
:104AD0008DF8143003A9FEF77BFBE2E70028E9D04C
:104AE000304607B0BDE8F043FFF778B948A500208D
:104AF000A86D07080CAD07082DE9F74F064601AA77
:104B000008462F49DFF8C880DFF8C890DFF8B0A06A
:104B100057F02AFF4FF0000B04465D4601271CBBEF
:104B2000BBF1000F28D1274C002D44D02648294640
:104B3000FEF74EFB94F884300BB904F025FFFCF728
:104B400067F8002384F88D30FEF7D0F915B12846B8
:104B5000FFF79FFE9FB13046FFF742FE78B1FEF7A8
:104B600015F80020FEF700FABBF1000F0AD020462E
:104B7000FCF7A0FE85B2C5B93046FFF723FF03B0AE
:104B8000BDE8F08F41462046FCF7C6FD80B9494696
:104B90002046FCF7C1FD0028EED05F4601AA514631
:104BA000002057F0E1FE0446B9E74FF0000BF5E7AF
:104BB0004FF0010BF2E70548FEF70CFABFE700BF24
:104BC000D8B1070814A100201CAD07083FAD0708A5
:104BD00013AD07080AB8070807B5009313460A463D
:104BE0000249FFF7E4F803B05DF804FB55AD070890
:104BF00020B10078B0FA80F040097047012070477A
:104C00002DE9F34106460846FFF7F2FF0D46074639
:104C100070B1002401A920464FF036FC0134014652
:104C20003046FFF7EDFF122CF4D102B0BDE8F08161
:104C30000846FCF73FFEC4B2112C71D8681CFBF784
:104C4000EBFE3B4D8046E8B93A4B03EB440393F847
:104C50001C198A1E51425141364B03EB440393F811
:104C60001C29AA5C002954D093F81D39192040F260
:104C7000EE2100FB03133048214602B0BDE8F041AD
:104C8000FEF7A6BA0178284657F0B2FE70B1032CA1
:104C900094BF00220122294902EB4202431B0A442D
:104CA00052FA83F393F86079032F04D1304602B0AF
:104CB000BDE8F04186E64046FBF7AEFE08B3022FA2
:104CC000F4D1FCF7F7FD40F6CA0280B29042194BCE
:104CD000A8BF104640F2EE22904203EB4403B8BF57
:104CE0001046A0F2EE201922B0FBF2F083F81D0965
:104CF000BB1E594259410F4B03EB440383F81C7907
:104D0000AAE7022FF4D1304602B0BDE8F041FFF728
:104D100065B80B48214602B0BDE8F041FEF758BA2D
:104D2000084911233A46304602B0BDE8F04153E746
:104D3000C86F07080CB200206EAD070844E80608EB
:104D40007EAD07088BAD07082DE9F04F024691B004
:104D50000846FFF74DFF0B46044628B1104611B038
:104D6000BDE8F04FFFF73AB84FF0FF32CDE9082029
:104D7000A74ADFF8E482D2F88020DFF8E09292F8C8
:104D80003810DFF8DCA2CDE90C10CDE90E02CDE938
:104D90000A00A04907AA184657F0E6FD274605462F
:104DA000049426464DB9089A0C9FBA4262D19A489B
:104DB000FEF70EFA11B0BDE8F08F062F12D8DFE82B
:104DC00007F0041E2328454C510051462846FCF7A5
:104DD000A3FC78B14FF480600DF000F990F9043035
:104DE000089301248B4907AA002057F0BDFD013725
:104DF0000546D7E72846FCF75DFD0890F2E7284610
:104E0000FCF758FD0990EDE72846FCF79CFC0A905A
:104E1000E8E7284655F07AF94146024605902846CB
:104E2000FCF756FC18B3059A49462846FCF750FC97
:104E300006460028D6D02846FCF73CFD0428064646
:104E4000D0D901467548FEF7C3F9B3E72846FCF709
:104E500031FD00230C900F93C4E72846FCF72AFD90
:104E60000D90BFE72846FCF76EFC0E90BAE70123D1
:104E70000493B7E7DFF8EC8151B2434613F9010B15
:104E8000884208D00135092DF8D10021644801314C
:104E9000FEF79EF98EE763480121FEF799F97AB291
:104EA000002318F9011B8A4200F00D810133092B00
:104EB000F7D13A460121E9E7A7F1140253425341E1
:104EC000059308AD002303F10108EB68A3BB95F936
:104ED00000B058460DF04AF8D5F804A020B1D0F83B
:104EE0000090B9F1000F5ED1BAF1000F19D14FF463
:104EF00061436B604FF0010AAB680BB90323AB60F1
:104F00000023D5F8049002932A7A1946CDE900923D
:104F100058461A460DF0C9F8E86028B9424841469B
:104F200091E74FF0000AE7E74A464146BAF1000F21
:104F300037D03E48FEF796F8B8F1020F05F110059C
:104F40004FF00103BFD1059BDDF83C800B9D53B1B1
:104F50003748FEF739F8D8F800301B6A1BB13549DD
:104F60002A4640469847049B002B4ED03249334B8B
:104F7000142F18BF19463248FEF72AF9142F09D109
:104F8000049B03B936B12B68DB691BB12D4932464E
:104F900028469847002C67D10022414628464FF00A
:104FA00027FA2948C6E7C5F80C90BAF1000F25D0BA
:104FB000264841465246FEF755F85146484602F00B
:104FC000A5FED5F808A0BAF1000F0FD099F804207B
:104FD00092450BD01E4853464146FEF743F8D9F898
:104FE00000305FFA8AF19B6948469847D9F82C301F
:104FF000002BA1D00023C9F82C309DE7D9F8082058
:1050000014484146FEF72EF8DBE70C49B3E700BF32
:1050100014A10020D8B10708C9AD0708B1AD070831
:105020000DAF0708E2AD0708EEAD07080AAE0708A6
:10503000C1AE07080D7D010893AD070849AE07080A
:10504000EAAE0708330A01082EAE07084AAE070881
:105050009CAE070877AE0708ABAD07088CAA070817
:10506000A0AD070800EC060805F072FF052007F068
:1050700079FA1A4FDFF86C9000264FF0030A99F87E
:105080009035B34288D917F801BBBBF1000F15D09A
:10509000584607F0EDFD044680B1584605F090FEF5
:1050A00008B1A0F806A001210490F5F737FFA37915
:1050B000049813F0010F03D0F5F7CCF80136DEE7C2
:1050C000F5F7B8F8FAE706483A460221FEF780F805
:1050D000099B002B3FF4F0AE0023F1E6EC28002002
:1050E000E2AD0708C00A001010B5044608460B469A
:1050F000FFF77EFD28B9094903221846FCF7E8FAB4
:1051000028B90748FDF766FF0120FDF72DFF20466F
:105110000449BDE81040FEF74ABE00BF1FAF0708B4
:1051200023AF070879AC07082DE9F74F0546084675
:10513000FFF75EFD0B46044618B9334A92F84079F2
:1051400027B9284603B0BDE8F04F3BE42F49DFF80C
:10515000C880DFF8C890DFF8C8A001AA184657F049
:1051600003FC264610B905F001FF08E056B90122FC
:1051700001462846FFF724F9421C04461BD103B020
:10518000BDE8F08FFCF796FB2F28834636D80FB189
:1051900005F0DEFEBBF1060F14D01D49012391F886
:1051A00090155FFA8BF2E0B207F052F95946484683
:1051B000FEF70EF80027154901AA0020013657F026
:1051C000D3FBCFE7DAF8A0351B0113D5FF2C0FD0A6
:1051D000E1B22846FFF71EF9E8E72846FFF71AF97B
:1051E00001370B4B93F89025F9B28A42F5D8DDE7E9
:1051F0000027F6E70748FDF7E7FED7E72F224146ED
:105200002846FEF7D4FDD6E70CB20020D8B1070837
:10521000C00A001091AA070856AF070845AF070853
:1052200014A100202DE9F04F064685B00846FFF78F
:10523000DFFC0B46044628B1304605B0BDE8F04F10
:10524000FEF7CCBD3149DFF8D490DFF8D4A0DFF809
:10525000D4B003AA184657F087FB27460546A04658
:1052600065B92B4B3A46D3F88000A1B24EF012FE3E
:1052700068BB28493046FEF79AFD28E0B8F1000FD8
:1052800006D0B8F1010F25D03046FEF7A7FD1EE08D
:10529000284654F03BFF4946024601902846FCF759
:1052A00017FA50B3019A51462846FCF711FA30B369
:1052B000019A59462846FCF70BFA10B3019A164991
:1052C0002846FCF705FAF0B13046FFF77BFB05B046
:1052D000BDE8F08FBB1E5A425A4129463046FFF7BF
:1052E0006FF8421C0446F2D0084903AA002057F088
:1052F0003BFB08F101080546B2E74746F4E7012702
:10530000F2E70227F0E70327EEE700BFD8B107086E
:1053100014A1002082AF07087FAF070876AF070807
:1053200079AF07087CAF07082DE9F74380460846A8
:10533000FFF75EFC0B46054628B14046FEF74EFDE2
:1053400003B0BDE8F0832E49DFF8B49001AA1846F7
:1053500057F00AFB2F4604462E467CB9022DECD1AD
:10536000A7F57A73B3F57A7F21D926494FF4FA630A
:105370004FF47A724046FFF72FFCE1E74DB1012D63
:1053800010D001AA4946002057F0EEFA0135044634
:10539000E3E7012221464046FFF712F8431C064688
:1053A000EFD1CDE72046FCF785FA0746E9E7164D31
:1053B000D5F84C3AB8B25B689847FF2EBCEEC00AED
:1053C000124B0BD195F89025F8EE407AA24212DCF0
:1053D00010EE101A0E48FDF7FBFEB1E7F8EE407A2A
:1053E00003EB860310EE102A0A48C3ED007A31461B
:1053F000FDF7EEFEA4E7E3EC017A0134E6E700BF37
:10540000D8B1070890B00708C00A001050BB0020B0
:10541000ADAF0708A0AF0708F8B507460846FFF785
:10542000E7FBC8B11F4BDE6A013630460CF06AFB61
:1054300034460546F0B90134192CA8BF0024204693
:105440000CF060FB0546A8B9B442F4D138461649C1
:10545000BDE8F840FEF7ABBC0846FCF72BFA044663
:105460000CF050FB054628B921461048BDE8F8402D
:10547000FDF7AEBE0B4BDC620CF0DCFE0C482A469E
:105480002146FDF7A5FE182C09D80A480C2101FB7E
:10549000040090F86809BDE8F8400CF001BF002056
:1054A000F9E700BF78050020BCAF0708D0AF0708B8
:1054B000E6AF070844E8060838B5124D044608462A
:1054C000FFF796FB60B1104B104893F900104B1C8E
:1054D0000ABF0F4BC9B2197ABDE83840FDF778BE54
:1054E0000846FCF7E7F9032804D8C0B2FDF7A0F995
:1054F0002946E4E720460749BDE838400322FEF785
:1055000056BC00BF49AE070878050020FFAF07086A
:1055100014A100200FB0070838B5124D0446084604
:10552000FFF766FB60B1104B104893F901104B1C5C
:105530000ABF0F4BC9B2597ABDE83840FDF748BEE3
:105540000846FCF7B7F9032804D8C0B21DF0E8FB01
:105550002946E4E720460749BDE838400322FEF724
:1055600026BC00BF49AE070878050020FBAF07083E
:1055700014A100200AB007082DE9F74F444BDFF8CB
:1055800028A11A7A8AF800205A7A93F884308AF887
:105590000120054688460BB904F0F6F9FBF738FB05
:1055A00000263C4CB1460D233A4A7343414652F81B
:1055B00003B05846FCF7B0F8002841D0B9F1000F0D
:1055C00001D0FDF7E9FC34485946FDF74BFD0022B8
:1055D00021462846FEF7DCFBFDF7DEFC237903F0CD
:1055E0001803082B46D0102B49D02046FDF7FFFDAD
:1055F000284A0D2303FB0623B3F80900FBF776FACC
:105600000746D8B12046FBF796F8D7E9022100906B
:10561000024401442046FBF747F878B90190594607
:105620001E48FDF71FFD019AB9681346009A2846E7
:105630000A442146FEF7BAFAFDF7AEFC09F101096A
:10564000013640F27E239E4204F10D04ABD10020CE
:10565000FFF71FF9FF238AF800308AF80130B9F10B
:10566000000F11D10E494246284603B0BDE8F04F65
:10567000FEF79DBB0B492846FFF71EFFB5E709491A
:105680002846FFF749FFB0E703B0BDE8F08F00BF41
:1056900014A10020ECFF0608B2AC07082AB00708E6
:1056A0005EAA070849AE0708780500202DE9F74FE4
:1056B000074608460E4654F029FD044620B101284D
:1056C00026D132782A2A23D1B348B44EDFF8E892A3
:1056D000FDF77AFC0025B2464FF00D0B40F27E2814
:1056E0000BFB05F348465AF80310FDF7BBFC221EDE
:1056F00018BF0122314638460135FEF749FBFDF758
:105700004BFC454506F10D06EAD103B0BDE8F08F2C
:105710003D21304657F06CF9002800F037810146F2
:105720000A4611F8014D202CFAD0921B0130814617
:1057300010F8011B2029FAD0DFF860B25FFA82FA74
:105740004FF000080D2303FB08F10BEB0104524658
:105750005BF8011000913046FBF7BAFF05460028C0
:1057600057D10099084654F0D1FC824551D1267991
:1057700006F0E001402900F0CC800ED8002956D078
:10578000202900F09E8038468549FEF710FB204610
:1057900003B0BDE8F04FFDF72ABD602900F092800C
:1057A0008029F0D1484654F0B1FCE379A679DB07B3
:1057B00005460CD52046FBF7AFF90378014633B117
:1057C0002A46484657F03AF9002840F0D980002D83
:1057D00000F0D680AE42C0F0D3800D2303FB08B3A7
:1057E000204693F805A0FBF797F93246002157F0C1
:1057F000E8F8AA452CD86B492A46484657F01EF9C6
:1058000030B32046FBF788F92A46494657F076F828
:105810001EE008F1010840F27E23984592D16249CA
:105820003246384603B0BDE8F04FFEF7C0BA06F086
:105830000703042B1CD10B460A224846FBF798FFAE
:10584000D4F80530834201469DD32046FBF77AF910
:105850000D2303FB08F855485BF80810FDF702FC20
:1058600000222146384603B0BDE8F04FFEF790BA5B
:10587000052B0FD101230A224846FBF779FFD4F804
:10588000053083420146FFF67EAF5B4283423FF71D
:105890007AAFDAE74846FCF70DF8B4F80550B4F8EB
:1058A000071016F0050FAAB218BF2AB28BB218BFA4
:1058B0000BB29042FFF667AF98423FF764AF0146E4
:1058C000C3E765793A4A02EBC505002695F8382505
:1058D0000092B2463346009AB24202D9BAF1000FA2
:1058E00003D0002B3FF44FAFB2E7D5F8341551F891
:1058F000260060B149460193FBF7C6FE019B30B913
:10590000314620464FF0010AFBF71CF95346013699
:10591000E1E76379009306F00706013E009BAB4286
:1059200096DD4846814610F8013B202BFAD02046F0
:10593000FBF7F2F88246042E04D8DFE806F00310E5
:1059400010161F004846FBF7B5FF0AF80500484649
:105950002C2157F04DF8013500F10109DEE74846EA
:10596000FBF7A8FF2AF81500F1E700230A2200211F
:105970004846FBF7FDFE4AF82500E8E70123F5E776
:105980000C4932463846FEF712FAFCE631463846F4
:1059900003B0BDE8F04FEFE53AB00708ECFF0608AA
:1059A00088B007082CD507085EAA07087DB007084D
:1059B00044E806084DB00708B2AC07082DE9F04FDF
:1059C000914689B00C461A4600218046FEF756FFE4
:1059D000DFF8ECB006464D460027B9F1000F6CD059
:1059E00029460622204656F0C2FF0028324614BF40
:1059F0000121002140460CBF4FF0010A4FF0000A80
:105A0000FEF73CFF0646287818F0AAF9079010B375
:105A1000687918F0A5F9079BEA785B790793AB786A
:105A200095F801E04FF461714FF0190C1CFB031362
:105A30001CFB0212297900B14079CDF804E0CDE9D0
:105A40000232079B0093CDE904103B465A4651466B
:105A50004046FDF7EFFA207818F082F9079010B36E
:105A6000607918F07DF9079BE2785B790793A3785A
:105A700094F801E04FF461714FF0190C1CFB031313
:105A80001CFB0212217900B14079CDF804E0CDE988
:105A90000232079B0093CDE904103B465A4651461B
:105AA0004046FDF77DFA0137142F04F1060405F195
:105AB000060592D109B0BDE8F08FCA46CBE700BF1A
:105AC00096B007082DE9F041064686B00846FFF774
:105AD0008FF80F46054638B100235D491A4601206C
:105AE00006B0BDE8F04169E70846FBF7E3FE13287E
:105AF000044600F3A38006264643781C8DF8175011
:105B0000FAF78AFF534D074670B1FBF7D3FEC0B2D8
:105B100018F03CF940B1AB19027983F810269DF8D2
:105B2000173001338DF817303846FAF775FF0746FE
:105B300068B1FBF7BFFE0D2809D8062303FB045309
:105B400083F811069DF8173001338DF81730DFF810
:105B50000081B11C0DF1170241443846FBF7AEFE3F
:105B6000FAF75AFF074668B1FBF7A4FE012809D8E7
:105B7000062303FB045383F814069DF81730013302
:105B80008DF817303846FAF747FF80B1FBF792FEE1
:105B9000C0B218F0FBF850B1062303FB045302799E
:105BA00083F815269DF8173001338DF817309DF8CE
:105BB0001720042A4FF006032FD103FB04530022C1
:105BC000A3F8142623F0E8F9062303FB04554FF449
:105BD000617695F8100618F0C3F895F8132695F835
:105BE00012761923804695F8150613FB076713FBF9
:105BF000026618F0B5F8437998F80520039395F8F4
:105C000014360097CDE90163134895F81136214603
:105C1000FDF7DEFA06B0BDE8F081052A05D103FBE9
:105C20000453002283F81526CCE7062ACAD008EBD5
:105C30000602002348F806309380C3E70749132380
:105C40002A46304606B0BDE8F041FEF7C5BF00BFAA
:105C500024A7002014A1002096B00708AFB00708C1
:105C60002DE9F04F174689B01A460C4600218146AF
:105C7000FEF704FE3B4EDFF8F4B007F16C038046FC
:105C80003D46079394F90410374A002392F908001F
:105C9000884263D00133092B02F10C02F6D1079B35
:105CA0000C359D4204F10C04ECD109B0BDE8F08F35
:105CB00029460C22204656F05AFE0028424614BFC0
:105CC0000121002148460CBF4FF0010A4FF0000AA5
:105CD000FEF7D4FDEA7995F9043006EB820280469E
:105CE000D2F8982704922A7A06EB82025146D2F81B
:105CF00098270392AA7906EB82024846D2F89827A1
:105D000002926A7906EB8202D2F8982701922A68F9
:105D100000925A46FDF78EF9E27994F9043006EBC9
:105D200082025146D2F898270492227A06EB820228
:105D30004846D2F898270392A27906EB8202D2F85D
:105D400098270292627906EB8202D2F89827019294
:105D5000226800925A46FDF723F9A0E7002FA7D149
:105D6000BA46D9E744E8060844A60020B5B00708BB
:105D70002DE9F04380468BB00846FEF739FF38B175
:105D800000234D491A4601200BB0BDE8F04367E7F8
:105D9000CDE90700099008464D1CFBF78BFD44B286
:105DA00020460CF09FF80646002843D08DF820408E
:105DB00001242846FAF730FE054638B100230A22AE
:105DC0001946FBF7D5FC01340790E4B2DFF8F090F8
:105DD00000272846FAF720FE054618B3FBF76AFDB0
:105DE0003649002251F804CB6045D3B203D00132CA
:105DF000102AF7D1002309EB8302D2F898279042AA
:105E000010D1022F1DD0032F20D05A1E012FD2B245
:105E100012D00B2A03D88DF821300134E4B20137B7
:105E2000042FD6D1052C17D840460BB0BDE8F0435F
:105E3000FDF7D4BF0446BCE7042AF0D88DF8223021
:105E4000EBE7052BEBD88DF82430E6E79A1E0D2AF8
:105E5000E5D88DF82330E0E707AB03CB9DF823208E
:105E600030601868164B716003EB8202B060D2F8A4
:105E7000982704929DF8242003EB82020021D2F897
:105E8000982703929DF8222003EB82020846D2F85D
:105E9000982702929DF8212003EB8203094AD3F848
:105EA00098370193079B00939DF92030FDF778F810
:105EB0000BB0BDE8F08300BF80A50020DCEF060832
:105EC00044E80608B5B007082DE9F04F8BB00C4642
:105ED000089200211A460746FEF7D0FCDFF8B4B05E
:105EE000089D099000264FF019094FF46178089B2E
:105EF000002B4BD029460A22204656F038FD0028B8
:105F0000099A14BF0121002138460CBF4FF0010A45
:105F10004FF0000AFEF7B2FC2A890692EA88059241
:105F20002A790492EA780392AA78099019FB0282EE
:105F300002926A7819FB028201922A780092334613
:105F40005A4651463846FDF775F822890692E2888E
:105F5000059222790492E2780392A27819FB0282D8
:105F60000292627819FB0282019214F80A2B0092C5
:105F700033465A46514638460136FDF711F81E2E73
:105F800005F10A05B3D10BB0BDE8F08FDDF820A014
:105F9000DBE700BFD2B007082DE9F04380468BB0A5
:105FA0000846FEF725FE0F46044638B10023654932
:105FB0001A4601200BB0BDE8F04385E70846FBF721
:105FC00079FC1D28054600F3B3800A264643781C59
:105FD0008DF82740FAF720FD044630B1FBF76AFC44
:105FE0009DF8273001338DF827302046FAF714FD4D
:105FF000554C074668B1FBF75DFC0D2809D80A230C
:1060000003FB054383F864099DF8273001338DF8BD
:106010002730DFF83091711C0DF1270249443846D2
:10602000FBF74CFCFAF7F8FC074668B1FBF742FCBB
:10603000222809D80A2303FB054383F867099DF842
:10604000273001338DF827303846FAF7E5FC07464C
:1060500068B1FBF72FFC0D2809D80A2303FB054381
:1060600083F868099DF8273001338DF827309DF8B3
:106070002730062B0CD009EB0602002349F8063026
:10608000404653601381FDF7A9FE0BB0BDE8F083D5
:106090000A2606FB054600233846A6F86A39A6F804
:1060A0006C39FAF7B9FC074640B1FBF703FC9DF8E1
:1060B0002730A6F86A0901338DF827303846FAF7F9
:1060C000ABFC58B1FBF7F6FB0A2303FB0543A3F82F
:1060D0006C099DF8273001338DF827301B4B4FF0AA
:1060E000FF325A600A2202FB05424FF46170B2F897
:1060F0006C390693B2F86A39059392F868390493BB
:1061000092F86739039392F86619192313FB01017A
:10611000029192F8651913FB0103019392F8643917
:10612000009300210A4A2B460846FCF739FFACE7EA
:1061300008491D23224640460BB0BDE8F043FEF758
:106140004BBD00BF70BB00200CB2002078050020C2
:10615000D2B00708AFB007082DE9F04F2DED088B3E
:10616000DFF82CA195B0804691461F460C46164696
:106170004FF0000B94ED008AB5EE408AF1EE10FA74
:106180007FD0D4ED019A94ED029AD4ED038AB9F14F
:10619000000F49D0D6ED00BA96ED01BAD6ED02AAAD
:1061A00096ED03AAB4EE6B8AF1EE10FA6ED1F4EE1E
:1061B0004B9AF1EE10FA69D1B4EE6A9AF1EE10FA48
:1061C00064D1F4EE4A8AF1EE10FA0CBF01210021ED
:1061D0003A460D46404681F00101FEF74FFBB0EE16
:1061E0006B0A074611A8FAF793FBB0EE4B0A07902B
:1061F0000EA8FAF78DFBB0EE6A0A06900BA8FAF724
:1062000087FBB0EE4A0A059008A8FAF781FB0599CA
:10621000069A079B039002910192009352465B46B7
:1062200029464046FCF706FFB0EE480A11A8FAF7E7
:106230006FFBB0EE690A05460EA8FAF769FBB0EEEF
:10624000490A06900BA8FAF763FBB0EE680A0590BE
:1062500008A8FAF75DFB069B059A0390CDE9005369
:1062600002925B465246002140460BF1010BFCF7BF
:1062700097FEBBF1080F04F1100406F110067FF43D
:1062800079AF15B0BDEC088BBDE8F08F00219FE71A
:10629000F5B007082DE9F74FDFF898A1DFF898B1BE
:1062A00007460D462846FEF7A3FC064638B10023F4
:1062B00059491A46012003B0BDE8F04F4CE70522CA
:1062C00051462846FBF704FA60B9534B00221A6086
:1062D0001A611A621A631A641A651A661A6703B099
:1062E000BDE8F08F4D4904222846FBF7F1F904463A
:1062F0002846002C44D1FAF78FFB80460028EED0C8
:1063000053F004FF464BC2B253F8049BB9F1000F9F
:1063100007D144492A46384603B0BDE8F04FFDF79F
:1063200046BD49464046CDE90023FBF7D1F901348B
:10633000DDE9002306460028E6D1374A0346154624
:1063400000210133082B42F8101BFAD10BEBC404D7
:10635000D4F8BCC0BCF1000F03D094F8B8E0764587
:1063600005DB3148314D4946FCF732FF9AE70CEB2B
:1063700006130FCB05EB061484E80F000136EEE799
:10638000FBF798FA072804463DD82846FAF744FB5D
:10639000064658B3FAF78CF81F4B03EB041383ED52
:1063A000000A01253046FAF737FB064638B1FAF7FE
:1063B0007FF8194B03EB041383ED010A01353046D6
:1063C000FAF72AFB064638B1FAF772F8124B03EBDC
:1063D000041383ED020A01353046FAF71DFB38B984
:1063E000384603B0BDE8F04FFDF7F8BC0546D9E7E5
:1063F000FAF75EF80848032D00EB041484ED030A55
:106400003FF455AFECE70A4907233246384603B05C
:10641000BDE8F04FFEF7E0BB54AA002009B1070821
:1064200038F106085EAA07080EB1070849AE07084A
:10643000AFB00708ABAD070844E806082DE9F74FF1
:1064400092460C461A4600218146FEF717FADFF8FD
:1064500070B0804656460025BAF1000F2ED0314666
:106460000422204656F083FA0028424614BF012138
:10647000002148460CBF01270027FEF7FFF973886B
:1064800001933AF82530009380462B465A46394608
:106490004846FCF7CFFD6388019334F8043B009332
:1064A0005A462B46394648460135FCF779FD042DFE
:1064B00006F10406D0D103B0BDE8F08F5746EAE7F5
:1064C00018B107082DE9F34105460846FEF790FB91
:1064D0000C46074638B1002333491A46012002B062
:1064E000BDE8F041AAE731492046FBF7CDF8034665
:1064F00070B92D4A4FF47A704FF4FA610133042BCE
:106500001080518002F10402F8D102B0BDE8F081A0
:106510002046FBF7CFF90328064641D82046FAF774
:106520007BFA074670B1FBF7C5F94FF00108044646
:106530003846FAF771FA48B9284602B0BDE8F0418A
:10654000FDF74CBC40F2EE248046F1E7FBF7B2F9D0
:10655000B8F1000FF0D0A4F2EE2240F2DC539A42E0
:1065600003D8A0F2EE229A420AD9114940F6CA0392
:1065700040F2EE22284602B0BDE8F041FEF72CBB07
:106580000C4B0D4A03EB86030021A3F8904AA3F8B5
:10659000920ACDE9004033460846FCF701FDB4E716
:1065A000064903233A46E5E79CBC0020ABAD07084B
:1065B00029B107080CB2002018B107088BAD0708F5
:1065C0002DE9F04F89468FB0174600211A4606463E
:1065D000FEF754F9DFF878A0054600240DF1240BEE
:1065E00059F824300293594602A84DF0AFFE67B324
:1065F00057F82430029A0393934218BF01212A4688
:1066000008BF002130460CBF4FF001084FF00008D2
:10661000FEF734F904A9054603A84DF097FE04A936
:1066200000912346524641463046FCF703FD23467F
:10663000CDF800B05246414630460134FCF7B0FC7C
:10664000402CCDD10FB0BDE8F08FB846EFE700BFCA
:1066500037B10708F0B5074689B00846FEF7C8FA13
:106660000E46054638B1002319491A46012009B0E3
:10667000BDE8F040A4E70846FBF71CF93F280446B4
:106680001DD83046FAF7C8F90146204640F08AFF87
:1066900078B10F4803AE314600EB84004DF056FE52
:1066A0000C4A0096234629462846FCF779FC09B097
:1066B000F0BD384609B0BDE8F040FEF783B90649A1
:1066C0003F232A46384609B0BDE8F040FEF784BAB9
:1066D000ACBC002037B10708AFB007082DE9F04F78
:1066E000924685B00C461A4600218146FEF7C6F850
:1066F000DFF874B0804655460026BAF1000F31D05D
:1067000029460422204656F032F90028424614BF9A
:106710000121002148460CBF01270027FEF7AEF8F3
:10672000EB780293AB7801932B8800938046334635
:106730005A4639464846FCF77DFCE3780293A37835
:10674000019334F8043B00935A4633463946484691
:106750000136FCF725FC102E05F10405CDD105B05E
:10676000BDE8F08F5746E8E741B10708F0B50746A6
:1067700085B00846FEF73CFA0E46054638B10023C0
:106780001C491A46012005B0BDE8F040A6E70846BE
:10679000FBF790F80F28044623DC3046FAF73CF963
:1067A0000146204640F07EFEA8B1134B04F14002A2
:1067B00003EB8203294693F8A32A029293F8A22AB4
:1067C0000192B3F8A03A00930C4A23462846FCF7FE
:1067D000E7FB05B0F0BD384605B0BDE8F040FEF778
:1067E000F1B807490F232A46384605B0BDE8F04006
:1067F000FEF7F2B9ACBD00200CB2002041B1070891
:10680000AFB007082DE9F04F87B0144603911A4640
:1068100000210546FEF732F8DFF838B106464FF0A2
:106820000008062303FB08F707F5A0774FF00009DF
:10683000039BDB5D0493002C00F08880E35D049AE9
:1068400005939A4218BF0121324608BF002128460D
:106850000CBF4FF0010A4FF0000AFEF70FF8059B3E
:106860000646CDE900935A46434651462846FCF772
:10687000E1FB049B5A46CDE9009351464346284626
:1068800009F10109FCF78CFBB9F1060F07F10107CB
:10689000CED108F10108B8F1060FC2D1DFF8B4B0CB
:1068A0004FF4B277039BA7F5B27913F807A0002C39
:1068B0004ED0E35D04939A45324614BF0121002176
:1068C00028460CBF4FF001084FF00008FDF7D6FF37
:1068D000049B0646CDE900935A46062341462846C6
:1068E000FCF7A8FB0623CDE9009A1A4A4146284640
:1068F000FCF756FB013740F26F139F42D2D1039B46
:1069000093F86F71B4B194F86F814745324614BF64
:106910000121002128460CBF01240024FDF7AEFF11
:10692000002300930B4ACDF8048007232146284614
:10693000FCF780FB00230093064A019707232146BA
:106940002846FCF72DFB07B0BDE8F08FA24690E784
:10695000A046C7E753B10708F0B5054687B008461B
:10696000FEF746F90B46044638B100231C491A4687
:10697000012007B0BDE8F04044E71A49194F02AAC8
:10698000184655F0F1FF03AEB8B1032C04D12846E8
:10699000FDF724FA07B0F0BDFAF78CFF02AA46F81B
:1069A000040B39460020013455F0DEFFECE70E48B9
:1069B00032462146FCF70CFCECE7032CE7D1DDE97D
:1069C0000346059B01931A463146E0B240F0AEFD06
:1069D000019B0028EBD12846FDF7F4FFDAE700BF62
:1069E000ACBC0020D8B1070853B107082DE9F04F1F
:1069F0000F4689B0164600211A460546FDF73EFFB0
:106A0000DFF83CB10790B84634464FF00009002E3D
:106A10007ED021460C22404655F0A9FF0028079A57
:106A200014BF0121002128460CBF4FF0010A4FF08E
:106A3000000AFDF723FF94F90B20049294F90A2031
:106A40000392B4F908200292B4F906200192B4F935
:106A50000420079000924B465A4651462846FCF7C0
:106A6000E9FA98F90B20049298F90A200392B8F9F0
:106A700008200292B8F906200192B8F90420009289
:106A80004B465A465146284609F10109FCF788FA57
:106A9000B9F1080F08F10C0804F10C04B7D1DFF8C4
:106AA000A49000240C2303FB04FA9EB34FF00008CB
:106AB000012303FA08FB56F80A2057F80A3053401E
:106AC0003BEA030314BF0121002112EA0B0F08D097
:106AD000CDF8008023464A4628460791FCF7AAFADB
:106AE000079957F80A301BEA030F06D0CDF800804B
:106AF00023464A462846FCF753FA08F10108B8F144
:106B00000E0FD5D10134082CCCD109B0BDE8F08FDF
:106B1000B246A6E7B04657F80A20012303FA08F365
:106B2000134207D0CDF8008023464A46012128466B
:106B3000FCF736FA08F10108B8F10E0FEBD1E1E7E6
:106B400067B107087FB10708F0B506468BB0084665
:106B5000FEF74EF80D46044620B300233F491A467F
:106B600001200BB0BDE8F04040E72D2B03D0A3F18E
:106B70003002092A4BD8052C05DD30460BB0BDE8A4
:106B8000F040FDF72BB92846FAF794FE0AAB621CD9
:106B900003EB440424F80C0C15F8013F303B092B9F
:106BA000FAD914462B78002BDFD1062CE5D1BDF89D
:106BB0001C20BDF91C30072ADFD8BDF91E10A1F535
:106BC000FA7292B2B2F5FA6F1AD8BDF92040A4F564
:106BD000FA7292B2B2F5FA6F12D8BDF92270B942C8
:106BE0000EDCBC420CDBA1420ADCBDF924C00CF176
:106BF000640292B2C82A03D8BDF92650112D11DDC6
:106C0000174930460BB0BDE8F040FDF7D0B8202B57
:106C100002D101352246C4E730460BB0BDE8F04052
:106C2000FDF7D0BE0F4A0C2000FB03226DB2A2F884
:106C3000141CA2F8164CA2F8187C82F81ACC82F820
:106C40001B5C00910021CDE903C5CDE90147064A4F
:106C50000846FCF7A5F90BB0F0BD00BF1CBE002034
:106C600094B107080CB2002067B107082DE9F04F76
:106C700089468DB0164600211A460746FDF7FEFDEF
:106C8000DFF8DCA005460024C4EBC40309EB0302D3
:106C900059F8030091889279089040F30748ADF8BD
:106CA00024108DF82620B8F1000F54D0002E55D0B6
:106CB000F218F058918893790A90ADF82C100722B9
:106CC0000AA908A88DF82E3055F051FE00282A4652
:106CD00014BF0121002138460CBF4FF0010B4FF0CB
:106CE000000BFDF7CBFD9DF82E3006939DF92D305E
:106CF00005939DF92C3004939DF82B3003939DF957
:106D00002A3002939DF8293001939DF82830009392
:106D100005462346524659463846FCF78BF99DF8FE
:106D2000263006939DF9253005939DF92430049370
:106D30009DF82330CDE902839DF8213001939DF821
:106D40002030009352462346594638460134FCF71A
:106D500027F9102C98D10DB0BDE8F08FB346DEE7CF
:106D6000AAB107082DE9F04F9D4FDFF8A882DFF8A0
:106D7000A8928DB006460D46284653F0C7F9034643
:106D800030B99849024601200DB0BDE8F04F6DE7DB
:106D9000052239462846FAF79BFC0446C8B9924DAD
:106DA0000146702205F5476055F00BFEC5F8104C02
:106DB000C5F81C4CC5F8284CC5F8344CC5F8404CF7
:106DC000C5F84C4CC5F8584CC5F8644C0DB0BDE83E
:106DD000F08F042241462846FAF77AFC044638BB75
:106DE0002846F9F719FE82460028EFD053F08EF9B5
:106DF000DFF828B202465BF8041B39B97B492A4602
:106E000030460DB0BDE8F04FFCF7D1BF5046CDE99C
:106E10000012FAF75DFC019A40B920462AF022FBE5
:106E20000099734D4846FCF7D3F9A5E70134E2E732
:106E3000704907222846FAF74BFC074600287AD10A
:106E40002021284655F0D4FD044670BB6A486B4D9E
:106E5000FCF708F9214628460134FCF703F90E2C0B
:106E6000F8D1FCF799F8DFF8B891654FDFF8B481F5
:106E7000002421464846FCF7F5F80C26DFF8A8A1C7
:106E800066430025F2595F480123AB40134214BF0B
:106E9000414651460135FCF7E5F80E2DF2D101349B
:106EA000FCF77AF8082CE4D190E75749564D03AA2D
:106EB00055F05AFD04AC002848D0022F11D1049A95
:106EC000072A07D805990D2904D80378722B13D007
:106ED0006E2B22D04D49082300223046FDF77CFE60
:106EE00074E7FAF7E7FC03AA44F8040B29460020EC
:106EF000013755F039FDDEE73B4B0C2000FB023338
:106F0000012000FA01F1D3F8100C0843C3F8100C6B
:106F100038493046FFF726FF58E7334B0C2000FB7B
:106F20000233012202FA01F1D3F8102C22EA010205
:106F3000C3F8102CECE728463349334F03AA55F029
:106F400013FD04AD0024A8B1082C03D13046FCF792
:106F500045FF3BE7FAF7AEFC03AA45F8040B3946B8
:106F60000020013455F000FDEDE729493046FCF7DB
:106F70001EFF2BE7082CE9D1049B0F2BF5D8DDF879
:106F800014E0BEF1070FF0D8DDF818C0BCF10D0F0A
:106F9000EBD8079F07F16402C82AE6D8089DFF2DA9
:106FA000E3D809986428E0D80A996429DDD8884292
:106FB000DBDA0B9C032CD8D8C3EBC3020A4B134477
:106FC00083F8751C83F870EC094983F871CC83F859
:106FD000727C83F8735C83F8740C83F8764C98E7C2
:106FE000ABAD07087CBE00200CB200205EAA0708EB
:106FF00049AE0708C7B1070851B70708CFB107085E
:107000001CBE0020D4B10708D8B10708DAB10708C0
:1070100094B1070809B107080EB1070838F106084E
:1070200028ED070892B10708E6B907082DE9F04FE7
:1070300089B00C46079200211A460746FDF71EFC50
:107040000026079DDFF8A0B00690B2464FF0190960
:107050004FF46178079B43B329460622204655F03A
:1070600086FC0028069A14BF0121002138460CBF77
:107070004FF0010A4FF0000AFDF700FC6A79069014
:1070800019FB028205922A7919FB02820492EA789E
:107090000392AA7802926A7801922A780092334683
:1070A0005A4651463846FBF7C5FF627919FB028202
:1070B0000592227919FB02820492E2780392A27867
:1070C00002926278019214F8062B009233465A46D7
:1070D000514638460136FBF763FF0A2E05F10605D7
:1070E000B8D109B0BDE8F08FE0B107082DE9F04F45
:1070F00080468BB00846FDF77BFD8946074638B1D0
:10710000002355491A4601200BB0BDE8F04F8DE72A
:10711000524C084694F81E3894F834B794F835A7C2
:107120000793FAF7C7FB0928054600F38B8006266C
:10713000464309F101008DF82770F9F76DFC074609
:1071400058B1FAF7B7FB0D2807D8A31983F8480BF5
:107150009DF8273001338DF827303846F9F75CFC6D
:10716000074668B1FAF7A6FB834509D3062303FB5C
:10717000054383F8490B9DF8273001338DF82730FC
:107180003846F9F749FC074668B1FAF793FB5045D2
:1071900009D8062303FB054383F84A0B9DF82730E3
:1071A00001338DF827303846F9F736FC074670B1C1
:1071B000FAF780FB079B834209D3062303FB0543B1
:1071C00083F84B0B9DF8273001338DF82730DFF81B
:1071D0008890311D0DF1270249443846FAF76EFBBD
:1071E0009DF82730062B0BD009EB0602002349F847
:1071F000063040469380FCF7F1FD0BB0BDE8F08F00
:1072000003FB05444FF4617194F84D2B192313FBD4
:107210000212059294F84C2B13FB0213049394F87A
:107220004B3B039394F84A3B029394F8493B0193F8
:1072300094F8483B00930021094A2B460846FBF787
:10724000AFFEDAE7074909233A4640460BB0BDE8EE
:10725000F04FFDF7C1BC00BF5CAC002014A10020C2
:10726000E0B10708AFB007082DE9F04F0F4689B02D
:10727000144600211A460646FDF700FB0546002C81
:1072800000F0DB8022783B789A4218BF0121024649
:1072900008BF002130460CBF4FF001084FF0000836
:1072A000FDF7ECFA23789B4A054641463046FBF74A
:1072B000C1FE3B78974A41463046FBF771FE002CF1
:1072C00000F0BD8062787B789A4218BF01212A467F
:1072D00008BF002130460CBF4FF001084FF00008F6
:1072E000FDF7CCFA63788C4A054641463046FBF7F9
:1072F000A1FE7B78884A41463046FBF751FE07F1F4
:10730000CA030493822304F1CA0B05934FF00209C8
:107310004FF0000A3B78534500F39380002C00F0B7
:10732000F38097F8EA3094F8EA209A4218BF0121D6
:107330002A4608BF002130460CBF4FF001084FF02D
:107340000008FDF79BFA94F8EA30744A0546414676
:107350003046FBF76FFE97F8EA30704A41463046F8
:10736000FBF71EFE07F1EC09002C00F0CF8004F1C2
:10737000EC034A4604F1FC014FF001089A4633F849
:1073800002CB32F8020B844518BF4FF000088B4245
:10739000F5D188F001012A46C9B23046FDF76EFAF0
:1073A000082105465046FAF7E5F85D4A034641468E
:1073B0003046FBF73FFE97F8EA104846FAF7DAF84E
:1073C000574A034641463046FBF7EAFD002C00F0E1
:1073D0009F804FF0FC094FF0010807EB090104EB17
:1073E0000900FAF751F909F10409002818BF4FF014
:1073F0000008B9F58E7FF0D188F001012A46C9B2A4
:107400003046FDF73BFA082104F1FC00F9F736FBA2
:10741000444A034641463046FBF70CFE97F8EA1013
:1074200007F1FC00F9F72AFB3E4A03464146304685
:1074300009B0BDE8F04FFBF7B3BDA04639E7A04661
:1074400057E7059B3B440693002C5BD0059B0698B1
:10745000234419460793FAF717F9049B1A789BF807
:1074600000309A4206BFB0FA80F84FEA58184FF041
:1074700000084B4609F11002F85AE15A02338842DB
:1074800018BF4FF000089342F6D188F001012A4658
:10749000C9B23046FDF7F2F9627804EB09010546FE
:1074A0009BF81800FAF738F802909BF80030019327
:1074B000079B00931C4A0AF1010341463046FBF743
:1074C000B9FD049B7A78187E079307EB0901FAF758
:1074D00023F8079B049A02901B7801930132069BC4
:1074E00004920AF1010A00930F4A5346414630467E
:1074F000FBF756FD059B09330BF1010B09F1100950
:10750000059307E7A046DCE7A04624E7A04652E73C
:10751000A04683E7F9B107080BB2070839B207089C
:1075200051B2070868B2070820B207082DE9F04FEA
:107530008FB0044602AA0846AF4955F015FA064630
:1075400040B903460246AD494120FFF78DFE0FB01A
:10755000BDE8F08FAA49FAF797F8074620BBA6497D
:1075600002AA55F001FAFAF7A5F90828054606D946
:10757000A44908233A462046FDF72EFBE7E7A24C34
:1075800094F83437834202DC84F83457DFE7064648
:1075900004F234773146384639F028FA94F8343713
:1075A0000136B342F6DCEFE798493046FAF76CF85B
:1075B0000546E0B9904902AA55F0D6F9FAF77AF9EA
:1075C0000828064603D9924908232A46D3E78E4C59
:1075D00094F83537834202DC84F83567B7E72846EC
:1075E000314601354CF08AFE082DF8D1F4E789497F
:1075F0003046FAF749F8074600BB7F4902AA55F022
:10760000B3F90028A3D0FAF755F90828054603D99D
:10761000814908233A46AEE77B4C94F81E388342F2
:1076200009DD014604F2347039F02AFA294604F2E1
:10763000347039F033FA84F81E5888E777493046B9
:10764000FAF722F8054618BB6F4BDFF8AC9193F8B8
:107650001E7806AE01461022304655F0B2F9B0460B
:10766000BD4202AA80F20E814946002055F07CF905
:1076700010B96B493A460EE1FAF71CF9013528F8C2
:10768000020BEDE796E80F00664C84E80F005EE71A
:1076900065493046F9F7F8FF054600283BD15A4BBB
:1076A0000DF1180893F81E98464607464F45524973
:1076B00002AA4FF0000080F2F28055F055F9014621
:1076C00010B95A494A46E6E00322304655F0CAF955
:1076D000B2464FF0000B304652F018FD584502D824
:1076E00001370436E2E79AF80000F9F7C7FF0BF11B
:1076F000010B0AF8010BEEE74D494A46CBE0414643
:107700002046032239F05AF90135043408F10408FF
:10771000AF42F4D11BE747493046F9F7B5FF0546BC
:10772000002840F0AC80384F334997F8348702AADC
:1077300055F01AF900283FF40AAFFAF7BBF8461ED5
:1077400001D4B04503DC3C494346012213E72A49F2
:1077500002AA002055F008F9014600283FF4F7AED0
:107760004FF00008082203A8CDE903888DF81480A3
:1077700055F078F90DF10C0903A852F0C7FC40450B
:107780001CD81D4902AA002055F0EEF800283FF44D
:10779000DEAE90F800A097F83597DFF8ACB04FF068
:1077A00000084D45144902AA4FF000007EDA55F05A
:1077B000DBF8024658B921494A466CE099F80000C6
:1077C000F9F75CFF08F1010809F8010BD4E7002D77
:1077D00040D11378303B092B3CD919490192F9F774
:1077E00053FF019A90B310465946F9F74DFF019A9D
:1077F000002838D013494EE0D8B1070848A8002027
:107800007FB2070885B2070814A1002090B20708CC
:1078100099B20708A7B20708B3B20708C5B20708AC
:10782000B4B3070834A90020EFB20708D4B307089F
:10783000FBB2070819B307081EB30708F4B307081B
:10784000E2A1070831B307082AB307084FF001087F
:107850004FF0FF3510460192FAF72CF80028019AF4
:1078600003DA214917E0A846F2E70EAB03EB450324
:10787000013523F8200C94E71C494A460BE01C49CB
:10788000324608E01B49002055F06EF800283FF40E
:10789000F9AE19493A462046FCF789FA57E655F001
:1078A00063F800287FF428AF144C31E755F05CF8FA
:1078B0000028E1D1124C06EBC6008230082203A951
:1078C000204439F07BF85046F9F7D8FE37446A0077
:1078D00087F8FE0704EB061006A9023055F00EF8F3
:1078E00087F8168833E600BF66B307087BB307083E
:1078F0009EB30708D8B10708D1B2070844A90020F1
:1079000048A800202DE9F04F89B00F46914600218C
:10791000139A98460646FCF7B1FF87EA09096FEA11
:107920000903DFF8849006930446002528460AF0F0
:10793000D7F8129B184230D0069BDFF870B0034096
:1079400014BF4FF0010A4FF0000A049310EA070336
:1079500014BF4A465A462846059307920AF0D2F8C1
:10796000079A03900090434651463046FBF762FB6E
:10797000049BB3FA83F1224649093046FCF77EFFA7
:10798000059A039B009304464346002A14BF5A46B7
:107990004A4651463046FBF703FB0135182DC5D149
:1079A00009B0BDE8F08F00BF03B1070819B407089C
:1079B00037B504460846019152F0A8FB01990546E7
:1079C00002462046F9F784FE70B9625D1046F9F769
:1079D00045FE00B932B901352C4420460134037804
:1079E000202BFAD003B030BD0020FBE7F0B503290F
:1079F00085B005460C46164614D80B4F3970FBF778
:107A0000CBFA0A492846FDF757FD0949224601A845
:107A1000F9F726FD01AB324608212846FCF75CFF4A
:107A2000FF233B7005B0F0BD7805002049AE070884
:107A3000FFAF0708F0B5032985B005460C4616468A
:107A400014D80B4F7970FBF7A7FA0A492846FDF7BF
:107A500063FD094922466846F9F702FD6B46324646
:107A600010212846FCF738FFFF237B7005B0F0BDDE
:107A70007805002049AE0708FBAF070830B587B08E
:107A8000104B0493104B0293104B114D0193114B6B
:107A90001149124A00930446114B12480395FBF713
:107AA000E1FAFBF779FA10482946FBF791FB3CB164
:107AB0000E4A0F490F4807B0BDE83040FBF788BBBE
:107AC00007B030BD60B407086FB4070878B4070882
:107AD00065B4070884B407082AB4070820B4070867
:107AE00023A1002035B407088AB40708445E0708BC
:107AF0003C5E07089BB407080120BFE7214BB0F5A7
:107B0000FA6F1A680346A8BF4FF4FA63B3F57A7F99
:107B1000B8BF4FF47A73D2041FD540F2DC529042C2
:107B20001ED007EE903A40F2DB529042F8EE677AB0
:107B300097BFDFED156ADFED156A9FED157A9FEDB2
:107B4000150A85BF9FED147A9FED140A77EEE67A49
:107B500077EEE67AA7EE870A7047B0F57A7F02D80B
:107B60009FED0F0A704707EE903ADFED0E6A9FED2A
:107B70000E7A9FED0E0AF8EE677A77EEE67AA7EEB8
:107B8000870A7047B4A6002000007A4400A0BB44D6
:107B9000D62000C000E08244D6200040000083448C
:107BA0000000000000407A4466100040000040429F
:107BB00010B584464FEA810E102312F4004F14BF13
:107BC0000E2407245200013BCCF8004092B2F4444A
:107BD000F3D100EB81128C01035142F821301220C5
:107BE00010BD00BF10B584464FEA810E0424130B6C
:107BF00003EB430318331201013CCCF8003092B27E
:107C0000F444F4D100EB01130A01845043F82140FD
:107C1000062010BD704700BF704700BF034B00EB4C
:107C2000400003EBC000407C704700BF48050010D7
:107C30002DE9FF471E46C368BDF83070DDF834807B
:107C400004468946924643B3CBB20D2B9ABF1A4ADB
:107C5000D5560025BAF1FF3F21D02368174A314697
:107C6000CDE9005A3846C047524620795FFA89F17B
:107C7000F2F7AAFE024600B10288D3B20393C2F320
:107C80000323120BCDE9005202930D4A23683146BB
:107C90003846C04704B0BDE8F0874D1CDAE77B06E4
:107CA000F8D42368074A0C9531463846C44604B0D8
:107CB000BDE8F047604700BF285E0708C8B4070862
:107CC000D5B40708F9B407080023472202704370AF
:107CD0008370C370704700BF704700BF00207047BB
:107CE000704700BF0020704701207047704700BFF9
:107CF000704700BF704700BF704700BF9FED010A8B
:107D0000704700BF000000000020704703681B6937
:107D1000184730B5084B002293F900405D780119EF
:107D20000132CD729D780555062ADC788C7503F1F9
:107D30000403F1D130BD00BF542007080023837035
:107D40000370C37043707047C36B33B15B68426D9F
:107D50009BB29A4205D3D01A7047D0E907239A42C2
:107D6000F9D2C0681044C01A704700BFD0E90912A8
:107D70000369914238BFC9188A1A016C39B1496840
:107D8000013B12FA81F2934204D9981A7047013BE1
:107D9000981A704700207047036C13B190F8640084
:107DA0007047D0E90903181AB0FA80F0400970470B
:107DB000C26B10B4034662B1426DC1685C69881A37
:107DC000013A205C5DF8044B08BF0A46C0B25A6510
:107DD0007047006A5C69411C205CDC68A14238BFC6
:107DE0000A46C0B25DF8044B1A627047836E70B5E4
:107DF00004460D460BB19847B8B1636AA269D554E1
:107E0000636A2169226C01338B4228BF00236362BD
:107E100032B3EFF31183502282F31288226C11687F
:107E2000C90703D5DBB283F3118870BD516889B2ED
:107E300071B9D4E90950854218D0A6690644D660C4
:107E400018D9281A80B25060A562002184F8641005
:107E5000116841F00101DBB2116083F3118870BD3C
:107E6000226ED36843F08003D36070BD012284F892
:107E70006420D7E72569281A80B25060A162E4E740
:107E8000836E03B118477047F8B590F87C30012B2A
:107E90001CD0002A164619DD0269436A05460F46C2
:107EA000D41AB442A869A8BF3446394618442246B9
:107EB00054F024FD6B6A2A692344361BB3FBF2F0AD
:107EC000002E02FB10336B622744E9DCF8BD00BFD3
:107ED00090F87C30012B0DD0036C43B3EFF311838A
:107EE000502282F31288026C1168C90703D5DBB2F5
:107EF00083F311887047516889B270B471B9D0E9C1
:107F00000954A54219D086692644D6601CD92C1B79
:107F1000A4B254608562002180F86410116841F0B9
:107F20000101DBB2116083F3118870BC7047026EEF
:107F3000D36843F08003D3607047012280F8642047
:107F4000DBB283F31188F0E705692C1BA4B25460FF
:107F50008162E0E70849002301E0152B09D003EB1B
:107F60004302013311F802C084450A44F5D110469A
:107F700070470020704700BF4425002010B311B3A4
:107F800010B5124C4FF0100C22464FF0010E00239A
:107F900004E001334E2B0ED092F804C0604502F18C
:107FA0001C02F6D1714508D001330EF1010E4E2BA3
:107FB0005FFA8EFEF0D1002010BDC3EBC30304EBCB
:107FC000830010BD70470846704700BFF4D2060812
:107FD0002DE9F04188B01E4603090E9F90464033BC
:107FE00000F00F0451B30793FFF7C8FFC279079B56
:107FF000CDE900420546164A41463046B847D0B161
:108000002868F2F705FFA9796A79DFF854C0ED799D
:10801000079B009411F0020F4FEA92020D4902F102
:10802000010208BF6146CDE90102CDE903150A4A04
:1080300000213046B84708B0BDE8F081074A0E94E9
:1080400041463046BC4608B0BDE8F041604700BF3D
:1080500008B5070891A307081AB507083CB5070833
:1080600049AE07082DE9F047DFF85CA0BAF8003008
:10807000043388469EB201F10909012518F8014B25
:10808000B4460021ACF1040305FA01F29BB2224090
:10809000C2B1878900EB830E01339BB29C45CEF8B9
:1080A0001470F5D101310CF1040C08291FFA8CFC75
:1080B000E8D12036C845B6B2E0D10023AAF8003096
:1080C000BDE8F0871746E5E794F100202DE9F04F71
:1080D000DFF89490B9F802300B330F4601F106082F
:1080E0001FFA83FB0125002117F801EB5A464FF0D8
:1080F000000C0126A2F10B039BB206E001339BB2F8
:108100008489CAF8144093420BD000EB830A002EF6
:10811000F4D100EB830A01339BB29342CAF8146096
:10812000F3D1043300EB8303BCF1090F596010D085
:10813000BCF1080F0BD005FA0CF313EA0E0F14BFB5
:10814000012600260C320CF1010C92B2D2E7002677
:10815000F8E70BF1780447451FFA84FBC4D1A9F86E
:108160000210BDE8F08F00BF94F100202DE9F0412E
:10817000057B0E780446C0E90555C0E90755C0E9FE
:108180000955C0E90B55C0E90D55F64328220021D9
:108190003C3054F016FCF6B24FF0140C4FF0050EC4
:1081A0004FF0000846FA0EF303F00103002B14BF52
:1081B00019270A2743441EF001000CEB07015FFA60
:1081C00083F818BF284689B2634604EB8302013363
:1081D0009BB299425061F8D10EF1FF3EBC44BEF112
:1081E000FF3F1FFA8CFCDDD118F0010F14BF1920DE
:1081F0000A200CEB000189B2634604EB83020133D1
:108200009BB28B425561F8D10CEB00039BB21A1D57
:108210000549013304EB82029BB2002050608B8041
:108220002361BDE8F08100BF94F1002070B5094CD6
:10823000A36873B10546002606E099681A681E73A4
:10824000A1609047A36823B15A68AA1A002A184669
:10825000F3DA70BD94F100202DE9F04F0A4687B0A3
:1082600000210646FCF70AFB3B4C05903B4A23786D
:10827000608802EB8303D3F890A1F8F737FC83689A
:108280000493374BC1681A78002A4BD0DDF8108070
:108290000491002721796279049B07FB012213F8DE
:1082A0000290B8F1000F3FD018F80250059A4D45E2
:1082B00014BF0121002130460CBF4FF0010B4FF0DD
:1082C000000BFCF7DBFA013705907DB305F00F02D8
:1082D0002D0940350292CDE90075224A5346594690
:1082E0003046FAF7A7FEB9F1000F2AD009F00F02C5
:1082F0004FEA1919029209F14002CDE90072534682
:10830000184A59463046FAF74BFEA279012A38BF7F
:108310000122BA42BEDC144B0834A342A6D107B0F6
:10832000BDE8F08F9046B4E74546BFE7B8F1000FCF
:10833000D9D00E4A0097534659463046FAF77AFE8E
:10834000D1E77306E1D4094A0097534659463046AF
:10835000FAF726FED9E700BF6C200708542007086B
:1083600098A100204EB50708E421070864B5070866
:1083700038B50B4B03EBC0050C462A7E094803EBCE
:108380008203D3F89011FAF76DFEAB7F33B1611C15
:108390000548BDE83840C9B2FAF764BE38BD00BF31
:1083A0005420070850B7070827ED07080246531C5A
:1083B000084605D1044B1A681B790A600B71704797
:1083C0000249F9F74DB800BF03B5070828ED0708C3
:1083D00010B501311446FFF7D1FD28B9064B1A68D4
:1083E0001B792260237110BDC27904492046BDE883
:1083F0001040F9F735B800BF03B5070815B50708F1
:108400002DE9F041154686B06A1C8846BDF83060FB
:108410000D9F194623D0030900F00F044033CDE926
:108420000045164A05933046B847A8B198F805109C
:10843000D8F800002A46F2F70FFB68B102880178ED
:108440000391C2F30321120BCDE900420291059B77
:108450000B4A00213046B84706B0BDE8F0817306EC
:10846000FAD40309074A00F00F000C90403330465D
:10847000BC4606B0BDE8F041604700BF78B50708CC
:108480008AB50708B3B507082DE9F04F2DED028B2B
:108490000A468BB000218246FCF7F0F96D4D81460B
:1084A00005F1800B00266C4B1C78AB7AB34200F3CD
:1084B00093801035AB45F5D140F21620F8F716FB46
:1084C000D0E902530CB12C461D460DF1100B1522BC
:1084D0000021584654F075FA00272E78002E42D01D
:1084E00069783046FFF74AFD95F9023002935A1C2D
:1084F000534208EE100A5341002C00F0A8800022DD
:1085000014F802C0B44504EB020040F09C8090F9DE
:108510000280029A424540F0948042788A4208BF25
:10852000012301220BF8072003F001034A4683F0E0
:10853000010150460393FCF7A1F9039B81464CB11E
:10854000464A18EE101ACDE900A230464246FFF71F
:1085500057FF039B424A18EE101ACDE900A230469D
:10856000029AFFF74DFF0137152F05F10305B4D12E
:108570006CB33A4FDFF8E88004F13F061BF8013B8B
:1085800002930BBB2078F8B194F9022001321BD082
:108590006178FFF7F3FC4A46054601215046FCF797
:1085A0006DF994F90220029B294681462078CDE995
:1085B00000A7FFF725FF2078029BCDE900A84FF028
:1085C000FF322946FFF71CFF0334B442D6D10BB06B
:1085D000BDEC028BBDE8F08FE888F8F787FAD0E9A8
:1085E00002230CB114461A46297A6B7A06FB013332
:1085F00012F9038014B3E756B8450CBF01230023DA
:108600004A4614BF0121002150460293FCF736F977
:10861000029B814644B1114A3146CDE900A2284669
:108620003A46FFF705FB029B0D4A3146CDE900A211
:1086300028464246FFF7FCFA013634E74FF0FF3791
:10864000DAE700236DE703323F2A7FF459AF4FF09A
:10865000FF386BE7DC05002098A1002035300108C9
:10866000A12F01082DE9F04F8BB0074640F21620EC
:108670000391F8F73BFA039A044600213846FCF7C9
:10868000FDF8404AD4E90253147806460CB12C4652
:108690001D461522002104A854F093F905F13F036B
:1086A000039395F80090B9F1000F31D095F801A02F
:1086B000002C65D0224600231178494558D1283333
:1086C0006B4492F80180012203F8182CD045324601
:1086D00014BF0121002138460CBF4FF0010B4FF0B1
:1086E000000BFCF7CBF8064654B1B8F1000F07D0E9
:1086F000254B00935A463B4641464846FFF768FCE7
:10870000224B00935A463B4651464846FFF760FCD1
:10871000039B03359D42C4D13CB3DFF86C90DFF876
:108720006CA0651C0DF11008403418F8013BCBB962
:1087300015F8013CB3B116B13046FAF74BFC297875
:1087400015F8010CCDF800903B460022FFF740FCE5
:10875000002215F8010CCDF800A03B461146FFF7AA
:1087600037FC00260335A542DFD10BB0BDE8F08F02
:108770000133152B02F103029ED14FF00008A5E74B
:10878000A046A3E798A1002035300108A12F0108D9
:1087900008B5254B1B68DB040AD5B5EE400AF1EE9F
:1087A00010FA12D19FED210A53F030FB80B208BDC0
:1087B000DFED1F7AB4EEE70AF1EE10FA28DA9FED4A
:1087C0001D0A53F023FB80B208BDDFED197AB4EE29
:1087D000E70AF1EE10FAE5D49FED177AB4EEC70A76
:1087E000F1EE10FA8BBFDFED157A9FED157A9FED54
:1087F000157A70EE677A8ABF70EE677A9FED120A7B
:108800009FED120AA7EE870A53F000FB80B208BD65
:1088100070EE677A9FED0E7A9FED0E0AA7EE870A3B
:1088200053F0F4FA80B208BDB4A600200080BB4427
:108830000000404200007A4400E08244000083448B
:1088400066BEFFBE66BEFF3E0060BB4400A0BB44E8
:1088500038DFFF3E00407A442DE9F04F6D4B1B7826
:1088600087B0002B00F0D0806B4D6C48A968DFF812
:10887000F0A1FAF7ADFC69686948FAF7A9FC694B01
:108880006948D3E90031C91A684BDA68B1FBF2F2E2
:10889000FAF79EFCFAF780FB6548FAF795FB654806
:1088A000FAF792FB4FF00008634B1B785FFA88F4ED
:1088B000A34222D8614C624FFAF76EFB2646002590
:1088C00056F8041B38460135FAF7CCFB162DF7D1C4
:1088D000FAF762FB5A4E0125234661681B68304651
:1088E000C91A0135FAF7BEFB162D04F10404F3D1C1
:1088F00007B0BDE8F04FFAF74FBB524B142603EB1D
:10890000840306FB045693ED000AB6F80E9053F06C
:108910007DFA96F81EE01EF0010F14BF52222D22A0
:108920001EF0020F14BF54232D231EF0040F07EE78
:10893000903A14BF56232D231EF0080F14BF4FF09A
:10894000430C4FF02D0C81B21EF0800F4FF03C0B0A
:10895000B1FBFBF105914FF0640114BF4FF0530ED2
:108960004FF02D0E80B201FB09F1671CCDE902E149
:108970000093049017EE903ACDF804C03946504663
:10898000FAF770FBB37FDB073AD55C232E4A6343CB
:10899000D118D05891ED010A70B1DFED2C7AB8EE04
:1089A000400A20EE270A07EE900AF8EE677A80EE7A
:1089B000270A53F02BFA00B2642290FBF2F102FB7B
:1089C00011022348FAF74EFB142101FB075701FB64
:1089D0000454F988628A0491218B0391E18A0291FF
:1089E000A18B0191A18A009102F0030319214B434D
:1089F0001848218A9208FAF7EBFB08F1010853E7BF
:108A00001548FAF7A9FADFE7144807B0BDE8F04FB8
:108A1000FAF7DABA0400001020090010C7B50708F9
:108A2000D7B5070834060010EEB5070894F100200A
:108A30001BB6070877B6070850100010CC090010C5
:108A400027B70708241600104006001000401C46F7
:108A5000F0B6070805B70708FCB607082BB70708E4
:108A6000D3B607082DE9F84F1F4DDFF88490DFF8E3
:108A700084A006460C463B274FF000082046FCF732
:108A8000B7F8D5F800B048B921465846F8F744FE83
:108A900020B968682146F8F73FFE80B15846FAF7DA
:108AA0005BFA696811B15046FAF7DCFAA96811B1AE
:108AB0004846FAF7D7FAFAF76FFA4FF00108013F84
:108AC00005F11005DAD12046FCF792F848B9B8F163
:108AD000000F06D1224630460449BDE8F84FFBF7A7
:108AE00066B9BDE8F88F00BF5423070853B70708DD
:108AF0004DB7070847B70708F1F7EABA10B50446BB
:108B000053F084F981B22046BDE81040F1F7E0BA95
:108B100070B50468236A1B69054643B1236AD0F81F
:108B200094001B69984701282AD002280DD0236A97
:108B3000DA699AB9586958B399692162BDE87040F9
:108B4000C3E90522F1F786BC2362236ADA6914338C
:108B5000002AF9D1236ADA69002AEBD0216A94F855
:108B600024200E7B1433F6B22362D2B996B928467C
:108B7000F1F7F4FB28460121BDE87040F1F7B6BBE0
:108B8000236A143B014623622846F1F7AFFBCEE788
:108B9000206270BDAB68002BE9D01A689B885383B4
:108BA000E5E700212846F1F7A1FB002384F82430F3
:108BB000002EDCD0EEE700BF8069002834D00368C7
:108BC0001A6A127B1ABBD3E904125B6849686AB15E
:108BD00010B4546800220A6022609A885DF8044B41
:108BE00022F003021204120C9A8091E71A891206ED
:108BF000FCD41A89D20708D400220A609A8822F08D
:108C000002021204120C9A8082E79A89F1E78268C4
:108C1000002AD8D0116892880A83D3E904125B68CD
:108C20004968002AD4D1E1E7704700BF806900B9E4
:108C30007047016830B4D1E904424B68646872B18E
:108C40005568002222602A609A8822F003021204EA
:108C5000120C9A800B6A1B7B9BB930BC58E71A89AF
:108C60001506FCD41A89D20713D4002222609A88F0
:108C700022F002021204120C9A800B6A1B7B002B5A
:108C8000EBD08368002BE8D01A689B88138330BC34
:108C90003EE79A89E6E700BF30B50446006E838957
:108CA000A16023F400531B041B0C838195B06379EE
:108CB000009113F0040F21794FEA03324FEA0323A6
:108CC00003F48063ADF8083001F0010302F40052B0
:108CD00014BF4FF480550025002B4FF00003ADF872
:108CE0000620ADF80C3007BF002208230C23042215
:108CF000ADF804508D07694654BFADF80A20ADF8B1
:108D00000A304AF04BF96279236ED00700F189806E
:108D100012F0080F9A8A0BBF22F0080292B21204D6
:108D200042F0080208BF120C9A829A8992B242F469
:108D300000529A812279D10732D5E06B002800F0E9
:108D400082800023E26D0793CDE90B33CDE90F3329
:108D5000CDE911334FF4807509936369E1680D958E
:108D600005920693626C04924FF480634FF4803551
:108D70000A9308910E9549F0C7FE04A9E06B49F0EB
:108D800059FFE16B236E0A6842F001020A609A8A79
:108D900092B242F040029A824968227989B26165B2
:108DA000920737D5206C002859D02369A26D08930B
:108DB000A36CCDE90432002240230025CDE906232F
:108DC0004FF480314FF480630A930E91CDE90B5537
:108DD000CDE90F55CDE9115509950D9549F094FE52
:108DE000206C04A949F026FF226C236E506940F0E4
:108DF00080005061106840F01600106055609A8A3B
:108E000092B242F0800203F10C019A820A6842F0A9
:108E100040020A609A8992B242F400529A8115B0D7
:108E200030BD1E498B4223D0A1F54C418B421DD051
:108E300001F580618B421DD102200121F1F7DBF8A1
:108E40006279236E64E74FF6DF711980D96841F0CB
:108E50002001D960D96841F01001D960A0E7DA6833
:108E600042F0800203F10C01DA60CFE70120E4E771
:108E70000020E2E701F580618B420AD001F58061B4
:108E80008B4208D001F544418B427FF441AF05206D
:108E9000D3E70320D1E70420CFE700BF0010014053
:108EA00030B50446006E21718389A26823F4005313
:108EB0001B041B0C8381637995B013F0040F00929F
:108EC00014BF4FF480520022ADF804201A031B0295
:108ED00003F48063ADF8083001F0010302F400529E
:108EE000002B4FF00003ADF80620ADF80C3007BFA3
:108EF000002208230C2304228D07694654BFADF8D5
:108F00000A20ADF80A304AF049F86279236ED0079A
:108F100000F1898012F0080F9A8A0BBF22F0080234
:108F200092B2120442F0080208BF120C9A829A8987
:108F300092B242F400529A812279D10732D5E06B85
:108F4000002800F082800023E26D0793CDE90B3307
:108F5000CDE90F33CDE911334FF48075099363697F
:108F6000E1680D9505920693626C04924FF480635C
:108F70004FF480350A9308910E9549F0C5FD04A978
:108F8000E06B49F057FEE16B236E0A6842F0010284
:108F90000A609A8A92B242F040029A824968227923
:108FA00089B26165920737D5206C002859D02369B2
:108FB000A26D0893A36CCDE9043200224023002562
:108FC000CDE906234FF480314FF480630A930E916C
:108FD000CDE90B55CDE90F55CDE9115509950D9505
:108FE00049F092FD206C04A949F024FE226C236E06
:108FF000506940F080005061106840F01600106029
:1090000055609A8A92B242F0800203F10C019A8272
:109010000A6842F040020A609A8992B242F4005211
:109020009A8115B030BD1E498B4223D0A1F54C4129
:109030008B421DD001F580618B421DD102200121A0
:10904000F0F7D9FF6279236E64E74FF6DF7119807C
:10905000D96841F02001D960D96841F01001D96088
:10906000A0E7DA6842F0800203F10C01DA60CFE792
:109070000120E4E70020E2E701F580618B420AD09D
:1090800001F580618B4208D001F544418B427FF4A9
:1090900041AF0520D3E70320D1E70420CFE700BF8D
:1090A000001001402DE9F047AD4B1B6886B03BB383
:1090B0005B69984720B3AB4DD5F8CC36002B01DD6A
:1090C000F6F762FDA84C6378022B43D0032B17D12F
:1090D00095F8E83713B1A548F6F792FD95F8D43620
:1090E00013B1A348F6F78CFD95F8183713B1A148D2
:1090F000F6F786FD95F85C3713B19F48F6F780FDCB
:109100009E4C2378012B02D006B0BDE8F0879C4B23
:109110001B68002BF8D09B4D2B6828465B6898474E
:109120000028F1D0984B994E1A68338892889A4259
:1091300023D2974B974A1B7852680021217003F085
:109140000203002AE0D0002B40F068811368928867
:109150001A83D9E7A37804F1040804F1080704F599
:10916000BD56072BCCD8DFE813F062001F01780052
:1091700059002400BA00C400210087490968002270
:109180004968EA622A6803FB01F12846D3689847D8
:10919000804A3388526801333380002AB4D0136880
:1091A000928859690A42D3D05A83ADE7032363708A
:1091B000A6E72378207D032B0CBF4FF080094FF4E6
:1091C00080794FF0010A002800F0B5800128FAD11B
:1091D000D5F840386268D5F83818580202314FF097
:1091E000FF33B3FBF0F39A184FF0000343EB030097
:1091F0009142834138BF0A4602203946F5F7C0FC48
:10920000032800F29A8101A353F820F0019101088C
:109210000B930108019101080B93010895F8A03701
:10922000002B3FF46DAF5D48F6F7EAFC68E70023DA
:1092300005A9092218460391F5F75EFB01287FF482
:109240005FAF059B93F8FE21552A00F0EA800222C9
:10925000012385F8E427637052E7514B0093032202
:10926000A27050494D483023052250F043FD47E796
:1092700023690622652BA2703BD92278032A0CBFF2
:109280006FF07F026FF0FF02A3F1650303EA0203B0
:1092900003F101030CBF80224FF480729A422361D4
:1092A00027D2E268D5F8381898180231884207D3D7
:1092B00095F8E41711B9012185F8E41701216170CF
:1092C000C4E90120C5F8C427D5F8402802FB03F300
:1092D0005B02C5F8A837C5F8AC370523A370A268B0
:1092E00041460120F5F7E8FC012840F0DD80062327
:1092F000A37000213046F5F79BFD012840F0D48093
:10930000A3780133DBB2A3702BE7D4E901C3226950
:10931000A3EB0C01914288BFC4E903C10328A7D085
:109320000133B3FBF9F209FB12320AB14B449B1A29
:10933000002063602075D5F8382841460232F5F7E1
:109340001FFC032800F2F98001A353F820F000BFAE
:10935000019101081194010801910108719201081D
:10936000385E0708F4520020F4420020DC5A002046
:10937000C85900200C5A0020505A00204C3C0020B4
:109380007022002074220020443C00204A3C00202F
:10939000C0220020C42200203C3C0020945A00201F
:1093A000218F0008E8BC0708D5F82C0805A9002380
:1093B0000922F5F7A1FA01287FF4A2AE0022059B4D
:1093C0002270B3F80B20B2F5007F1BD11A7C022A61
:1093D00018D193F8FE21552A14D193F8FF21AA2A17
:1093E00010D1B3F80EC0D5F82C686644C5F83068C3
:1093F0005F7BC5F840787A1E7F2A03D87A4237EA25
:10940000020259D00322012385F8E427637077E62E
:10941000636884F814A00133A360D4E613689288CB
:10942000C2E693F8FF21AA2A7FF411AFD3F8C62130
:1094300003994AB193F8C201A0F10B06012E2DD970
:1094400000F0F700062829D0D3F8D6214AB193F8C6
:10945000D201A0F10B06012E20D900F0F70006285A
:109460001CD0D3F8E6214AB193F8E201A0F10B0633
:10947000012E13D900F0F70006280FD0D3F8F621FB
:10948000002A3FF4E4AE93F8F231A3F10B00012877
:1094900004D903F0F703062B7FF4D9AE0123C5F8F6
:1094A0002C28A370104682E702287FF429AE0123FE
:1094B00085F8E437637023E67A02013AC5F8482854
:1094C000D88A00B9586AC5F83408B3F81120520197
:1094D00002F2FF125212C5F85028B3F8131001B966
:1094E000196A94440CEB400CA1EB0C01B1FBF7F1B1
:1094F00040F6F477B9424FEA4000C5F8381819D958
:109500004FF6F477B94211D903212170DB6AC5F80F
:109510004C38324495F810381044C5F83C080BB963
:10952000F6F762FCA3780133A370E9E50223237008
:109530000023ECE70123237064E7207D43E600BFAE
:109540002DE9F843CB4CA36820469847002800F04B
:109550008F80B4F90E30A17D06EE903AB4F9103048
:1095600007EE903AB4F9123007EE103AF8EEE66AD8
:10957000F8EEE77AB8EEC77A0123092984F8543067
:10958000C4ED126AC4ED137A84ED147A72D004F13A
:1095900048002EF025F9B84DAA8DAB6A002A40F09C
:1095A000F880B64A1268520700F1C180B3F9002072
:1095B00094ED125A94ED136A94ED147A05EE902A04
:1095C000B3F90220B3F9043006EE902A07EE903A80
:1095D000F8EEE55AF8EEE66AF8EEE77A75EE655AC7
:1095E00076EE666A77EE677A2B88C4ED125AC4ED80
:1095F000136AC4ED147ADBB395ED025A95ED056A52
:1096000095ED087AD5ED033A95ED064AD5ED094A70
:1096100075EEC55A76EEC66A77EEC77AA5EEA35AFE
:10962000A6EE846AA4EEA77AD5ED015AD5ED046AB8
:10963000D5ED077A85ED025A35EE652A76EE662A73
:1096400037EE673AE3EE825AE2EE846AE4EE837A1A
:10965000C5ED015AC4ED125A85ED056AC5ED046ADF
:10966000C4ED136A85ED087AC5ED077AC4ED147A66
:10967000BDE8F883D4ED0B5A94ED0C6A94ED0D5AC5
:10968000D4ED094A94ED084A7D4B67EEA55A27EEC2
:10969000866A67EE857A94ED0A5A1B78A6EEA46A6C
:1096A000E6EE845AE6EE857AD4ED0E6AD4ED0F4AE2
:1096B00094ED105AE6EE875AF0EE466AE4EE876AB9
:1096C000E5EE077AC4ED125AC4ED136AC4ED147ABC
:1096D000002B7FF460AF6B4B93ED055A93ED036A5B
:1096E00093ED047AD3ED014A93ED004A26EE866AA3
:1096F00026EE877A66EE856A93ED025AA5EEA47A85
:10970000E5EE856AA5EE846AD3ED064A93ED075A25
:10971000D3ED085AA7EEA46AA7EE857AE7EEA56A0C
:1097200084ED126A84ED137AC4ED146A33E7564E61
:10973000B28B322A62D0002A40F0CA8096F83A20D2
:10974000002A3FF433AF06F12C0007C84F4F4FF00B
:10975000000C87FB028E86F83AC0D217A689C2EBAE
:109760002E12921B9A8087FB0062C017C0EB22105A
:1097700087FB0127C917C1EB271118805980444B7B
:109780000122A3F80EC0C3F80A20F9F757FAAB6A12
:109790000CE7B2F5C87F7FD03B4994ED127AD1ED4A
:1097A000046AD4ED137A94ED146AF8EEE66A0026A2
:1097B00076EE876A91ED057AA664B8EEC77AFDEE7B
:1097C000E66A37EE277AD1ED067AC1ED046AF8EE43
:1097D000E77ABDEEC77A77EE867A0020FDEEE77A6B
:1097E000012A188081ED057AE6645880C1ED067A79
:1097F0002665988071D0013AAA85D2E61A6832624D
:10980000B3F90420B284224ADFED227AD268B26230
:1098100094ED127A0020002177EE877AA0641980F7
:10982000B28BFDEEE77A322AC6ED0B7A00F0828029
:1098300096ED0C7AD4ED137AD4ED146AE064B8EEA8
:10984000C77A012A37EE277AD6ED0D7A5980F8EEDD
:10985000E77ABDEEC77A77EEA67A2065FDEEE77A65
:10986000998086ED0C7AC6ED0D7A74D0013AB283F8
:1098700064E700BF10150010D8110010B4A6002036
:109880008205002000AC002094F100201F85EB51E0
:1098900008A7002000000000D4ED126A94ED137AAE
:1098A000D4ED147A354EFDEEE66ABDEEC77AFDEED4
:1098B000E77A00200021A064C6ED046A198086EDD5
:1098C000057AE0645980C6ED067A2065998092E7B2
:1098D000D6ED0B7AF8EEE77A9AE717EE906ADFF8A2
:1098E000A4E0B4F80C80C8368EFB061916EE90CAB8
:1098F000F11717EE107AC1EBE9110CF1C80CA1EBCE
:1099000008019980C8378EFB0C614FEAEC7CCCEBE8
:10991000E11C8EFB071EFF17C7EBEE17A3F800C074
:109920005F80174BC3F80A20D881F9F787F9AA8D11
:10993000AB6A60E794ED137AD4ED147AE064BDEE7F
:10994000C77AFDEEE77A598086ED0C7A2065C6ED80
:109950000D7A99808AE70B2086F8392086F838102E
:1099600008F09EFCAB6A326A1A60B6F924209A802D
:10997000034AB16AD160B28B78E700BF94F100204E
:1099800008A700201F85EB5138B5074C074DAC42A6
:1099900003D3074B01221A7038BDD4E90210A28804
:1099A00052F0ACFF1C34F2E734F30708F0FC070870
:1099B00098A100202DE9F04F0C4695B0344905469A
:1099C00020461746FDF7F4FF064600284FD13149DF
:1099D0002046FDF7EDFF064600284AD12E492046D5
:1099E000FDF7E6FF0646002845D12C492046FDF745
:1099F000DFFF0646002840D120462949FDF7D8FF61
:109A00000028064612BF0824264601240FB144F060
:109A1000100424493046FDF7CBFF80B344F0200406
:109A2000214B1B780BB9FFF7AFFFF7F7F1F814F0F4
:109A3000090F00F049831D48F9F7CCFA0020FEF722
:109A40001DF814F4807306933CD11948F9F7C2FA53
:109A50001848F9F7B9FA04F01803182B05D116487D
:109A6000F9F7B8FA1548F9F7AFFA01232BE001240A
:109A7000CCE70224CAE70424C8E78124C6E71049DA
